:0200000460009A
:100000004643464200000156000000000103030081
:1000100000000000000000000000000000000000E0
:1000200000000000000000000000000000000000D0
:1000300000000000000000000000000000000000C0
:1000400000000000010408000000000000000000A3
:100050000000800000000000000000000000000020
:100060000000000000000000000000000000000090
:100070000000000000000000000000000000000080
:10008000EB04180A063204260000000000000000FD
:10009000050404240000000000000000000000002F
:1000A0000000000000000000000000000000000050
:1000B0000604000000000000000000000000000036
:1000C0000000000000000000000000000000000030
:1000D00020041808000000000000000000000000DC
:1000E0000000000000000000000000000000000010
:1000F0000000000000000000000000000000000000
:10010000D8041808000000000000000000000000F3
:100110000204180804200000000000000000000095
:1001200000000000000000000000000000000000CF
:10013000600400000000000000000000000000005B
:1001400000000000000000000000000000000000AF
:10015000000000000000000000000000000000009F
:10016000000000000000000000000000000000008F
:10017000000000000000000000000000000000007F
:10018000000000000000000000000000000000006F
:10019000000000000000000000000000000000005F
:1001A000000000000000000000000000000000004F
:1001B000000000000000000000000000000000003F
:1001C000000100000010000001000000000000001D
:1001D000000001000000000000000000000000001E
:1001E000000000000000000000000000000000000F
:1001F00000000000000000000000000000000000FF
:10020000FFFFFFFFFFFFFFFFFFFFFFFFFFFFFFFFFE
:10021000FFFFFFFFFFFFFFFFFFFFFFFFFFFFFFFFEE
:10100000D100204327140060000000000000000011
:10101000201000600010006000A4016000000000CB
:101020000000006000B0010000000000FFFFFFFFB3
:10103000FFFFFFFFFFFFFFFFFFFFFFFFFFFFFFFFC0
:10104000FFFFFFFFFFFFFFFFFFFFFFFFFFFFFFFFB0
:10105000FFFFFFFFFFFFFFFFFFFFFFFFFFFFFFFFA0
:10106000FFFFFFFFFFFFFFFFFFFFFFFFFFFFFFFF90
:10140000884207D0904205D251F8043B40F8043B93
:101410008242F9D87047884204D2002340F8043B46
:101420008142FBD870472DE9F843644A644B5A6403
:10143000644A1A644FF42A029A63634B9D46BFF3D1
:101440004F8FBFF36F8F00F023FA604B0822604983
:101450006048C3F85421604AFFF7D2FF5F4A6049F1
:101460006048FFF7CDFF60496048FFF7D4FF4FF4B5
:1014700070025F4B5F491A6000235F4A42F82310F5
:1014800001335D4DB02BF9D15C4B80215C4A03F8F0
:10149000011B9342FBD14D4C4FF08037594A5A4BB8
:1014A000DFF89C91DFF89C811D60C4F80471C4F8DA
:1014B0000091C4F8F470C4F8F0801368534E43F4FC
:1014C000E02313604FF0FF32F36923F07F0343F012
:1014D0004003F361736A23F07F0343F040037362B8
:1014E000374B9A66DA661A675A6700F0D4F9484BA8
:1014F0006322AB63474BEB630025474B1A60032223
:101500005D6043F8042C454AC3F80C2D444A136827
:1015100043F080731360434A136843F00103136080
:10152000414B1A68414B1A6000F06EFBC4F804711D
:101530003F48C4F80091C4F8F470C4F8F08000F09B
:10154000FFFCF36E43F44053F3663A4B1D60C3F85F
:101550000851C3F81851C3F82851C3F8385103F59E
:10156000A0239A6BD20708D4334A5A6542F6156213
:101570001A659A6B42F001029A639A6842F001126E
:101580009A6000F0F7F900F097FC00F0E9FC00F039
:1015900069FB00F07EF9294A1368284C132BFBD90C
:1015A00000F0EEFB2368B3F5967FFBD300F072F9F1
:1015B00000F0D2FC00F0BCFC30BFFDE7BFAAAAAA35
:1015C00000C00A40070020000080062000800D4077
:1015D0009854006000000000A0100100C03E0020F0
:1015E0003C65016000000020E0870120C03E002033
:1015F00088ED00E085E60000003C002000E400E00B
:10160000A0E400E024ED00E008ED00E000C00F40A1
:101610006DF8000071F8000014E000E000002020E8
:10162000FCED00E0001000E0041000E0B07B0020C2
:10163000002CA330004008400000C056B47B0020BE
:101640001B1018200C0D1113F8B58F005C4B0C46C5
:1016500038461A6000F088FC5A4B054618601E4652
:1016600020B92021584800F053FCA4E03A4600215C
:1016700000F06EFC25F01F033D44BFF34F8F534A2B
:10168000136020339D42FBD8BFF34F8FBFF36F8FA2
:101690004F4B32681A604F4B4F4A1C804F4B1A60B9
:1016A0004F4AD36F43F44023D3674E4B4E4A1A67D9
:1016B0004FF43162C3F8802042F21072C3F89020D8
:1016C0001A6F22F480521A67196F464A0029FBDA12
:1016D000D2F870314FF48035444923F40003444874
:1016E000444E23F40043C2F87031136F23F4803367
:1016F000136702F51032D36923F4406343F40063A7
:10170000D361936A23F4FF7323F0010343F0F903D9
:101710009362A2F5A022536823F4002323F0070369
:1017200043F4002353600022334B1A66DA601961D8
:1017300032495D619861D961C3F8E020C3F88C201B
:10174000C3F89060C3F89450C3F898000320C3F81E
:101750009C102B49C1F82801C1F82401C1F880016F
:10176000D3F88810274841F01041C3F88810264963
:1017700099602649C1F8200125484FF08075056021
:1017800080F883237F20234A1070234AC1F8582110
:10179000D021224A224811704021A2F23E3211602B
:1017A00016219A6842F480729A6000F0B1FB2146DB
:1017B0001C4800F0C9FB1B48BDE8F84000F0B0BB76
:1017C000C0650020004200205634002070EF00E089
:1017D000FC650020E27B002020403840003B0020D8
:1017E00000C00F4000800D401B2011000100004789
:1017F000130F01000100000700403840000F0F0FD9
:1018000000801F402100000001000090003C0020EB
:1018100004E100E038E400E07500000046E400E088
:1018200077340020883A0020024B186808B100F095
:1018300083BB7047004200200004084B012200F4E3
:101840007020C3F8A010C3F8A400C3F8B0205A69F0
:10185000D207FCD50122014B5A61704700402A4053
:10186000094B0A4AC3F8A000C3F8A4200122C3F818
:10187000B0205969044AC907FBD5D2F800012123D9
:1018800080B25361704700BF00402A40040003004B
:1018900070477047704710B5214A0020214C102333
:1018A000214920601360214B1960112111602049EA
:1018B0001960122111601F4919601F4911601F49E9
:1018C00019601F4911601F4919601F4941F0150136
:1018D00011601E49196001F181510D3111601C49DF
:1018E00019601C4911601C4919601C4911601C4990
:1018F00019601C4911601C4A1A6001232360BFF360
:101900004F8FBFF36F8F194B1860BFF34F8FBFF32B
:101910006F8F174A136843F44033136010BD00BF44
:101920009CED00E094ED00E03F000010A0ED00E031
:101930002500080309001000130020002100020701
:101940001400002025000813E08701200900001082
:1019500027000B131700004033001013180000601D
:101960002F000B07190000702F000B1350EF00E041
:1019700014ED00E073B58F4B4FF400548E4A8F493D
:10198000C3F85C22C3F8601248F20C71C3F86422F9
:10199000A2F53042C3F8682202F5E042C3F86C2297
:1019A000C3F87022C3F87422C3F878221822DA66CA
:1019B0001A675A679A67DA67C3F88020C3F88420E9
:1019C000C3F888200122C3F82C27C3F83027C3F8B6
:1019D0003427C3F83827C3F83C27C3F85027784A80
:1019E000936923F0604323F4407343F0204343F4AE
:1019F00040739361D2F8843043F00C03C2F8843012
:101A0000704B1A6842F002021A601A6811406E4A5E
:101A10000A436E491A604FF0FF325A6002F57702AE
:101A2000886802F56052024042F000529A60DA681B
:101A300022F07802DA60664A186A024042F00042F8
:101A400042F040021A62624A186A0240614842F05B
:101A5000004242F040025A625F4A9A62DA62D1F86A
:101A6000B82022F03F0242F00102C3F8B820D1F8BA
:101A7000BC2040F2056122F03F0242F00102C3F8AF
:101A8000BC2000221A611C661867C3F880105C66CF
:101A90005867C3F884101968504821F00201196092
:101AA0004F4999610221D9614E4941F8042B814285
:101AB000FBD11A6842F001021A60424A1468414B95
:101AC00014F00104FAD1464A0226214620469A61C2
:101AD00040F2F562DE61C3F8002240F26642C3F8CC
:101AE000102240F29942C3F820223F4AC3F8302224
:101AF00042F20142C3F8342240F23542C3F8402298
:101B00003A4AC3F850223A4AC3F85422394AC3F831
:101B1000602242F20122C3F86422FFF78DFE2146C3
:101B20000120FFF789FE21463046FFF785FE20465B
:101B3000FFF796FE45F60D530546984231D12146F2
:101B40000420FFF779FE20464FF400012A4CFFF7EE
:101B500073FE4FF400010120FFF76EFE4FF4000109
:101B60003046FFF769FE4FF40000FFF779FEA84208
:101B700007D14FF400010420FFF75EFE102323700D
:101B800001E0082323701D4900231D4A2078521AC2
:101B90000093012302EB00521A4800F0E9F902B069
:101BA00070BD10222146174802B0BDE8704000F019
:101BB000CFB900BF00801F40F9B00100F91001004B
:101BC00000C00F4000402A401200FFFF00802A4062
:101BD00000FFF07C63000200FF000F8300432A40F7
:101BE000F05AF05A00422A409F041830EB06180AB7
:101BF000063201263806180A088700200000007007
:101C00000000007084870120F0B5154B40204FF490
:101C100080314FF480544FF400554FF4404643F266
:101C200042071A6912F0020F03D09E6159619F6149
:101C3000F7E712F4005F01D15D61F2E712F4805F13
:101C400001D15C61EDE7002AEBDA12F4803F01D0AC
:101C50009961E6E7520601D45861E2E7F0BD00BFA2
:101C600000800D40394AB3EE096A394813689FED88
:101C7000395A23F0010310B513600323364C136166
:101C8000364BD3F8E030D9B2016007EE901AC3F3B7
:101C90000B201B0DB8EEE77A314907EE900A206061
:101CA000F8EEE76A07EE903A37EE455A2D4BF8EE1C
:101CB000E77A37EE466A77EEE67A81ED006A25EE3E
:101CC000275AC3ED007A1368C5EE065A75EEA65A78
:101CD000FCEEE55A15EE901ADFED235A37EE657AE1
:101CE00043EA0153136027EE277A204B66EE277AEA
:101CF000D2F81011C7EE065A35EEA67ABCEEC77AB6
:101D000017EE100A87EE867A03EA00430B43C2F807
:101D10001031D2F8101177EE267AFCEEE77A17EE42
:101D2000903AC3F30B030B43C2F81031136843F02E
:101D30000203136000220E4B1A700E4A0E4BC3F8BA
:101D4000402101220D4B1A6010BD00BF80810D4063
:101D5000A07B00200000AA429C7B002000441F4082
:101D6000A47B0020A87B00200000B4420000FF0FED
:101D700040E400E029E80000003C002008E100E029
:101D800038B540F661722D4BC3F8202100F0C4F83D
:101D90002B4A2C49D2F8803043F00303C2F880303C
:101DA00040F20442284BC3F86021284A10680140E1
:101DB00019B9D3F8A811890718D04FF00041516321
:101DC000D3F8402142F00202C3F840211E4AD2F863
:101DD00040319B07FBD44FF400321D4B19201A6091
:101DE0004FF00042194B9A6300F09EF8174B002108
:101DF0004FF08042174D144C9A63284619600A230D
:101E00004FF42072C4F8A83100F0A2F84FF4810317
:101E1000114A2B604FF480032B6440F24313C4F843
:101E20005851C4F848310D4BC3F804220C4B4FF401
:101E300000321A600123C4F8403138BD00800D40E3
:101E400000C00F40001C1E0000002E4000900D40FE
:101E50008CE200E000000020E5EA0000003C0020E9
:101E60000CE100E008B50E4B1B6E9B0701D4FBBED6
:101E700016E072B600220B4BC3F84021A3F50D13F8
:101E8000094A1A64A3F1FF53A3F52B239D46BFF320
:101E90004F8F064B06480360064B1B689B689847AC
:101EA00000441F4000002E4003002000000012EB01
:101EB000008020201C0020000F4BDA6E42F44032DC
:101EC000DA66DA6E42F44072DA66A3F5603340F205
:101ED00037625A64A0229A649A6C1206FCD4074BAB
:101EE00040F237625A64A0229A649A6C12F080021F
:101EF000FBD1034B1A70704700C00F4000800C40AC
:101F0000FF860020F8B500BFF8BC08BC9E467047AD
:101F10005FF800F0D1F400005FF800F041F000003D
:101F20005FF800F02DFA00005FF800F065E50000B2
:101F30005FF800F025FC00005FF800F045020100AA
:101F40005FF800F03DFD00005FF800F0EBFA0000E4
:101F50005FF800F0C5E400005FF800F0E90101005F
:101F60005FF800F0790001005FF800F03502010031
:101F70005FF800F03701010025010000391E000064
:101F8000953E000099490000554F0000D58800009B
:101F9000090180961180FF3A81550A3601082A040A
:101FA000000000F02B040000014021800A13800A89
:101FB0002980FF0000000000000000000000000079
:101FC0000000000000000000000000000000000011
:101FD0000000000000000000000000000000000001
:101FE00000000000000000000000000000000000F1
:101FF00000000000000000000000000000000000E1
:1020000000000000000000000000000000000000D0
:1020100000000000000000000000000000000000C0
:1020200000000000000000000000000000000000B0
:102030000000007F41414141417F000027312721BD
:1020400071000000774177117100000077417741FE
:10205000710000001751774141000000771177416E
:1020600071000000771177517100000077414741FE
:102070004100000077517751710000000020243E9C
:1020800004000000594B5B4BD90000000000000029
:102090000000000000000000000000000000000040
:1020A0000000000000000000000000000000000030
:1020B0000000000000000000000000183C3C181860
:1020C000001800363600000000000036367F367FEC
:1020D0003636000C3E031E301F0C00006333180C14
:1020E0006663001C361C6E3B336E00060603000060
:1020F000000000180C0606060C1800060C1818182C
:102100000C060000663CFF3C660000000C0C3F0C17
:102110000C000000000000000C0C060000003F0056
:1021200000000000000000000C0C006030180C06DD
:102130000301003E63737B6F673E000C0E0C0C0CBA
:102140000C3F001E33301C06333F001E33301C3062
:10215000331E00383C36337F3078003F031F303069
:10216000331E001C06031F33331E003F3330180C90
:102170000C0C001E33331E33331E001E33333E302F
:10218000180E00000C0C00000C0C00000C0C0000E1
:102190000C0C06180C0603060C180000003F00008B
:1021A0003F0000060C1830180C06001E3330180CC7
:1021B000000C003E637B7B7B031E000C1E33333F11
:1021C0003333003F66663E66663F003C66030303AA
:1021D000663C001F36666666361F007F46161E1672
:1021E000467F007F46161E16060F003C66030373EB
:1021F000667C003333333F333333001E0C0C0C0C3E
:102200000C1E007830303033331E006766361E36C1
:102210006667000F06060646667F0063777F7F6B62
:1022200063630063676F7B736363001C3663636380
:10223000361C003F66663E06060F001E3333333BF6
:102240001E38003F66663E366667001E33070E384E
:10225000331E003F2D0C0C0C0C1E00333333333374
:10226000333F0033333333331E0C006363636B7FC0
:102270007763006363361C1C3663003333331E0CF4
:102280000C1E007F6331184C667F001E0606060692
:10229000061E0003060C18306040001E181818189F
:1022A000181E00081C36630000000000000000003B
:1022B0000000FF0C0C18000000000000001E303E63
:1022C000336E000706063E66663B0000001E3303C1
:1022D000331E003830303E33336E0000001E333F73
:1022E000031E001C36060F06060F0000006E333377
:1022F0003E301F0706366E666667000C000E0C0C3B
:102300000C1E00300030303033331E070666361E98
:102310003667000E0C0C0C0C0C1E000000337F7F87
:102320006B630000001F333333330000001E333370
:10233000331E0000003B66663E060F00006E33331E
:102340003E307800003B6E66060F0000003E031E24
:10235000301F00080C3E0C0C2C18000000333333E7
:10236000336E0000003333331E0C000000636B7FBC
:102370007F3600000063361C3663000000333333C1
:102380003E301F00003F190C263F00380C0C070C94
:102390000C38001818180018181800070C0C380C06
:1023A0000C07006E3B000000000000000000000071
:1023B0000000001C224A564C201E001824427E4277
:1023C0004242007C22223C22227C001C22404040CF
:1023D000221C0078242222222478007E404078406B
:1023E000407E007E404078404040001C22404E42EB
:1023F000221C004242427E424242001C0808080859
:10240000081C000E04040404443800424448704888
:102410004442004040404040407E0042665A5A429A
:102420004242004262524A4642420018244242421C
:102430002418007C42427C40404000182442424A1A
:10244000241A007C42427C484442003C42403C0208
:10245000423C003E08080808080800424242424246
:10246000423C0042424224241818004242425A5A36
:1024700066420042422418244242002222221C08C2
:102480000808007E02041820407E003C2020202006
:10249000203C000C10103C10706E003C040404043E
:1024A000043C0000081C2A08080808000010207FCF
:1024B00020100000000000000000000808080800CC
:1024C000000800242424000000000024247E247E30
:1024D000242400081E281C0A3C080000626408101E
:1024E000264600304848304A443A000408100000AC
:1024F000000000040810101008040020100808084C
:10250000102000082A1C3E1C2A08000008083E086B
:1025100008000000000000000808100000007E0015
:10252000000000000000000018180000020408105D
:102530002040003C42465A62423C000818280808E5
:10254000083E003C42020C30407E003C42021C022D
:10255000423C00040C14247E0404007E40780402F3
:102560004438001C20407C42423C007E420408105B
:102570001010003C42423C42423C003C42423E027F
:1025800004380000000800000800000000080000F7
:102590000808100E18306030180E0000007E007E13
:1025A00000000070180C060C1870003C42020C1061
:1025B00000100000000000FF000000081C3E7F7FAC
:1025C0001C3E001010101010101010000000FF0032
:1025D0000000000000FF000000000000FF000000FD
:1025E0000000000000000000FF000020202020204C
:1025F000202020040404040404040400000000E07B
:10260000100808080808040300000008080810E083
:1026100000000080808080808080FF804020100843
:102620000402010102040810204080FF80808080A5
:10263000808080FF01010101010101003C7E7E7E5E
:102640007E3C00000000000000FF00367F7F7F3EE0
:102650001C08004040404040404040000000000353
:102660000408088142241818244281003C42424256
:10267000423C00081C2A772A0808000202020202D3
:10268000020202081C3E7F3E1C080008080808FFE2
:10269000080808A050A050A050A05008080808083A
:1026A0000808080000013E54141400FF7F3F1F0F6C
:1026B0000703010000000000000000F0F0F0F0F05F
:1026C000F0F0F000000000FFFFFFFFFF000000003F
:1026D00000000000000000000000FF80808080807B
:1026E000808080AA55AA55AA55AA55010101010169
:1026F00001010100000000AA55AA55FFFEFCF8F0F8
:10270000E0C0800303030303030303080808080F62
:10271000080808000000000F0F0F0F080808080F36
:1027200000000000000000F8080808000000000099
:1027300000FFFF000000000F08080808080808FF55
:1027400000000000000000FF08080808080808F85A
:10275000080808C0C0C0C0C0C0C0C0E0E0E0E0E001
:10276000E0E0E00707070707070707FFFF00000093
:10277000000000FFFFFF000000000000000000005C
:10278000FFFFFF01010101010101FF00000000F056
:10279000F0F0F00F0F0F0F0000000008080808F815
:1027A000000000F0F0F0F000000000F0F0F0F00F9A
:1027B0000F0F0FE3DDB5A9B3DFE1FFE7DBBD81BD9F
:1027C000BDBDFF83DDDDC3DDDD83FFE3DDBFBFBF57
:1027D000DDE3FF87DBDDDDDDDB87FF81BFBF87BF9B
:1027E000BF81FF81BFBF87BFBFBFFFE3DDBFB1BDFB
:1027F000DDE3FFBDBDBD81BDBDBDFFE3F7F7F7F76D
:10280000F7E3FFF1FBFBFBFBBBC7FFBDBBB78FB71C
:10281000BBBDFFBFBFBFBFBFBF81FFBD99A5A5BDEA
:10282000BDBDFFBD9DADB5B9BDBDFFE7DBBDBDBD48
:10283000DBE7FF83BDBD83BFBFBFFFE7DBBDBDB52A
:10284000DBE5FF83BDBD83B7BBBDFFC3BDBFC3FD1C
:10285000BDC3FFC1F7F7F7F7F7F7FFBDBDBDBDBDBE
:10286000BDC3FFBDBDBDDBDBE7E7FFBDBDBDA5A5AE
:1028700099BDFFBDBDDBE7DBBDBDFFDDDDDDE3F702
:10288000F7F7FF81FDFBE7DFBF81FFC3DFDFDFDF9E
:10289000DFC3FFF3EFEFC3EF8F91FFC3FBFBFBFB46
:1028A000FBC3FFFFF7E3D5F7F7F7F7FFFFEFDF8095
:1028B000DFEFFFFFFFFFFFFFFFFFFFF7F7F7F7FF78
:1028C000FFF7FFDBDBDBFFFFFFFFFFDBDB81DB81F4
:1028D000DBDBFFF7E1D7E3F5C3F7FFFF9D9BF7EFE6
:1028E000D9B9FFCFB7B7CFB5BBC5FFFBF7EFFFFF38
:1028F000FFFFFFFBF7EFEFEFF7FBFFDFEFF7F7F778
:10290000EFDFFFF7D5E3C1E3D5F7FFFFF7F7C1F737
:10291000F7FFFFFFFFFFFFFFF7F7EFFFFFFF81FF6D
:10292000FFFFFFFFFFFFFFFFE7E7FFFFFDFBF7EF05
:10293000DFBFFFC3BDB9A59DBDC3FFF7E7D7F7F75D
:10294000F7C1FFC3BDFDF3CFBF81FFC3BDFDE3FDF5
:10295000BDC3FFFBF3EBDB81FBFBFF81BF87FBFD0F
:10296000BBC7FFE3DFBF83BDBDC3FF81BDFBF7EF87
:10297000EFEFFFC3BDBDC3BDBDC3FFC3BDBDC1FD43
:10298000FBC7FFFFFFF7FFFFF7FFFFFFFFF7FFFFAB
:10299000F7F7EFF1E7CF9FCFE7F1FFFFFF81FF816F
:1029A000FFFFFF8FE7F3F9F3E78FFFC3BDFDF3EF01
:1029B000FFEFFFFFFFFFFF00FFFFFFF7E3C1808096
:1029C000E3C1FFEFEFEFEFEFEFEFEFFFFFFF00FFF0
:1029D000FFFFFFFFFF00FFFFFFFFFFFF00FFFFFF05
:1029E000FFFFFFFFFFFFFFFF00FFFFDFDFDFDFDF96
:1029F000DFDFDFFBFBFBFBFBFBFBFBFFFFFFFF1F47
:102A0000EFF7F7F7F7F7FBFCFFFFFFF7F7F7EF1F1D
:102A1000FFFFFF7F7F7F7F7F7F7F007FBFDFEFF73D
:102A2000FBFDFEFEFDFBF7EFDFBF7F007F7F7F7FBB
:102A30007F7F7F00FEFEFEFEFEFEFEFFC3818181E2
:102A400081C3FFFFFFFFFFFFFF00FFC9808080C140
:102A5000E3F7FFBFBFBFBFBFBFBFBFFFFFFFFFFCAD
:102A6000FBF7F77EBDDBE7E7DBBD7EFFC3BDBDBD8A
:102A7000BDC3FFF7E3D588D5F7F7FFFDFDFDFDFDED
:102A8000FDFDFDF7E3C180C1E3F7FFF7F7F7F700BE
:102A9000F7F7F75FAF5FAF5FAF5FAFF7F7F7F7F746
:102AA000F7F7F7FFFFFEC1ABEBEBFF0080C0E0F0F4
:102AB000F8FCFEFFFFFFFFFFFFFFFF0F0F0F0F0FE1
:102AC0000F0F0FFFFFFFFF0000000000FFFFFFFFE1
:102AD000FFFFFFFFFFFFFFFFFFFF007F7F7F7F7F85
:102AE0007F7F7F55AA55AA55AA55AAFEFEFEFEFE77
:102AF000FEFEFEFFFFFFFF55AA55AA000103070FC8
:102B00001F3F7FFCFCFCFCFCFCFCFCF7F7F7F7F03C
:102B1000F7F7F7FFFFFFFFF0F0F0F0F7F7F7F7F048
:102B2000FFFFFFFFFFFFFF07F7F7F7FFFFFFFFFFC5
:102B3000FF0000FFFFFFFFF0F7F7F7F7F7F7F700E9
:102B4000FFFFFFFFFFFFFF00F7F7F7F7F7F7F707C4
:102B5000F7F7F73F3F3F3F3F3F3F3F1F1F1F1F1FFD
:102B60001F1F1FF8F8F8F8F8F8F8F80000FFFFFF4B
:102B7000FFFFFF000000FFFFFFFFFFFFFFFFFFFF62
:102B8000000000FEFEFEFEFEFEFE00FFFFFFFF0F48
:102B90000F0F0FF0F0F0F0FFFFFFFFF7F7F7F70769
:102BA000FFFFFF0F0F0F0FFFFFFFFF0F0F0F0FF0C4
:102BB000F0F0F01C224A564C201E00000038043C65
:102BC000443A0040405C6242625C0000003C42408B
:102BD000423C0002023A4642463A0000003C427E35
:102BE000403C000C12107C1010100000003A4646C9
:102BF0003A023C40405C6242424200080018080829
:102C0000081C0004000C04040444384040444850AC
:102C10006844001808080808081C000000764949A4
:102C200049490000005C624242420000003C4242CE
:102C3000423C0000005C62625C404000003A464654
:102C40003A020200005C624040400000003E403C0E
:102C5000027C0010107C1010120C00000042424256
:102C6000463A00000042424224180000004149490F
:102C70004936000000422418244200000042424627
:102C80003A023C00007E0418207E003C20202020D8
:102C9000203C000C10103C10706E003C0404040436
:102CA000043C0000081C2A08080808000010207FC7
:102CB00020100000000000000000000808080800C4
:102CC000000800242424000000000024247E247E28
:102CD000242400081E281C0A3C0800006264081016
:102CE000264600304848304A443A000408100000A4
:102CF0000000000408101010080400201008080844
:102D0000102000082A1C3E1C2A08000008083E0863
:102D100008000000000000000808100000007E000D
:102D20000000000000000000181800000204081055
:102D30002040003C42465A62423C000818280808DD
:102D4000083E003C42020C30407E003C42021C0225
:102D5000423C00040C14247E0404007E40780402EB
:102D60004438001C20407C42423C007E4204081053
:102D70001010003C42423C42423C003C42423E0277
:102D800004380000000800000800000000080000EF
:102D90000808100E18306030180E0000007E007E0B
:102DA00000000070180C060C1870003C42020C1059
:102DB00000100000000000FF0000001824427E42C6
:102DC0004242007C22223C22227C001C22404040C5
:102DD000221C0078242222222478007E4040784061
:102DE000407E007E404078404040001C22404E42E1
:102DF000221C004242427E424242001C080808084F
:102E0000081C000E0404040444380042444870487E
:102E10004442004040404040407E0042665A5A4290
:102E20004242004262524A46424200182442424212
:102E30002418007C42427C40404000182442424A10
:102E4000241A007C42427C484442003C42403C02FE
:102E5000423C003E0808080808080042424242423C
:102E6000423C0042424224241818004242425A5A2C
:102E700066420042422418244242002222221C08B8
:102E80000808007E02041820407E0008080808FF99
:102E9000080808A050A050A050A050080808080832
:102EA000080808CCCC3333CCCC3333CC663399CC44
:102EB0006633990000000000000000F0F0F0F0F030
:102EC000F0F0F000000000FFFFFFFFFF0000000037
:102ED00000000000000000000000FF808080808073
:102EE000808080AA55AA55AA55AA55010101010161
:102EF00001010100000000AA55AA55993366CC993A
:102F00003366CC0303030303030303080808080F15
:102F1000080808000000000F0F0F0F080808080F2E
:102F200000000000000000F8080808000000000091
:102F300000FFFF000000000F08080808080808FF4D
:102F400000000000000000FF08080808080808F852
:102F5000080808C0C0C0C0C0C0C0C0E0E0E0E0E0F9
:102F6000E0E0E00707070707070707FFFF0000008B
:102F7000000000FFFFFF0000000000000000000054
:102F8000FFFFFF010244485060400000000000F0D5
:102F9000F0F0F00F0F0F0F0000000008080808F80D
:102FA000000000F0F0F0F000000000F0F0F0F00F92
:102FB0000F0F0FE3DDB5A9B3DFE1FFFFFFC7FBC3D1
:102FC000BBC5FFBFBFA39DBD9DA3FFFFFFC3BDBF8B
:102FD000BDC3FFFDFDC5B9BDB9C5FFFFFFC3BD81C1
:102FE000BFC3FFF3EDEF83EFEFEFFFFFFFC5B9B90D
:102FF000C5FDC3BFBFA39DBDBDBDFFF7FFE7F7F78D
:10300000F7E3FFFBFFF3FBFBFBBBC7BFBFBBB7AFE8
:1030100097BBFFE7F7F7F7F7F7E3FFFFFF89B6B6D0
:10302000B6B6FFFFFFA39DBDBDBDFFFFFFC3BDBD86
:10303000BDC3FFFFFFA39D9DA3BFBFFFFFC5B9B9E0
:10304000C5FDFDFFFFA39DBFBFBFFFFFFFC1BFC306
:10305000FD83FFEFEF83EFEFEDF3FFFFFFBDBDBD9E
:10306000B9C5FFFFFFBDBDBDDBE7FFFFFFBEB6B6C5
:10307000B6C9FFFFFFBDDBE7DBBDFFFFFFBDBDB98D
:10308000C5FDC3FFFF81FBE7DF81FFC3DFDFDFDFBC
:10309000DFC3FFF3EFEFC3EF8F91FFC3FBFBFBFB3E
:1030A000FBC3FFFFF7E3D5F7F7F7F7FFFFEFDF808D
:1030B000DFEFFFFFFFFFFFFFFFFFFFF7F7F7F7FF70
:1030C000FFF7FFDBDBDBFFFFFFFFFFDBDB81DB81EC
:1030D000DBDBFFF7E1D7E3F5C3F7FFFF9D9BF7EFDE
:1030E000D9B9FFCFB7B7CFB5BBC5FFFBF7EFFFFF30
:1030F000FFFFFFFBF7EFEFEFF7FBFFDFEFF7F7F770
:10310000EFDFFFF7D5E3C1E3D5F7FFFFF7F7C1F72F
:10311000F7FFFFFFFFFFFFFFF7F7EFFFFFFF81FF65
:10312000FFFFFFFFFFFFFFFFE7E7FFFFFDFBF7EFFD
:10313000DFBFFFC3BDB9A59DBDC3FFF7E7D7F7F755
:10314000F7C1FFC3BDFDF3CFBF81FFC3BDFDE3FDED
:10315000BDC3FFFBF3EBDB81FBFBFF81BF87FBFD07
:10316000BBC7FFE3DFBF83BDBDC3FF81BDFBF7EF7F
:10317000EFEFFFC3BDBDC3BDBDC3FFC3BDBDC1FD3B
:10318000FBC7FFFFFFF7FFFFF7FFFFFFFFF7FFFFA3
:10319000F7F7EFF1E7CF9FCFE7F1FFFFFF81FF8167
:1031A000FFFFFF8FE7F3F9F3E78FFFC3BDFDF3EFF9
:1031B000FFEFFFFFFFFFFF00FFFFFFE7DBBD81BD6C
:1031C000BDBDFF83DDDDC3DDDD83FFE3DDBFBFBF4D
:1031D000DDE3FF87DBDDDDDDDB87FF81BFBF87BF91
:1031E000BF81FF81BFBF87BFBFBFFFE3DDBFB1BDF1
:1031F000DDE3FFBDBDBD81BDBDBDFFE3F7F7F7F763
:10320000F7E3FFF1FBFBFBFBBBC7FFBDBBB78FB712
:10321000BBBDFFBFBFBFBFBFBF81FFBD99A5A5BDE0
:10322000BDBDFFBD9DADB5B9BDBDFFE7DBBDBDBD3E
:10323000DBE7FF83BDBD83BFBFBFFFE7DBBDBDB520
:10324000DBE5FF83BDBD83B7BBBDFFC3BDBFC3FD12
:10325000BDC3FFC1F7F7F7F7F7F7FFBDBDBDBDBDB4
:10326000BDC3FFBDBDBDDBDBE7E7FFBDBDBDA5A5A4
:1032700099BDFFBDBDDBE7DBBDBDFFDDDDDDE3F7F8
:10328000F7F7FF81FDFBE7DFBF81FFF7F7F7F700F7
:10329000F7F7F75FAF5FAF5FAF5FAFF7F7F7F7F73E
:1032A000F7F7F73333CCCC3333CCCC3399CC66330C
:1032B00099CC66FFFFFFFFFFFFFFFF0F0F0F0F0F00
:1032C0000F0F0FFFFFFFFF0000000000FFFFFFFFD9
:1032D000FFFFFFFFFFFFFFFFFFFF007F7F7F7F7F7D
:1032E0007F7F7F55AA55AA55AA55AAFEFEFEFEFE6F
:1032F000FEFEFEFFFFFFFF55AA55AA66CC99336676
:10330000CC9933FCFCFCFCFCFCFCFCF7F7F7F7F079
:10331000F7F7F7FFFFFFFFF0F0F0F0F7F7F7F7F040
:10332000FFFFFFFFFFFFFF07F7F7F7FFFFFFFFFFBD
:10333000FF0000FFFFFFFFF0F7F7F7F7F7F7F700E1
:10334000FFFFFFFFFFFFFF00F7F7F7F7F7F7F707BC
:10335000F7F7F73F3F3F3F3F3F3F3F1F1F1F1F1FF5
:103360001F1F1FF8F8F8F8F8F8F8F80000FFFFFF43
:10337000FFFFFF000000FFFFFFFFFFFFFFFFFFFF5A
:10338000000000FEFDBBB7AF9FBFFFFFFFFFFF0FB9
:103390000F0F0FF0F0F0F0FFFFFFFFF7F7F7F70761
:1033A000FFFFFF0F0F0F0FFFFFFFFF0F0F0F0FF0BC
:1033B000F0F0F078E367E443424D42415349433033
:1033C000C841C71DCDF7C8A4CBBECB80D005CCA4C7
:1033D000C99FC870C827C91CC882C8D1C83AC92E9D
:1033E000C84AC92CD864E152E161E1B2D323D87F45
:1033F000CA9FCA56C89BC65DC685CA26E1BAE1C344
:10340000E17ACB41C639DCCCDC58DC00007DD39EB0
:10341000D371DF94E0EAD9EDDF61E268E2B1E20B5B
:10342000E30DD87CD765D4ADD78BD7ECD600D72C9D
:10343000D737D77969D87952D87B2ADA7B11DB7FE5
:103440007ADF50E8CF46E5CF7DB3DF5AD3CE64159F
:10345000D0454EC4464FD24E4558D4444154C1493C
:103460004E505554A3494E5055D44449CD52454130
:10347000C44C45D4474F54CF5255CE49C6524553FC
:10348000544F52C5474F5355C25245545552CE52D0
:1034900045CD53544FD04FCE574149D44C4F41C4E2
:1034A000534156C55645524946D94445C6504F4BDF
:1034B000C55052494E54A35052494ED4434F4ED456
:1034C0004C4953D4434CD2434DC45359D34F504528
:1034D000CE434C4F53C54745D44E45D7544142A8DF
:1034E00054CF46CE535043A8544845CE4E4FD453A4
:1034F0005445D0ABADAAAFDE414EC44FD2BEBDBC29
:103500005347CE494ED44142D35553D24652C5506B
:103510004FD35351D2524EC44C4FC74558D0434F4E
:10352000D35349CE5441CE4154CE504545CB4C4562
:10353000CE535452A45641CC4153C3434852A44C99
:10354000454654A45249474854A44D4944A447CF42
:1035500000544F4F204D414E592046494C45D346CB
:10356000494C45204F5045CE46494C45204E4F547E
:10357000204F5045CE46494C45204E4F5420464F93
:10358000554EC4444556494345204E4F5420505251
:103590004553454ED44E4F5420494E505554204625
:1035A000494CC54E4F54204F555450555420464910
:1035B0004CC54D495353494E472046494C45204E32
:1035C000414DC5494C4C4547414C20444556494323
:1035D00045204E554D4245D24E45585420574954EA
:1035E000484F555420464FD253594E5441D8524516
:1035F0005455524E20574954484F555420474F5325
:1036000055C24F5554204F4620444154C1494C4C5B
:103610004547414C205155414E544954D94F564588
:1036200052464C4FD74F5554204F46204D454D4F95
:1036300052D9554E44454627442053544154454D94
:10364000454ED4424144205355425343524950D4ED
:10365000524544494D27442041525241D94449568C
:103660004953494F4E204259205A4552CF494C4C5C
:103670004547414C204449524543D4545950452074
:103680004D49534D415443C8535452494E47205419
:103690004F4F204C4F4EC746494C4520444154C1E2
:1036A000464F524D554C4120544F4F20434F4D50A3
:1036B0004C45D843414E275420434F4E54494E5514
:1036C000C5554E44454627442046554E4354494F20
:1036D000CE5645524946D94C4F41C49EC1ACC1B5A6
:1036E000C1C2C1D0C1E2C1F0C1FFC110C225C23503
:1036F000C23BC24FC25AC26AC272C27FC290C29D4E
:10370000C2AAC2BAC2C8C2D5C2E4C2EDC200C30EC8
:10371000C31EC324C383C30D4F4B0D000D20455260
:10372000524F520020494E20000D0A524541445943
:103730002E0D0A000D0A425245414B00A0BAE8E89E
:10374000E8E8BD0101C981D021A54AD00ABD020126
:103750008549BD0301854ADD0301D007A549DD0286
:1037600001F0078A186912AAD0D8602008C48531F0
:10377000843238A55AE55F8522A8A55BE560AAE8F2
:1037800098F023A55A38E522855AB003C65B38A5C0
:1037900058E5228558B008C6599004B15A91588806
:1037A000D0F9B15A9158C65BC659CAD0F2600A69BD
:1037B0003EB0358522BAE422902E60C4349028D0E1
:1037C00004C533902248A2099848B557CA10FA2078
:1037D00026D5A2F7689561E830FA68A868C43490E5
:1037E00006D005C533B00160A2106C00038A0AAA96
:1037F000BD26C38522BD27C3852320CCFFA9008514
:103800001320D7CA2045CBA000B12248297F2047EA
:10381000CBC86810F4207AC6A969A0C3201ECBA427
:103820003AC8F00320C2DDA976A0C3201ECBA98030
:103830002090FF6C02032060C5867A847B20730091
:10384000AAF0F0A2FF863A90062079C54CE1C72085
:103850006BC92079C5840B2013C69044A001B15FC9
:103860008523A52D8522A5608525A55F88F15F1894
:10387000652D852D8524A52E69FF852EE560AA3846
:10388000A55FE52DA8B003E8C6251865229003C6FC
:103890002318B1229124C8D0F9E623E625CAD0F234
:1038A0002059C62033C5AD0002F08818A52D855AD1
:1038B000650B8558A42E845B9001C8845920B8C339
:1038C000A514A4158DFE018CFF01A531A432852D10
:1038D000842EA40B88B9FC01915F8810F82059C68A
:1038E0002033C54C80C4A52BA42C8522842318A08A
:1038F00001B122F01DA004C8B122D0FBC8986522F6
:10390000AAA0009122A5236900C8912286228523BE
:1039100090DD60A200200FE1C90DF00D9D0002E8CE
:10392000E05990F1A2174C37C44CCACA6C0403A6E4
:103930007AA004840FBD00021007C9FFF03EE8D052
:10394000F4C920F0378508C922F056240F702DC91C
:103950003FD004A999D025C9309004C93C901D845A
:1039600071A000840B88867ACAC8E8BD000238F9C5
:103970009EC0F0F5C980D030050BA471E8C899FB52
:1039800001B9FB01F03638E93AF004C949D00285A3
:103990000F38E955D09F8508BD0002F0DFC508F05B
:1039A000DBC899FB01E8D0F0A67AE60BC8B99DC048
:1039B00010FAB99EC0D0B4BD000210BE99FD01C678
:1039C0007BA9FF857A60A52BA62CA001855F866068
:1039D000B15FF01FC8C8A515D15F9018F00388D05B
:1039E00009A51488D15F900CF00A88B15FAA88B14C
:1039F0005FB0D71860D0FDA900A8912BC8912BA566
:103A00002B186902852DA52C6900852E208EC6A94C
:103A100000D02D20E7FFA537A43885338434A52DA9
:103A2000A42E852F843085318432201DC8A21986AA
:103A30001668A868A2FA9A489848A900853E851099
:103A40006018A52B69FF857AA52C69FF857B60909E
:103A500006F004C9ABD0E9206BC92013C620790059
:103A6000F00CC9ABD08E207300206BC9D08668687B
:103A7000A5140515D006A9FF85148515A001840F8E
:103A8000B15FF043202CC820D7CAC8B15FAAC8B123
:103A90005FC515D004E414F002B02C844920CDDDBC
:103AA000A920A449297F2047CBC922D006A50F49C8
:103AB000FF850FC8F011B15FD010A8B15FAAC8B1DF
:103AC0005F865F8560D0B54C74C46C060310D7C99F
:103AD000FFF0D3240F30CF38E97FAA8449A0FFCA72
:103AE000F008C8B99EC010FA30F5C8B99EC030B20F
:103AF0002047CBD0F5A980851020A5C9208AC3D046
:103B0000058A690FAA9A6868A90920FBC32006C91B
:103B10001898657A48A57B690048A53A48A53948B0
:103B2000A9A420FFCE208DCD208ACDA566097F25B2
:103B3000628562A98BA0C7852284234C43CEA9BC91
:103B4000A0D920A2DB207900C9A9D00620730020CB
:103B50008ACD202BDC2038CEA54A48A54948A9812A
:103B600048202CC8A57AA47BC002EAF004853D84D5
:103B70003EA000B17AD043A002B17A18D0034C4BDA
:103B8000C8C8B17A8539C8B17A853A98657A857A94
:103B90009002E67B6C080320730020EDC74CAEC793
:103BA000F03CE9809011C923B0170AA8B90DC048AC
:103BB000B90CC0484C73004CA5C9C93AF0D64C08A2
:103BC000CFC94BD0F9207300A9A420FFCE4CA0C8C8
:103BD00038A52BE901A42CB00188854184426020DE
:103BE000E1FFB00118D03CA57AA47BA63AE8F00C1E
:103BF000853D843EA539A43A853B843C6868A9810B
:103C0000A0C390034C69C44C74C4D017A21AA43E3C
:103C1000D0034C37C4A53D857A847BA53BA43C8565
:103C200039843A6008A9002090FF28D0034C59C677
:103C30002060C64C97C8A90320FBC3A57B48A57A82
:103C400048A53A48A53948A98D4820790020A0C840
:103C50004CAEC7206BC92009C938A539E514A53A6F
:103C6000E515B00B9838657AA67B9007E8B004A5F7
:103C70002BA62C2017C6901EA55FE901857AA560AA
:103C8000E900857B60D0FDA9FF854A208AC39AC9D7
:103C90008DF00BA20C2CA2114C37C44C08CF6868D5
:103CA000853968853A68857A68857B2006C99818C1
:103CB000657A857A9002E67B60A23A2CA20086079C
:103CC000A0008408A508A60785078608B17AF0E851
:103CD000C508F0E4C8C922D0F3F0E9209ECD2079D0
:103CE00000C989F005A9A720FFCEA561D00520094C
:103CF000C9F0BB207900B0034CA0C84CEDC7209E92
:103D0000D748C98DF004C989D091C665D004684CE4
:103D1000EFC7207300206BC9C92CF0EE6860A200C9
:103D200086148615B0F7E92F8507A5158522C919D0
:103D3000B0D4A5140A26220A262265148514A522C9
:103D40006515851506142615A514650785149002BA
:103D5000E6152073004C71C9208BD08549844AA98F
:103D6000B220FFCEA50E48A50D48209ECD682A2082
:103D700090CDD018681012201BDC20BFD1A000A568
:103D8000649149C8A5659149604CD0DB68A44AC0DC
:103D9000DFD04C20A6D6C906D03DA0008461846641
:103DA0008471201DCA20E2DAE671A471201DCA20A8
:103DB0000CDCAAF005E88A20EDDAA471C8C006D0B0
:103DC000DF20E2DA209BDCA664A463A5654CDBFF60
:103DD000B12220800090034C48D2E92F4C7EDDA018
:103DE00002B164C5349017D00788B164C533900E12
:103DF000A465C42E9008D00DA564C52DB007A56498
:103E0000A4654C68CAA000B1642075D4A550A45123
:103E1000856F8470207AD6A961A0008550845120D6
:103E2000DBD6A000B1509149C8B1509149C8B150FA
:103E30009149602086CA4CB5CB209ED7F005A92CAD
:103E400020FFCE0886132015E1284CA0CA2021CBE4
:103E5000207900F035F043C9A3F050C9A618F04B03
:103E6000C92CF037C93BF05E209ECD240D30DE20FA
:103E7000DDDD2087D42021CB203BCBD0D3A9009DF2
:103E80000002A2FFA001A513D010A90D2047CB244A
:103E9000131005A90A2047CB49FF603820F0FF988E
:103EA00038E90BB0FC49FF6901D016083820F0FF53
:103EB0008409209BD7C929D0592890068AE5099002
:103EC00005AAE8CAD0062073004CA2CA203BCBD07A
:103ED000F22087D420A6D6AAA000E8CAF0BCB1225E
:103EE0002047CBC8C90DD0F320E5CA4C28CBA51379
:103EF000F003A9202CA91D2CA93F2009E129FF606E
:103F0000A511F0113004A0FFD004A53FA4408539CD
:103F1000843A4C08CFA513F005A2184C37C4A90C5D
:103F2000A0CD201ECBA53DA43E857A847B6020A633
:103F3000D3C923D010207300209ED7A92C20FFCEF8
:103F40008613201BE1A201A002A9008D0102A94055
:103F5000200FCCA613D01360209ED7A92C20FFCE13
:103F60008613201BE120CECBA51320CCFFA2008618
:103F70001360C922D00B20BDCEA93B20FFCE20214B
:103F8000CB20A6D3A92C8DFF0120F9CBA513F00DD2
:103F900020B7FF2902F00620B5CB4CF8C8AD0002CF
:103FA000D01EA513D0E32006C94CFBC8A513D0062C
:103FB0002045CB203BCB4C60C5A641A442A9982C00
:103FC000A900851186438444208BD08549844AA565
:103FD0007AA47B854B844CA643A444867A847B20B8
:103FE0007900D0202411500C2021E18D0002A2FF85
:103FF000A001D00C3075A513D0032045CB20F9CB00
:10400000867A847B207300240D103124115009E836
:10401000867AA9008507F00C8507C922F007A93A1E
:104020008507A92C188508A57AA47B69009001C88A
:10403000208DD420E2D720DAC94C91CC20F3DCA526
:104040000E20C2C9207900F007C92CF0034C4DCBDB
:10405000A57AA47B85438444A54BA44C857A847BB4
:10406000207900F02D20FDCE4C15CC2006C9C8AA21
:10407000D012A20DC8B17AF06CC8B17A853FC8B130
:104080007AC8854020FBC8207900AAE083D0DC4CA8
:1040900051CCA543A444A61110034C27C8A000B1DD
:1040A00043F00BA513D007A9FCA0CC4C1ECB603F5E
:1040B00045585452412049474E4F5245440D003F08
:1040C0005245444F2046524F4D2053544152540DB7
:1040D00000D004A000F003208BD08549844A208AB8
:1040E000C3F005A20A4C37C49A8A186904486906C5
:1040F000852468A00120A2DBBABD09018566A54917
:10410000A44A2067D820D0DBA001205DDCBA38FDAE
:104110000901F017BD0F018539BD1001853ABD12A7
:1041200001857ABD1101857B4CAEC78A6911AA9AB7
:10413000207900C92CD0F12073002024CD209ECD01
:10414000182438240D3003B00360B0FDA2164C379C
:10415000C4A67AD002C67BC67AA20024488A48A99F
:104160000120FBC32083CEA900854D20790038E9CA
:10417000B19017C903B013C9012A4901454DC54D76
:104180009061854D2073004CBBCDA64DD02CB07BEB
:1041900069079077650DD0034C3DD669FF85220AEB
:1041A0006522A868D980C0B067208DCD482020CE78
:1041B00068A44B1017AAF056D05F460D8A2AA67A3B
:1041C000D002C67BC67AA01B854DD0D7D980C0B09F
:1041D0004890D9B982C048B981C0482033CEA54D96
:1041E0004CA9CD4C08CFA566BE80C0A8688522E644
:1041F000226885239848201BDCA56548A56448A54E
:104200006348A56248A561486C2200A0FF68F023BE
:10421000C964F003208DCD844B684A851268856996
:1042200068856A68856B68856C68856D68856E458C
:1042300066856FA561606C0A03A900850D20730077
:10424000B0034CF3DC2013D190034C28CFC9FFD02E
:104250000FA9A8A0CE20A2DB4C730082490FDAA1DF
:10426000C92EF0DEC9ABF058C9AAF0D1C922D00FCF
:10427000A57AA47B69009001C82087D44CE2D7C9F5
:10428000A8D013A018D03B20BFD1A56549FFA8A591
:104290006449FF4C91D3C9A5D0034CF4D3C9B49061
:1042A000034CA7CF20FACE209ECDA9292CA9282CDB
:1042B000A92CA000D17AD0034C7300A20B4C37C4B8
:1042C000A01568684CFACD38A564E900A565E9C079
:1042D0009008A987E564A9E3E56560208BD0856433
:1042E0008465A645A446A50DF026A9008570201476
:1042F000CF901CE054D018C0C9D0142084CF845E65
:10430000888471A006845DA0242068DE4C6FD46090
:10431000240E100DA000B164AAC8B164A88A4C9103
:10432000D32014CF902DE054D01BC049D025208439
:10433000CF98A2A04C4FDC20DEFF866484638565A5
:10434000A000846260E053D00AC054D00620B7FFBA
:104350004C3CDCA564A4654CA2DB0A48AA2073008F
:10436000E08F902020FACE209ECD20FDCE208FCD54
:1043700068AAA56548A564488A48209ED768A88A87
:10438000484CD6CF20F1CE68A8B9EABF8555B9EB25
:10439000BF85562054004C8DCDA0FF2CA000840B6F
:1043A00020BFD1A564450B8507A565450B85082071
:1043B000FCDB20BFD1A565450B2508450BA8A564EE
:1043C000450B2507450B4C91D32090CDB013A56E1E
:1043D000097F256A856AA969A000205BDCAA4C6177
:1043E000D0A900850DC64D20A6D68561866284635E
:1043F000A56CA46D20AAD6866C846DAA38E561F000
:1044000008A9019004A661A9FF8566A0FFE8C8CAB3
:10441000D007A666300F18900CB16CD162F0EFA2F5
:10442000FFB002A201E88A2A2512F002A9FF4C3C43
:10443000DC20FDCEAA2090D0207900D0F460A2002C
:10444000207900860C85452079002013D1B0034CDB
:1044500008CFA200860D860E20730090052013D190
:10446000900BAA20730090FB2013D1B0F6C924D082
:1044700006A9FF850DD010C925D013A510D0D0A94D
:1044800080850E054585458A0980AA2073008646E9
:10449000380510E928D0034CD1D1A0008410A52DF7
:1044A000A62E8660855FE430D004C52FF022A54596
:1044B000D15FD008A546C8D15FF07D8818A55F6997
:1044C0000790E1E8D0DCC9419005E95B38E9A560D7
:1044D0006848C92AD005A913A0DF60A545A446C92C
:1044E00054D00BC0C9F0EFC049D0034C08CFC9531A
:1044F000D004C054F0F5A52FA430855F8460A531A9
:10450000A432855A845B1869079001C8855884597C
:1045100020B8C3A558A459C8852F8430A000A5454C
:10452000915FC8A546915FA900C8915FC8915FC817
:10453000915FC8915FC8915FA55F186902A4609000
:1045400001C88547844860A50B0A6905655FA460BA
:104550009001C88558845960908000000020BFD128
:10456000A564A46560207300209ECD208DCDA56636
:10457000300DA561C9909009A9A5A0D1205BDCD020
:104580007A4C9BDCA50C050E48A50D48A000984868
:10459000A54648A5454820B2D16885456885466846
:1045A000A8BABD020148BD010148A5649D0201A54C
:1045B000659D0101C8207900C92CF0D2840B20F739
:1045C000CE68850D68850E297F850CA62FA53086BF
:1045D0005F8560C532D004E431F039A000B15FC816
:1045E000C545D006A546D15FF016C8B15F18655F16
:1045F000AAC8B15F656090D7A2122CA20E4C37C436
:10460000A213A50CD0F72094D1A50BA004D15FD0A4
:10461000E74CEAD22094D12008C4A0008472A205FD
:10462000A545915F1001CAC8A546915F1002CACA8C
:104630008671A50BC8C8C8915FA20BA900240C50B5
:104640000868186901AA686900C8915FC88A915F03
:10465000204CD386718572A422C60BD0DC6559B07C
:104660005D8559A88A65589003C8F0522008C48512
:10467000318432A900E672A471F005889158D0FB0C
:10468000C659C672D0F5E65938A531E55FA002914A
:104690005FA532C8E560915FA50CD062C8B15F85A7
:1046A0000BA90085718572C868AA8564688565D183
:1046B0005F900ED006C88AD15F90074C45D24C352A
:1046C000C4C8A572057118F00A204CD38A6564AA83
:1046D00098A42265658671C60BD0CA8572A205A50D
:1046E000451001CAA5461002CACA8628A90020554D
:1046F000D38A655885479865598548A8A547608439
:1047000022B15F852888B15F8529A910855DA20047
:10471000A0008A0AAA982AA8B0A406712672900B53
:10472000188A6528AA986529A8B093C65DD0E36069
:10473000A50DF00320A6D62026D538A533E531A84F
:10474000A534E532A200860D85628463A2904C44B4
:10475000DC3820F0FFA900F0EBA63AE8D0A0A215C3
:104760002CA21B4C37C420E1D320A6D320FACEA91B
:10477000808510208BD0208DCD20F7CEA9B220FFD0
:10478000CE48A54848A54748A57B48A57A4820F8C3
:10479000C84C4FD4A9A520FFCE098085102092D007
:1047A000854E844F4C8DCD20E1D3A54F48A54E4872
:1047B00020F1CE208DCD68854E68854FA002B14E88
:1047C0008547AAC8B14EF0998548C8B147488810B6
:1047D000FAA44820D4DBA57B48A57A48B14E857A57
:1047E000C8B14E857BA54848A54748208ACD688535
:1047F0004E68854F207900F0034C08CF68857A68B1
:10480000857BA00068914E68C8914E68C8914E683B
:10481000C8914E68C8914E60208DCDA00020DFDD8C
:104820006868A9FFA000F012A664A46586508451B0
:1048300020F4D486628463856160A222860786089C
:10484000856F847085628463A0FFC8B16FF00CC56A
:1048500007F004C508D0F3C922F0011884619865F7
:104860006F8571A6709001E88672A570F004C90288
:10487000D00B982075D4A66FA4702088D6A616E019
:1048800022D005A2194C37C4A5619500A5629501F7
:10489000A5639502A00086648465847088840D8673
:1048A00017E8E8E8861660460F4849FF386533A4E4
:1048B00034B00188C4329011D004C531900B8533D7
:1048C000843485358436AA6860A210A50F30B620DE
:1048D00026D5A980850F68D0D0A637A53886338520
:1048E00034A000844F844EA531A632855F8660A92E
:1048F00019A20085228623C516F00520C7D5F0F73A
:10490000A9078553A52DA62E85228623E430D00441
:10491000C52FF00520BDD5F0F385588659A903852C
:1049200053A558A659E432D007C531D0034C06D65A
:1049300085228623A000B122AAC8B12208C8B122CC
:1049400065588558C8B122655985592810D38A30D1
:10495000D0C8B122A0000A6905652285229002E62E
:1049600023A623E459D004C558F0BA20C7D5F0F3E4
:10497000B1223035C8B1221030C8B122F02BC8B1F5
:1049800022AAC8B122C5349006D01EE433B01AC59D
:10499000609016D004E45F9010865F8560A522A623
:1049A00023854E864FA5538555A55318652285222C
:1049B0009002E623A623A00060A54F054EF0F5A5C2
:1049C0005529044AA88555B14E655F855AA5606989
:1049D00000855BA533A6348558865920BFC3A455EE
:1049E000C8A558914EAAE659A559C8914E4C2AD54A
:1049F000A56548A564482083CE208FCD68856F6863
:104A00008570A000B16F1871649005A2174C37C46F
:104A10002075D4207AD6A550A45120AAD6208CD6B1
:104A2000A56FA47020AAD620CAD44CB8CDA000B1DE
:104A30006F48C8B16FAAC8B16FA86886228423A83E
:104A4000F00A4888B122913598D0F8681865358504
:104A5000359002E63660208FCDA564A4658522845A
:104A60002320DBD608A000B12248C8B122AAC8B1D1
:104A700022A86828D013C434D00FE433D00B4818D0
:104A8000653385339002E634688622842360C41837
:104A9000D00CC517D0088516E9038517A000602043
:104AA000A1D78A48A901207DD468A00091626868D6
:104AB0004CCAD42061D7D150989004B150AA9848DC
:104AC0008A48207DD4A550A45120AAD668A8681889
:104AD000652285229002E62398208CD64CCAD420E9
:104AE00061D718F15049FF4C06D7A9FF8565207999
:104AF00000C929F00620FDCE209ED72061D7F04BBB
:104B0000CA8A4818A200F150B0B649FFC56590B1F5
:104B1000A565B0AD20F7CE68A8688555686868AA15
:104B2000688550688551A555489848A0008A60203E
:104B300082D74CA2D320A3D6A200860DA8602082E3
:104B4000D7F008A000B122A84CA2D34C48D22073C1
:104B500000208ACD20B8D1A664D0F0A6654C79009B
:104B60002082D7D0034CF7D8A67AA47B86718472B2
:104B7000A622867A1865228524A623867B9001E8E2
:104B80008625A000B1244898912420790020F3DCE8
:104B900068A0009124A671A472867A847B60208A22
:104BA000CD20F7D720FDCE4C9ED7A566309DA561C0
:104BB000C991B097209BDCA564A465841485156019
:104BC000A51548A5144820F7D7A000B114A86885FA
:104BD000146885154CA2D320EBD78AA000911460ED
:104BE00020EBD78649A200207900F00320F1D78678
:104BF0004AA000B114454A2549F0F860A911A0DF88
:104C00004C67D8208CDAA56649FF8566456E856FAE
:104C1000A5614C6AD82099D9903C208CDAD0034CFD
:104C2000FCDBA6708656A269A569A8F0CE38E561BE
:104C3000F02490128461A46E846649FF6900A0008C
:104C40008456A261D004A0008470C9F930C7A8A519
:104C500070560120B0D9246F1057A061E069F002AE
:104C6000A0693849FF65568570B90400F50485656B
:104C7000B90300F5038564B90200F5028563B90143
:104C800000F5018562B0032047D9A0009818A662FC
:104C9000D04AA6638662A6648663A6658664A6700B
:104CA000866584706908C920D0E4A900856185669D
:104CB0006065568570A565656D8565A564656C85BF
:104CC00064A563656B8563A562656A85624C36D9A8
:104CD00069010670266526642663266210F238E5AF
:104CE00061B0C749FF69018561900EE661F04266D7
:104CF00062666366646665667060A56649FF856680
:104D0000A56249FF8562A56349FF8563A56449FFE4
:104D10008564A56549FF8565A57049FF8570E670C6
:104D2000D00EE665D00AE664D006E663D002E662FD
:104D300060A20F4C37C4A225B4048470B403940459
:104D4000B4029403B4019402A4689401690830E8A1
:104D5000F0E6E908A8A570B01416019002F60176F5
:104D60000176017602760376046AC8D0EC18608179
:104D700000000000037F5E56CB7980139B0B64809C
:104D8000763893168238AA3B20803504F334813577
:104D900004F334808000000080317217F8202BDC8F
:104DA000F00210034C48D2A561E97F48A9808561D3
:104DB000A9D6A0D92067D8A9DBA0D9200FDBA9BC30
:104DC000A0D92050D8A9C1A0D92040E0A9E0A0D9FD
:104DD0002067D868207EDDA9E5A0D9208CDAD00331
:104DE0004C8BDA20B7DAA900852685278528852906
:104DF000A5702059DAA5652059DAA5642059DAA5ED
:104E0000632059DAA562205EDA4C8FDBD0034C8335
:104E1000D94A0980A8901918A529656D8529A52862
:104E2000656C8528A527656B8527A526656A852677
:104E300066266627662866296670984AD0D66085F9
:104E4000228423A004B122856D88B122856C88B1AB
:104E500022856B88B122856E4566856FA56E0980B7
:104E6000856A88B1228569A56160A569F01F18650A
:104E7000619004301D182C101469808561D0034C9A
:104E8000FBD8A56F856660A56649FF300568684C4C
:104E9000F7D84C7ED9200CDCAAF010186902B0F2C9
:104EA000A200866F2077D8E661F0E76084200000DA
:104EB00000200CDCA9F9A0DAA200866F20A2DB4C4E
:104EC00012DB208CDAF076201BDCA90038E5618546
:104ED0006120B7DAE661F0BAA2FCA901A46AC46253
:104EE000D010A46BC463D00AA46CC464D004A46DB5
:104EF000C465082A9009E89529F0321034A90128E0
:104F0000B00E066D266C266B266AB0E630CE10E237
:104F1000A8A56DE565856DA56CE564856CA56BE55B
:104F200063856BA56AE562856A984C4FDBA940D022
:104F3000CE0A0A0A0A0A0A8570284C8FDBA2144C92
:104F400037C4A5268562A5278563A5288564A5297C
:104F500085654CD7D885228423A004B12285658835
:104F6000B122856488B122856388B1228566098073
:104F7000856288B1228561847060A25C2CA257A0F2
:104F800000F004A649A44A201BDC86228423A00446
:104F9000A565912288A564912288A563912288A5A0
:104FA00066097F2562912288A5619122847060A59F
:104FB0006E8566A205B5689560CAD0F986706020D6
:104FC0001BDCA206B5609568CAD0F9867060A56141
:104FD000F0FB067090F7206FD9D0F24C38D9A5615C
:104FE000F009A5662AA9FFB002A90160202BDC8583
:104FF00062A9008563A288A56249FF2AA900856588
:1050000085648661857085664CD2D8466660852445
:105010008425A000B124C8AAF0C4B124456630C2DA
:10502000E461D021B1240980C562D019C8B124C57A
:1050300063D012C8B124C564D00BC8A97FC570B1B4
:1050400024E565F028A566900249FF4C31DCA56196
:10505000F04A38E9A024661009AAA9FF8568204D06
:10506000D98AA261C9F910062099D9846860A8A5D7
:1050700066298046620562856220B0D9846860A591
:1050800061C9A0B020209BDC8470A566846649803D
:105090002AA9A08561A56585074CD2D8856285635C
:1050A00085648565A860A000A20A945DCA10FB9083
:1050B0000FC92DD0048667F004C92BD005207300DA
:1050C000905BC92EF02EC945D0302073009017C9CF
:1050D000ABF00EC92DF00AC9AAF008C92BF004D014
:1050E000076660207300905C2460100EA90038E50C
:1050F0005E4C49DD665F245F50C3A55E38E55D8583
:105100005EF012100920FEDAE65ED0F9F00720E228
:10511000DAC65ED0F9A5673001604CB4DF48245F81
:105120001002E65D20E2DA6838E930207EDD4C0AC4
:10513000DD48200CDC68203CDCA56E4566856FA64A
:10514000614C6AD8A55EC90A9009A964246030112F
:105150004C7ED90A0A18655E0A18A000717A38E9EF
:1051600030855E4C30DD9B3EBC1FFD9E6E6B27FD87
:105170009E6E6B2800A971A0C320DADDA53AA6397E
:1051800085628663A290382049DC20DFDD4C1ECB8F
:10519000A001A92024661002A92D99FF008566842C
:1051A00071C8A930A661D0034C04DFA900E080F0EB
:1051B00002B009A9BDA0DD2028DAA9F7855DA9B84C
:1051C000A0DD205BDCF01E1012A9B3A0DD205BDCAB
:1051D000F002100E20E2DAC65DD0EE20FEDAE65DC7
:1051E000D0DC2049D8209BDCA201A55D18690A30DB
:1051F00009C90BB00669FFAAA90238E902855E86D3
:105200005D8AF0021013A471A92EC899FF008AF0DC
:1052100006A930C899FF008471A000A280A5651876
:105220007919DF8565A5647918DF8564A563791729
:10523000DF8563A5627916DF8562E8B00410DE3091
:105240000230DA8A900449FF690A692FC8C8C8C8C1
:105250008447A471C8AA297F99FF00C65DD006A91A
:105260002EC899FF008471A4478A49FF2980AAC0EB
:1052700024F004C03CD0A6A471B9FF0088C930F066
:10528000F8C92EF001C8A92BA65EF02E1008A900BF
:1052900038E55EAAA92D990101A9459900018AA2C4
:1052A0002F38E8E90AB0FB693A9903018A990201AB
:1052B000A900990401F00899FF00A900990001A92B
:1052C00000A001608000000000FA0A1F000098960C
:1052D00080FFF0BDC0000186A0FFFFD8F0000003F2
:1052E000E8FFFFFF9C0000000AFFFFFFFFFFDF0A4F
:1052F0008000034BC0FFFF736000000E10FFFFFD36
:10530000A80000003CBFAAAAAAAAAAAAAAAAAAAA56
:10531000AAAAAAAAAAAAAAAAAAAAAAAAAAAAAAAAED
:10532000AAAAAAAA200CDCA911A0DF20A2DBF07097
:10533000A569D0034CF9D8A24EA00020D4DBA56EFD
:10534000100F20CCDCA94EA000205BDCD00398A479
:105350000720FEDB984820EAD9A94EA0002028DAD1
:1053600020EDDF684A900AA561F006A56649FF8531
:1053700066608138AA3B29077134583E5674167E00
:10538000B31B772FEEE3857A1D841C2A7C63595862
:105390000A7E75FDE7C6803172181081000000009A
:1053A000A9BFA0DF2028DAA570695090032023DC74
:1053B000855620A2A0D0EBE5B9334487C068B6B7C4
:1053C0002699C700160355005300420020005300E1
:1053D00065007200690061006C00180354006500EC
:1053E00065006E00730079006400750069006E004E
:1053F0006F000403090409024B00020100C03208D7
:105400000B00020202010009040000010202010077
:1054100005240010010524010101042402060524CD
:105420000600010705820310001009040100020AAA
:105430000000000705030240000007058402400049
:105440000009024B00020100C032080B00020202F8
:1054500001000904000001020201000524001001FE
:1054600005240101010424020605240600010705A4
:10547000820310000509040100020A00000007056C
:105480000302000200070584020002000A0600026F
:08549000EF02014001000100E0
:105498000000000000000000000000000000000004
:1054A80000000000000000000000000000000000F4
:1054B8000E480F4B02881B6833F8121001320D4B4F
:1054C8001B6819800C4B19884B00013B13409BB299
:1054D800038013B9094A137004E0994205D10122E7
:1054E800064B1A704022064B1A607047E47B002076
:1054F800FC650020003B0020E27B0020A03B002050
:1055080008E200E0194B1A78194B70B5194E1A4D7C
:105518001A4C8AB131881B682868984731882A68EC
:10552800490822F01F0302EB8102BFF34F8F23606B
:1055380020339A42FBD814E031882A6848081B684F
:1055480002EB8000984733882A685B089900531853
:1055580023F01F020B44BFF34F8F22602032934287
:10556800FBD8BFF34F8FBFF36F8F70BDA03B0020F8
:10557800C0650020E27B00200042002070EF00E0C0
:10558800024B1B780BB104F08DBC70470A870020D2
:1055980010B5054C237833B9044B13B10448AFF365
:1055A80000800123237010BDD0600020000000009F
:1055B800A4100100084B10B51BB108490848AFF307
:1055C80000800848036803B910BD074B002BFBD0C7
:1055D800BDE81040184700BF00000000D46000205C
:1055E800A4100100C03E0020000000000122014B71
:1055F8001A7070470A8700200022026070477047BF
:105608004160704710B50446FFF7F6FF00230449D0
:105618002046638223756375FFF7F2FF204610BDAD
:1056280080841E0010B50446FFF7E9FF204610BD30
:1056380081607047418270470175704701440A7361
:1056480070470000FF2149F21113014AD1547047F5
:10565800308700200F4A49F21113017BD35C11B93E
:1056680043F03C0303E003F0DF0343F01C03417BFA
:1056780009B103F0FB03817B09B103F0F703C17B98
:1056880009B103F0EF0349F21111535449F21F1104
:105698005354704730870020094B49F2221149F2D0
:1056A800201259569A5C0029017CA8BF42F080025A
:1056B80009B102F07F0249F220115A54704700BF25
:1056C80030870020194A49F2201370B5448AD55C06
:1056D800E1B225B9002C14BF0B46FF231FE0260AB0
:1056E800B54204D1002914BF0B46FF2300E0FF2375
:1056F800F72D07D1007D90B174B1F72E0CD101F0D0
:10570800FD030CE0DF2D0AD1407D40B134B1DF2E1E
:1057180004D101F0FE0302E0FD2300E0FE2349F27C
:105728002111535449F22F11535470BD3087002072
:10573800F8B5404C49F2271649F2261E49F22D12B7
:1057480014F806C049F22E1314F80E1049F219176E
:10575800A55C49F2181251EA0C21E35CA25CE75DF2
:1057680005D145F0400549F22D1165540BE001F1D2
:10577800FF3C023989B204F80EC04FEA112E04F832
:1057880006E00029EDD049F229162A49A65D46B35C
:1057980052EA072215D149F2281245F02005A15CEA
:1057A80049F21812A15449F2191249F22911A654C2
:1057B8000022625449F22A11625449F22D12A5546A
:1057C8000FE002F1FF3E023A49F2181792B201F8CF
:1057D80007E049F219174FEA122E01F807E0002AEC
:1057E800D9D003F07F031D4223D0806803F070FCFA
:1057F800F8B1690616D549F22B120E4BA25C520677
:105808000BD549F224110C4A585C49F2261112882A
:10581800585449F2271112125A5405F0BF0549F29B
:105828002D13E554AB0642BF25F0200349F22D1293
:10583800A354F8BD308700205418012010B5044641
:10584800FFF776FF2046FFF705FF2046FFF724FF06
:105858002046FFF737FF23680133236010BD00009F
:1058680010B50446FFF7C8FE0023044920462372FA
:105878000123A373FFF7C4FE204610BD20E81000E3
:1058880010B50446FFF7BBFE204610BD184B00229A
:105898001A804FF6FF725A804BF2E4029A8044F65F
:1058A8009F72DA804BF2FF121A8144F206725A8113
:1058B80040F6BE229A814DF6A362DA814CF6A02208
:1058C8001A824EF68E525A824EF292429A8249F6C5
:1058D800BF72DA824EF2FF421A8348F632725A8356
:1058E80048F29F429A834EF2F062DA83704700BF13
:1058F800C27B0020EF2910B511D8094A49F20F03DD
:105908000846D35C074A03F0070332F8134003F054
:1059180099FC00F5207320F8024B9842FBD110BD8A
:1059280030870020C27B00202DE9F04F1F468BB046
:105938006D4849F20303102F0191C35C04D1C3F3EE
:105948004503162BC8BF521007FB02FB019B5B44A3
:10595800EF2B00F3C58049F2020349F20501002448
:10596800C35C415C03F07F069B00890103F400736C
:10597800724301F4E051C6F128059BB2AD00194409
:10598800A3F5D8439BB211441A44411883180291D5
:10599800564A039349F20F03C35C03F007011B093E
:1059A80032F8133032F81110ADF8203025EAE573DB
:1059B800ADF822105B00059333010693BC4280F2D8
:1059C8008F80019B03EB0B00204403F03BFCBDF8E8
:1059D80022200023AB4203DA20F813200133F9E731
:1059E800059B0021DFF80CC1C318414ADFF8FC8091
:1059F80000931CF8093B03F00F0332F81320BDF89D
:105A0800203022440493009B07920433B14258DAB1
:105A1800029A0798525C02FB070240F6FE7092B2A7
:105A280002F55F4E0EF1FF0E1FFA8EFE86452E48D8
:105A38009CBF02F5C04292B210F80290039A12F885
:105A480001E00EF007020EF0080E38F812A00EF072
:105A5800FF02ADF824A0BEF1000F13D1A3F1020E8E
:105A680009FA02F001320EF1020E000656BFBDF827
:105A780010002EF804AC2EF8040C082AF0D10131DD
:105A88001033C3E79CF800209A464FF0000E120925
:105A980038F81220ADF8262009FA0EF20AA80EF1FD
:105AA800020E0AF1040AC2F38112BEF1080F00EBDC
:105AB800420232F8082C2AF8082C2AF8062CEBD1D6
:105AC800DDE7069B009A1A4400231046BDF8222001
:105AD800AB4203DA20F813200133F9E701346DE70C
:105AE8000BB0BDE8F08F00BF30870020C27B0020DC
:105AF800880F002035170120002383737047807BAF
:105B080070470000F8B547230D4601680446B1FB0D
:105B1800F3F203FB1213F3B9344849F2030649F2CE
:105B28000403825DC15CD31143EA4101D3074BD41E
:105B3800B1F59C7F3ADC0823013149F2030649F2AA
:105B48000407825D02F07F0242EAC11282554A10C0
:105B5800C255A2891AB923681D442560F8BD678912
:105B6800B9421FD33A4491421CDAC81B591E90FB14
:105B7800F3F203FB1202D2B28A42ECD1227A3946FE
:105B88002046FFF7D1FE237A184A0133DBB223728D
:105B9800925DC2F345029342DDDB002323720123A9
:105BA800A373D8E72046FFF7A5FED4E7C2F3450262
:105BB8000823D200A281A2890221C2F1F00292FB3D
:105BC800F1F200216281B8E7B1F59C7F01DC102376
:105BD800B2E7C2F345021201A281835DC3F3450314
:105BE800162B01DDDB00A3811023E4E730870020BA
:105BF8000020704770477047704701207047704712
:105C0800006910B10368DB6818477047006910B174
:105C180003681B6918477047006910B103685B691E
:105C280018474FF0FF307047006910B103689B694F
:105C38001847704707B5006910B94FF0FF3009E001
:105C4800036801220DF107019B6898470028F4D0EA
:105C58009DF8070003B05DF804FB07B500698DF8EF
:105C6800071028B1036801220DF10701DB68984786
:105C780003B05DF804FB0000314B012201461A70A5
:105C8800304B93F86E00402820D13D291BD007DC0B
:105C9800242916D0262918D0222908BF232115E047
:105CA800E0290CD003DCA72908BF5E210EE0E72914
:105CB80003D0E92908BF402108E07B2106E07D21C7
:105CC80004E05D2102E07E2100E07C211E4B1B7870
:105CD800002B32D0D72920D00ADC0A2922D020294B
:105CE80025D009292BD1194A137823F0400322E043
:105CF800D92903D00CDBDA2905D07047134A137869
:105D080023F0080317E0114A137823F0040312E084
:105D18000E4A137823F002030DE00C4A137823F09F
:105D2800010308E0094A137823F0100303E0074A47
:105D3800137823F020031370704704F077B9704785
:105D4800197C0020A04D0020A13B0020F7860020F0
:105D5800314B012201461A70304B93F86E004028EF
:105D680020D13D291BD007DC242916D0262918D09C
:105D7800222908BF232115E0E0290CD003DCA7293C
:105D880008BF5E210EE0E72903D0E92908BF4021BA
:105D980008E07B2106E07D2104E05D2102E07E2110
:105DA80000E07C211E4B1B78002B32D0D72920D055
:105DB8000ADC0A2922D0202925D009292BD1194A01
:105DC800137843F0400322E0D92903D00CDBDA2909
:105DD80005D07047134A137843F0080317E0114AB7
:105DE800137843F0040312E00E4A137843F00203D9
:105DF8000DE00C4A137843F0010308E0094A1378D0
:105E080043F0100303E0074A137843F020031370AC
:105E1800704704F0FDB87047197C0020A04D0020A1
:105E2800A13B0020F786002013B50346006D0C4601
:105E380028B10DF1060201A90AF063F908E0586DCE
:105E480008B9002021E00DF1060201A907F0EAFFD8
:105E58000028F6D0BDF80430BDF806200BB9002A9A
:105E6800EFD002F01F0149002170C2F34511D21290
:105E78006170A27003F01F022271C3F343125B1218
:105E8800013A03F5EA636271A37102B010BD13B55C
:105E98000346006D0C4628B10DF1060201A90AF06F
:105EA80040F908E0586D08B9002021E00DF106021C
:105EB80001A907F0C7FF0028F6D0BDF80430BDF8E7
:105EC80006200BB9002AEFD002F01F01490021700B
:105ED800C2F34511D2126170A27003F01F02227141
:105EE800C3F343125B12013A03F5EA636271A371CB
:105EF80002B010BD38B5856D0446BDB94FF4807049
:105F08000FF0E0FB0146A06570B10570206D20B16F
:105F18004FF480720BF0DEFA08E0606D30B14FF498
:105F2800807209F0D9FA01E0014BA365A06D38BD74
:105F3800FD860020D0B5046D6CB1012B08BF002A86
:105F480014D21146204609F0F4FE78B120460AF032
:105F5800F5FA58B1D0BD446D44B1204608F0ABF80D
:105F680020B12046BDE8D04008F070BE0020D0BD6A
:105F780010B5044600684368013B43603BB90368B9
:105F8800DB6A9847206810B103685B68984700236C
:105F9800236010BD054B10B503600446036913B1B7
:105FA8001030FFF7E5FF204610BD00BF6407002052
:105FB80010B50446FFF7EEFF142120460FF084F8D1
:105FC800204610BD10B5084C04F13C00FFF7E2FF75
:105FD80004F12800FFF7DEFF04F11400FFF7DAFFF1
:105FE8002046FFF7D7FF10BD983A002010B103688C
:105FF8009B681847704738B50B6804460D4613B1BF
:106008005A6801325A6023691BB104F11000FFF786
:10601800AFFF2B682046236138BD10B103681B6BA6
:106028001847704710B103689B6A18470020002181
:106038007047036D13B1586900217047436D13B160
:1060480093E8030070471846F6E7036D13B1D86963
:1060580000217047436D13B1186959697047184694
:10606800F6E770B5044608460D460FF098FC23681D
:106078000246294620465B68BDE87040184738B597
:106088000546FFF7EEFF044628460EF017FF2044AA
:1060980038BD38B505460EF070FF044628460EF0A8
:1060A8000DFF204438BD826B30B562B1137803F020
:1060B800080303F0FF00FBB1D3695069181A1BD518
:1060C8006FF0004018E0C06BB0B190F831301B079A
:1060D80007D5D0E90445D0E90023A01A65EB0301F0
:1060E80001E00020002100236FF000428B4208BF2E
:1060F800824201D2104630BD30BD08B51030FFF7DE
:10610800D2FF08BD08B51830FFF7CDFF08BD836B77
:106118001BB11B7813F0700F05E0C06B30B190F81D
:10612800313013F0500F14BF01200020704708B51C
:106138001830FFF7ECFF08BD10B504461830FFF71C
:10614800E6FF60B1206D10B1002109F0F2FD606D2D
:1061580028B100220023BDE8104007F0ACBF10BDF5
:10616800836B23B9C06B003018BF01207047012032
:10617800704708B51830FFF7F3FF08BD10B504469F
:10618800806D18B10FF0A6FA0023A36518342046D5
:10619800FFF7E6FF20B12046BDE810400BF083BBB7
:1061A80010BD0000064B10B503600446FFF7E6FF7C
:1061B800044B04F11800A3600BF075FB204610BDDA
:1061C800B40700200406002010B50446FFF7EAFFD4
:1061D8005C2120460EF078FF204610BD0346806BF8
:1061E80008B109F076BDD86B08B107F04FBF4FF082
:1061F800FF30704708B51030FFF7F0FF08BD08B54D
:106208001830FFF7EBFF08BD0346806B08B109F0B3
:10621800A5BCD86B08B107F077BE4FF0FF307047C8
:1062280007B501220DF107011030FFF7EDFF012836
:106238000CBF9DF807004FF0FF3003B05DF804FB7A
:1062480008B51830FFF7E0FF08BDD0B4846B44B13F
:10625800012B08BF002A09D220461146D0BC09F0FC
:1062680068BDC06B10B1D0BC07F025BF0020D0BC02
:10627800704738B50146049814461D4610B901F117
:1062880018001DE001280AD10B6D01F118000BB1AF
:106298005A6912E04B6D7BB1D3E900230EE0022866
:1062A80011D10B6D01F118000BB1DA6905E04B6DE6
:1062B80013B1D3E9042301E00022002312196B4132
:1062C800FFF7C3FF38BD002038BD0346806B08B117
:1062D80009F05ABED86B08B108F0C8BA704708B5BB
:1062E8001030FFF7F2FF08BD08B51830FFF7EDFFD3
:1062F80008BDF0B5D0F838E09DF814409DF8185066
:106308009DF81C609DF82070BEF1000F08D008971A
:106318007046079606950594BDE8F0400AF0B7B8B0
:10632800C06B38B10897079606950594BDE8F0400C
:1063380008F002BCF0BD1FB58A79A2F150031B0614
:1063480011D40C7802F26C724B79183003944C78A3
:1063580001330294DBB28C7801940979009104210D
:10636800FFF7C7FF00E0002004B010BD1FB58A7911
:10637800A2F150031B0611D40C7802F26C724B790F
:10638800183003944C7801330294DBB28C78019472
:10639800097900910221FFF7ACFF00E0002004B06A
:1063A80010BD0346806B08B10AF0FCB8D86B08B181
:1063B80008F0ACBC704708B51830FFF7F2FF08BD0D
:1063C80008B51030FFF7EDFF08BD07B502AB012295
:1063D800103003F8011D1946FFF7E3FF03B05DF81D
:1063E80004FB000000234FF47A7203710373054B1A
:1063F800826003600B69036113B15A6801325A6005
:10640800704700BF6407002010B50446006940B11A
:106418000368DB6A984704F11000BDE81040FFF7F5
:10642800A7BD10BD38B500250E4B04461031456098
:10643800183040F8183C11F80C3C00F80C3C0A4B9A
:1064480040F8103C51F8083C40F8083C11F8043C6E
:1064580000F8043C0BF0F6F9044BA5652046A36050
:1064680038BD00BFB40700201008002090070020A6
:106478002DE9F04395B000251C4B4FF47A760DF1C9
:1064880050082A461831044604A848F8503D8DF8AB
:10649800045002968DF80C50129513950BF056FA8D
:1064A80004A8DFF85090FFF75BFE80B15C200EF087
:1064B80009FE07464146FFF7B5FF7B6825710133A2
:1064C800A6602573C4F8009027617B6005E0207101
:1064D800A6602073C4F800902061054B04A80093BF
:1064E8000BF0E1F9204615B0BDE8F08390070020D5
:1064F8000406002064070020012B70B5044694B000
:1065080005D0022B40F2022318BF002301E044F219
:106518000223043168460BF0A9FA04A8FFF720FE0D
:10652800114E90B15C200EF0CDFD69460546FFF78F
:1065380079FF00234FF47A722660237123736B6806
:10654800A260013325616B6006E04FF47A73207115
:106558002073A36026602061044B04A800930BF00D
:10656800A2F9204614B070BD64070020040600207C
:1065780070B5324B8AB00024314A00934FF47A73D5
:10658800304905A8029323468DF804408DF80C4045
:106598000494FFF7B1FF2C4E09A92B48FFF72BFDF8
:1065A80005A8FFF7F7FC316929B10B68002205A897
:1065B800DB6B984703E0244905A8FFF713FF09A9F7
:1065C8006846FFF718FD05A8FFF7E4FC0498FFF7F5
:1065D80024FD48B3049820B103685B6B98470546CF
:1065E80000E01A4D29461A48FFF749FD049868B19A
:1065F80003689B6B984748B1164928460FF0BDF9C8
:1066080068B1154928460FF0B8F940B1134B182066
:106618001722294600FB043001340FF0DDF96846E3
:10662800FFF7F2FE3F2CBEDD0748FFF7EDFE684698
:10663800FFF7B0FC20460AB070BD00BF6407002019
:10664800B7860020EC600020EC3A00207E3900205C
:10665800883A00202F3600202E3600208B7D00201F
:106668000146024808B5FFF70AFD08BD883A002030
:106678000146024808B5FFF70CFD08BD883A00201E
:10668800044B28B91A780AB1187001E001221A706F
:1066980018787047107C0020014B1888704700BF9D
:1066A800C07B00202DE9F04F232085B00DF0D8F9EC
:1066B80000284FF0240014BF002404240DF0D0F962
:1066C80010B944F00804A4B226200DF0C9F910B995
:1066D80044F00104A4B225200DF0C2F910B944F029
:1066E8000204A4B222200DF0BBF910B944F0100442
:1066F800A4B2A04B1B780BB92402A4B29E4B1B7802
:106708005E0744BF44F00404A4B21D0744BF44F02C
:106718000804A4B298074FF0290044BF44F00204CB
:10672800A4B2D90744BF44F00104A4B2DA0644BFB6
:1067380044F01004A4B29F0644BF44F02004A4B25D
:106748005E0644BF44F04004A4B20DF089F910B9C4
:1067580044F02004A4B228200DF082F910B944F0C6
:106768004004A4B2854A4FF0FF33854D00271068D6
:106778000DF1040B2B6001AB5168DFF808A203C3CD
:10678800906818601BF81760012130460DF07AF9FF
:10679800002130460DF044F913200DF061F9B0FAEC
:1067A80080F812200DF05CF900284FEA58184FF0D5
:1067B800110014BF0023022348EA03080DF050F922
:1067C80000284FF0050014BF0023042348EA0308FB
:1067D8000DF046F900284FF01D0014BF00230823D0
:1067E80048EA03080DF03CF900284FF01E0014BFDA
:1067F8000023102348EA03080DF032F900284FF06F
:10680800200014BF0023202348EA03090DF028F9CB
:1068180000284FF00101304614BF4FF000084FF038
:1068280040080DF0FDF8304649EA080805210DF04A
:1068380029F9544E0AF807800137062FA2D1737937
:1068480003F0080202F0FF011AB123F00803012146
:106858007371727902F0100000F0FF0320B1494B08
:1068680022F010025A7101230027D5F800E03846BB
:10687800325C002A18BF864600F1010018BF0127C4
:106888000628F5D10FB1C5F800E0550644BF44F01D
:106898000204A4B2900644BF44F00104A4B2D7078E
:1068A800394F48BF44F00804BE4648BFA4B2550754
:1068B800364D44BF44F00404A4B2900738682A68EF
:1068C80048BF44F01004A0EB020248BFA4B2642AF7
:1068D80007D92F4A286015780DB9012500E0002551
:1068E80015702C4D2C4F2D4A13B101232B703CE011
:1068F8002B70002938D097F800C02949BCF1000F47
:106908001BD1D1F800E0BEF1000F03D1254B186070
:10691800012325E00EF1010EBEF1010FC1F800E0E0
:106928001FD90B601F490968401AB0F5FA7F18D2C1
:10693800117801B90123137013E00868012810D1F8
:10694800DEF80000DFF85CE0DEF800E0CEEB0000E7
:10695800B0F57A7F05D91078B0FA80F04009107048
:106968000B6001233B7000E039701378E3B1084BEA
:1069780019781EE0107C0020F78600208C0D00207E
:10698800E83A0020B0860020B47B0020DC7A0020A2
:10699800187C0020AD830020AC830020167C0020EA
:1069A800F8650020CC6500203B780BB9297801B147
:1069B80001210E200DF034F83B78002B3AD03279C3
:1069C80044F04003102A9BB202D144F06004A3B201
:1069D8002A78002A2DD0194B9C6BDA6C42F0010200
:1069E800DA649A6B22F002029A639A6B9207FCD4DB
:1069F80072B61248036D426D466D1049B242056D7C
:106A0800F8D1AB42F6D1D20B42EA434302338B654D
:106A18008A6D0A489342FBD144F002038363836B77
:106A2800064A9B07FBD5936B43F04003936330BF43
:106A3800FDE71C46204605B0BDE8F08F00400D403C
:106A480008B5FFF72FFE034A1388108020EA0303D6
:106A580098B208BDC07B00201B4B1C4A19781278DD
:106A68001B4B30B549B10AB11A4A0FE01A4A1278DD
:106A78000AB11A4A0AE01A4A08E00AB1194A05E0B6
:106A8800154A12780AB1184A00E0184A1A60184ADA
:106A98001268002A15DB1102164801F47F41825C56
:106AA80015481143002230F8125054008D4205D188
:106AB8000021124A1B681160185B30BD01322A2A76
:106AC800F1D1002030BD00BF167C0020AC8300202F
:106AD800387A0020A0110020AD8300204C1100203E
:106AE800F8100020A410002050100020FC0F0020F7
:106AF800E83A0020B0860020A80F0020F8650020A2
:106B080008B5022123200CF0BDFF022124200CF03F
:106B1800B9FF022126200CF0B5FF022125200CF038
:106B2800B1FF022122200CF0ADFF022129200CF038
:106B3800A9FF022128200CF0A5FF01210E200CF04E
:106B4800A1FF01210E200CF06BFF012110200CF099
:106B580099FF012106200CF095FF012118200CF067
:106B680091FF012119200CF08DFF01211C200CF050
:106B780089FF01211F200CF085FF012110200CF056
:106B88004FFF012106200CF04BFF012118200CF0CB
:106B980047FF012119200CF043FF01211C200CF0B4
:106BA8003FFF01211F200CF03BFF022113200CF0B6
:106BB80069FF022112200CF065FF022111200CF060
:106BC80061FF022105200CF05DFF02211D200CF061
:106BD80059FF02211E200CF055FF02212020BDE89C
:106BE80008400CF04FBF000030B50B4C01250B4B93
:106BF80085B0204600211D7002F036FE40F2FF727B
:106C08001F23204602958DE80C000022044B1146F4
:106C180002F0B2FE05B030BD1F8700209E3B002069
:106C28008C350020A54A03462DE9F04F14789FB013
:106C3800002C40F07B8141F21002A14D0240002A55
:106C480058D0A0490EA80EF0A2FE9F490EA80EF03B
:106C580085FE9E490EA80EF081FE0EA999480EF0F9
:106C680096FE9B48FFF7FCFC9648FFF7F9FC04A842
:106C78002346944A9749FFF73FFC089850B10368A8
:106C88009B6B984730B1944B1C60FFF771FC934B9A
:106C9800186029E0924B1B782BB30123914A8D4948
:106CA80009A8FFF729FC0DA98F48FFF7A4F9006987
:106CB800FFF7B3F9044609A8FFF76CF99CB18148BE
:106CC8000EF06DFE7F4902468748FEF799FF04469D
:106CD8007C480EF064FEA04202D08448FFF7C0FC56
:106CE8008148FFF791FB8124012304A82B70FFF74B
:106CF80051F970E000F02004A1B299B10123734961
:106D08007B4882242B700EF042FE6E4979480EF0C3
:106D18003EFE6D4977480EF021FE754975480EF024
:106D28001DFE58E000F04004A0B230B1012308462F
:106D38002B70FFF7A5FC0C464DE040F204441C40C4
:106D48004CB1654A1368002B40D00121013B044631
:106D5800297013603FE040F201121A406AB15E4A9E
:106D68001368082B03DD0121093B297003E06BB38D
:106D78000121013B297013602DE040F608011940FC
:106D880061B1564B54491C680B68601E98421FDD60
:106D98000CB301330B6001232B7019E040F202247D
:106DA8001C40C4B14D4B4C4A1C681368A4F109013E
:106DB800994202DD0CB1093304E0611E8B4209DA05
:106DC8004CB10133136001232B7003E01C4602E031
:106DD800144600E000242B78002B00F0A9803F4BDC
:106DE8001A689B46002A00F0A38090234FF0080CF5
:106DF8002022302140480026DFF808A137468DE8D8
:106E08000810C02302F06EFD334A13689146082B20
:106E1800D4BF0023043BCAF80030DBF800209742B7
:106E280023DB00264FF01F0E40F2FF73C8223021EB
:106E3800314802968DE80840304B02F09DFD08234A
:106E4800C82278210093C0232B48019602F04AFDFE
:106E58004FF6FF730296C822009378210196244BBF
:106E6800254802F089FD2E7062E0DAF800309F4272
:106E780056DB33449A4252DD214A4FF0180808FB8A
:106E88000728D9F8002093424FF0010306F10202C7
:106E980002934FEA021237D14FF6E0704FF478436D
:106EA80012B230218DE809004346134802F064FD10
:106EB800414606480EF06BFD31E000BFAE8300206E
:106EC8009E3B0020B78600200D3500205B7D00200A
:106ED800A0350020EC600020A07A0020D07A0020A5
:106EE800167C0020B0350020043B0020C03500206F
:106EF800737D00201B7C00201F870020D4350020D4
:106F08008B7D0020D87A00204FF6FF71082312B23B
:106F180009488DE80A004346302102F02DFD01366C
:106F2800082E07F101077FF778AF7AE7812000E0A4
:106F380020461FB0BDE8F08F1F870020014B18784E
:106F4800704700BFA13B0020034B18B101221A7003
:106F5800FFF74ABE18707047A13B002000487047F1
:106F6800B78600202DE9F041074686B01B4D002664
:106F7800DFF87C802869FFF750F80446D8F810003D
:106F880084F00104FFF749F8E4B2844208D10136DD
:106F98001435042EEED11248FFF762FB002019E0E9
:106FA80000233A460F4901A8FFF7A6FA05A9284683
:106FB800FFF721F80069FFF730F8044601A8FEF74B
:106FC800E9FF0CB1701C05E007492846FFF713F8E4
:106FD8000648E1E706B0BDE8F08100BF983A002016
:106FE800DD350020EC600020FC3A0020F23500205E
:106FF800EC3A002030B50B4B87B00D46013A14210E
:10700800044601A801FB0231FFF7ECF921462A46A4
:107018000598FEF7EBFF044601A8FEF7BBFF2046E4
:1070280007B030BD983A002010B50B4B0138142436
:1070380086B004FB003401A82146FFF7D3F901A864
:10704800FFF7E2F901A8FEF7A5FF04492046FEF77D
:10705800D2FF06B010BD00BF983A0020FC3A0020CD
:1070680030B5044687B0124DFFF7FAFA22460023DE
:10707800104901A8FFF740FA05A92846FEF7BBFF0B
:107088000069FEF7CAFF044601A8FEF783FF5CB15A
:107098000948FFF7E5FA2869FEF7C4FF0446FFF739
:1070A800E7FA2846FFF7B0F9204607B030BD00BF21
:1070B800043B0020EC60002016360020674B68492E
:1070C8001868F0B50C4693B0664D40F2EE27664E50
:1070D8000A784AB12A78D20706D51A68D6F800E0A5
:1070E800CEEB02020E2A0AD81A6894F800E0121AA7
:1070F800BEF1000F00F0B080B2F5FA6FE8D903F0E6
:107108002BFC5A4B5A4A9A645A4ADA64FE215A4866
:1071180006F054FD40B959495948FEF7B0FF4FF4FD
:107128007A700CF067FCF1E70024564D5649574831
:107138000EF02DFC281914345549FEF75CFF502C2D
:10714800F8D1544CFFF714FA5349002520604C48F5
:10715800FEF787FF21684A48FEF79BFFFFF7D0FC40
:107168004E4B29464E481D7002F08CFAFFF79AFAEA
:1071780010F008043DD04FF47841494802F074FB00
:1071880001244FF6E0724FF47843402144488DE8DB
:107198001C00444B302202F0EFFB374BD3F8841429
:1071A80079B12346404A04A88DF810508DF8115043
:1071B8008DF8125008F084FFB0B104A809F0F6FD6C
:1071C80012E0D3F8880478B18DF8411023468DF881
:1071D80042108DF843100146334A04A807F0D8F945
:1071E80010B104A807F065FA4FF47A700CF002FCAD
:1071F8002BE02E4E23462C4A04A81F49FFF77CF9A2
:1072080008A93046FEF7F7FE0069FEF706FF0546B7
:1072180004A8FEF7BFFEC5B130691C4FFEF702FF98
:107228000546024639463069FEF7E0FE854203D03E
:107238001F48FFF715FA01E07C5501241B48FFF7AA
:10724800E3F814B101221B4B1A7001221A4B1A7071
:10725800FFF7CAFC13B0F0BDBA424FE7B47B002079
:107268002C8700202B8700209C870120A04D002020
:10727800C1080000E9070000EC6000205236002039
:10728800883A0020983A00206F360020B786002000
:10729800FC3A0020D07A002073360020107C0020B1
:1072A8001F87002091360020B0350020043B0020C5
:1072B800A6360020AE830020A13B00200022014B0F
:1072C8001A707047F786002070B54B4800244B4D64
:1072D80020264B4B44608460C0F82403C0F8440364
:1072E800036005F0D7F821466C60AC6032462C612B
:1072F80005F128006C61EC6185F820406C620CF0A7
:1073080029FB404B284685F8854203F140022B6053
:107318006C332C65EA60AB616C6585F87840C5F81C
:10732800804285F8844285F8864285F8874205F0D0
:107338008DFD3548354D364B44608460C0F8900665
:10734800036080F87546C0F87846C0F87C4680F837
:10735800804680F8A44604F0D9FC324621466C6089
:1073680005F11C00AC602C612C75AC610CF0F2FAD4
:10737800284B284685F841402B603833EC63EB6096
:1073880085F8404085F8424085F843406C64AC6419
:10739800EC642C6506F046FA1F4D204B6C602846BD
:1073A8002B6005F59F63AC606B6305F5A7632D62E1
:1073B800AB6305F5AF631A4EEB6305F5B7636B6412
:1073C8004023A5F84A305023A5F84C3006F0E6F8DB
:1073D800144B314614482B60144D2A460EF027F9F9
:1073E8002A46134920460EF022F92A46314611480A
:1073F800BDE870400EF01BB9E0490020A04D002008
:1074080034080020DC06002020430020447B0020B4
:107418002806002060060020405000204406002076
:10742800050B0000E8050020EC3A0020DC390020BC
:10743800350B0000043B002083885A1C82801846C4
:107448007047000083885A1C10B592B2044C8280A1
:10745800E15C02338380A05C01EB002080B210BDA8
:107468003087002083885A1C8280014AD05C70478C
:10747800308700200020704782880649531C9BB241
:1074880083808A5C90B2120648BF40F47F4018445B
:1074980080B270473087002082880B4910B5541C91
:1074A800A4B284808B5C023282800A5D43EA0223A4
:1074B8005A1C03F47F40CB5C51FA82F2105C03EB58
:1074C800002080B210BD00BF3087002083885A1C7E
:1074D8008280034AD25C4378D018C0B2704700BF9C
:1074E8003087002083885A1C8280034AD25C8378C4
:1074F800D018C0B2704700BF308700208388074982
:107508005A1C92B210B58280CC5C023383804378D7
:107518008A5CE01800EB022080B210BD30870020A2
:10752800838807495A1C92B210B58280CC5C02331A
:10753800838083788A5CE01800EB022080B210BD5B
:107548003087002083885A1C8280064AD15C4378A1
:107558000B44DBB2591CD35CC9B2505C03EB00206E
:1075680080B27047308700208288531C8380064B86
:10757800995C4A1C595CD2B29A5C8378C81800EBB3
:10758800022080B2704700BF30870020012241F2FC
:107598000843C254704700002D4B0278F0B55D5C7B
:1075A8008379AC1885EA020703F00101214411F040
:1075B800FF0F0C460CBF43F0020323F00203837154
:1075C800837913F0080F24D002F00F0E05F00F0690
:1075D8007546354403F001063544092DC8BF8C1D96
:1075E80021064CBF63F07F0303F07F0317F0800F81
:1075F8008371837905D16240160602D543F04003B2
:1076080001E023F04003992C837183791BD96034FE
:1076180016E00D064CBF63F07F0303F07F0317F0FD
:10762800800F8371837905D14A40120602D543F051
:10763800400301E023F04003FF298371837902DDD1
:1076480043F0010301E023F0010383710470F0BDEE
:10765800308700200B4B5A5C03781A40837912F06C
:10766800800F02D063F07F0305E003F07F0312B9B7
:1076780043F0020303E08371837923F002038371EB
:10768800027070473087002010B5114C8379625C16
:1076980012F0800F4FEA4202D2B214BF43F0010346
:1076A80023F0010312F0800F8371837902D063F015
:1076B8007F0305E003F07F0312B943F0020303E000
:1076C8008371837923F002038371625410BD00BF74
:1076D800308700200278837912F0800F4FEA420247
:1076E800D2B214BF43F0010323F0010312F0800F5C
:1076F8008371837902D063F07F0305E003F07F0391
:1077080012B943F0020303E08371837923F0020383
:107718008371027070478379DB0758BF8180704797
:107728008379DB0748BF8180704783799B0748BF0F
:10773800818070470D4B5A5C01788379114022F0A3
:107748003F0211F0800F14BF63F07F0303F07F0343
:107758008371837903F03F031343837111B943F0B5
:10776800020301E023F00203837170473087002091
:1077780090F90630002BB8BF8180704783799B074A
:1077880058BF8180704790F90630002BA8BF8180D0
:10779800704783795B0658BF8180704783795B06A1
:1077A80048BF81807047837923F001038371704754
:1077B800837923F0080383717047837923F00403E6
:1077C80083717047837923F0400383717047000009
:1077D8000F4A0378525C9A1A8379FF2A94BF43F0C0
:1077E800010323F0010312F0800F8371837914BF22
:1077F80063F07F0303F07F0312F0FF0F8371837937
:107808000CBF43F0020323F002038371704700BFEB
:10781800308700200F4A4378525C9A1A8379FF2AEE
:1078280094BF43F0010323F0010312F0800F83712A
:10783800837914BF63F07F0303F07F0312F0FF0F17
:10784800837183790CBF43F0020323F00203837131
:10785800704700BF308700200F4A8378525C9A1A1D
:107868008379FF2A94BF43F0010323F0010312F048
:10787800800F8371837914BF63F07F0303F07F0364
:1078880012F0FF0F837183790CBF43F0020323F0DA
:1078980002038371704700BF308700200C4B10B57E
:1078A8005A5C013A12F0800FD4B21A46837914BF99
:1078B80063F07F0303F07F038371837914B943F086
:1078C800020301E023F002038371545410BD00BF8A
:1078D800308700204378013B13F0800FDAB28379B8
:1078E80014BF63F07F0303F07F038371837912B9B8
:1078F80043F0020301E023F00203837142707047F2
:107908008378013B13F0800FDAB2837914BF63F0F8
:107918007F0303F07F038371837912B943F0020375
:1079280001E023F002038371827070470B4B5A5CAD
:1079380003785A40837912F0800F02D063F07F03F6
:1079480005E003F07F0312B943F0020303E08371FB
:10795800837923F002038371027070473087002017
:107968000C4B10B55A5C013212F0800FD4B21A4693
:10797800837914BF63F07F0303F07F0383718379F6
:1079880014B943F0020301E023F002038371545455
:1079980010BD00BF308700204378013313F0800FFB
:1079A800DAB2837914BF63F07F0303F07F03837136
:1079B800837912B943F0020301E023F002038371D3
:1079C800427070478378013313F0800FDAB28379FD
:1079D80014BF63F07F0303F07F038371837912B9C7
:1079E80043F0020301E023F00203837182707047C1
:1079F800818070470A4B5A5C837912F0800F02D05D
:107A080063F07F0305E003F07F0312B943F002033C
:107A180003E08371837923F0020383710270704756
:107A2800308700200A4B5A5C837912F0800F02D00D
:107A380063F07F0305E003F07F0312B943F002030C
:107A480003E08371837923F00203837142707047E6
:107A5800308700200A4B5A5C837912F0800F02D0DD
:107A680063F07F0305E003F07F0312B943F00203DC
:107A780003E08371837923F0020383718270704776
:107A8800308700200E4B70B55A5C1C46837912F083
:107A9800010F14BF43F0010323F001038371531056
:107AA8008279DEB202F07F0585711BB945F00205C7
:107AB800857102E002F07D028271665470BD00BFDC
:107AC800308700200278837912F0010F14BF43F049
:107AD800010323F0010383715310827902F07F01BF
:107AE80010B58171DCB21BB941F00201817102E06D
:107AF80002F07D028271047010BD70470B4B5A5C16
:107B080003781A43837912F0800F02D063F07F0361
:107B180005E003F07F0312B943F0020303E0837129
:107B2800837923F002038371027070473087002045
:107B380030B5124C8279635CD5074FEA430348BFDE
:107B480043F00103FF2BDDB28CBF42F0010222F0AB
:107B5800010213F0800F8271827914BF62F07F02F4
:107B680002F07F028271827915B942F0020201E0C7
:107B780022F002028271635430BD00BF30870020BA
:107B880082790378D1074FEA430348BF43F00103E2
:107B9800FF2BD9B28CBF42F0010222F0010213F090
:107BA800800F8271827914BF62F07F0202F07F0237
:107BB8008271827911B942F0020201E022F00202D8
:107BC8008271037070470000827910B5114C12F071
:107BD800010F635C18BF43F4807313F0010F4FEA81
:107BE800630314BF42F0010222F0010213F0800F78
:107BF8008271827914BF62F07F0202F07F02827183
:107C0800827913B942F0020201E022F00202827185
:107C1800635410BD3087002082790378D10748BFAC
:107C280043F48073D9074FEA63034CBF42F0010263
:107C380022F0010213F0800F8271827914BF62F082
:107C48007F0202F07F028271827913B942F0020248
:107C580001E022F002028271037070478279234B9F
:107C680030B55C5C02F00103017883F001030D1B61
:107C7800EB1A1D064CBF62F07F0202F07F0213F080
:107C8800FF0F827182790CBF42F0020222F00202D9
:107C9800827181EA030212F0800F827906D084EAA9
:107CA80001052D0602D542F0400201E022F0400213
:107CB8008271827915070ED502F0010501F00F01D6
:107CC80004F00F0485F00105491BA142B8BF063B2B
:107CD800992B02D9603BFF2B02D842F0010201E048
:107CE80022F001028271037030BD00BF308700208E
:107CF800837943F0010383717047837943F0080364
:107D080083717047837943F00403837170470000DF
:107D18000278014B5A547047308700204278014B53
:107D28005A547047308700208278014B5A54704764
:107D3800308700200278837912F0800F02D063F038
:107D48007F0305E003F07F0312B943F0020303E069
:107D58008371837923F0020383714270704702783C
:107D6800837912F0800F02D063F07F0305E003F0FF
:107D78007F0312B943F0020303E08371837923F090
:107D88000203837182707047C278837912F0800F82
:107D980002D063F07F0305E003F07F0312B943F0DC
:107DA800020303E08371837923F002038371427035
:107DB80070474278837912F0800F02D063F07F0316
:107DC80005E003F07F0312B943F0020303E0837177
:107DD800837923F002038371027070474378C3707C
:107DE80070478278837912F0800F02D063F07F03A6
:107DF80005E003F07F0312B943F0020303E0837147
:107E0800837923F002038371027070470378054A6F
:107E1800134483F8001103780BB9FF2300E0013BFA
:107E280003707047308700208188013138B589B2E6
:107E3800C51C04468180090A2846FFF7E7FF217917
:107E48002846FFF7E3FFA179284641F01001FFF724
:107E5800DDFFA379064A43F00403A3714FF6FF73CD
:107E6800D15C4FF6FE73D35C03EB0123A38038BDCE
:107E78003087002070B50E468188C51C044601393C
:107E880089B28180090A2846FFF7C0FF2179284670
:107E9800FFF7BCFFA68070BD10F8031BFFF7B6BF45
:107EA8008179033041F01001FFF7B0BF0378054A2C
:107EB800FF2B0CBF0023013303700378134493F89E
:107EC80000017047308700200146033008B5FFF7EE
:107ED800EDFF10F0800F08708B7902D063F07F03FC
:107EE80005E003F07F0310B943F0020303E08B7150
:107EF8008B7923F002038B7108BD0146033008B566
:107F0800FFF7D4FF40F02000887108BD38B5C51CC4
:107F180001462846FFF7CAFF88712846FFF7C6FFC3
:107F280004462846FFF7C2FF44EA0020888038BD8F
:107F380038B5C51C04462846FFF7B8FF0146284651
:107F4800FFF7B4FF41EA00200130A08038BD0020CF
:107F5800704700002DE9F04F024600F5A055DFF804
:107F6800D0E30021F14F0023C2F808E0D1601432B9
:107F780042F8047C11601371AA42ED4CF3D1ED4D27
:107F88000221ED4A4FF0030EC0F8EC574FF0050BF5
:107F9800EA4DEB4FEB4EDFF8C0C3DFF8C083DFF8E4
:107FA800C093C0F83C280422C0F89C570625C0F8A6
:107FB800DC78E54FC0F84498C0F88C68C0F894980D
:107FC80080F89C28C0F8F497C0F8A49780F8AC57BC
:107FD800C0F8E49880F8EC58C0F8349980F83C2947
:107FE800C0F84038C0F8483880F84C18C0F89038C5
:107FF800C0F89838C0F8F037C0F8F83780F8FCE7D0
:10800800C0F8A037C0F8A837C0F8E038C0F8E8389A
:10801800C0F82CC9C0F83039C0F83839C0F8CC8954
:10802800C0F8D039C0F8D499C0F87C79C24FC0F8EC
:108038008499C0F83C73BF4FDFF82893C0F8EC72FE
:10804800BE4F80F8DC29C0F89C72BD4F80F88C299F
:10805800C0F8DC73BC4FC0F84493C0F88C63C0F818
:10806800949380F89C23C0F8F492C0F8A49280F806
:10807800AC52C0F8E493C0F8D839C0F88039C0F8D9
:108088008839C0F84033C0F8483380F84C13C0F83A
:108098009033C0F89833C0F8F032C0F8F83280F85E
:1080A800FCE2C0F8A032C0F8A832C0F8E033C0F84B
:1080B800E83380F8ECB3DFF8B0A2C0F82CC4C0F8FD
:1080C8007C749C4FC0F83494C0F8D494C0F884945D
:1080D800C0F88070DFF89492C0F8D8A09B4FDFF802
:1080E80090A280F83C2480F8DC2480F88C24C0F826
:1080F8002061C0F8289180F83051C0F88890C0F805
:10810800D0704FF00707C0F8C891C0F83034C0F8F5
:108118003834C0F8CC84C0F8D034C0F8D834C0F8AB
:108128008034C0F88834C0F82431C0F82C31C0F845
:108138008430C0F88C3080F890B0C0F8D430C0F8E3
:10814800DC3080F8E010C0F8C0C1C0F8C431C0F815
:10815800CC31C0F850ABDFF81CA2C0F86892C0F868
:10816800D0AD41F2C82ADFF8109280F8D05180F8DB
:108178007072C0F8489BC0F8C89DC0F86082C0F80B
:108188006432C0F86C32C0F84C3BC0F8543B80F8FD
:10819800581BC0F8CC3DC0F8D43D80F8D81D40F835
:1081A8000A9041F2CC2A6A4F40F80A3041F2D02AAC
:1081B80040F80A7041F2D42A5E4F40F80A3041F282
:1081C800D82A00F80A10DFF8B4A1C0F87863C0F81C
:1081D80080A3C0F8E0A2DFF8A8A180F88823C0F83F
:1081E800D872C0F8C893C0F87C33C0F88433C0F89C
:1081F800DC32C0F8E43280F8E8E2C0F8CC33C0F8EA
:10820800D0A341F2480AC0F8D43380F8D81340F814
:108218000A9041F24C0A4F4F40F80A3041F2500A96
:1082280040F80A7041F2540A4FF0070740F80A3044
:1082380041F2580A00F80A10C0F84891C0F8489668
:10824800C0F8C898DFF83CA1DFF83C91C0F850A10D
:10825800C0F8D098DFF834A1DFF83491C0F810A046
:10826800C0F8F09141F2E809DFF828A10776C0F8D4
:1082780050A6C0F84C31C0F8543180F858118460C9
:10828800C3604361C0F84C36C0F8543680F85816BD
:10829800C0F8CC38C0F8D43880F8D818C0F8E8410D
:1082A800C0F8EC31C0F8F43180F8F81140F8094012
:1082B80041F2EC09DFF8E0A040F8093041F2F0099A
:1082C8001D4F40F809A041F2F40941F20C0A40F8A8
:1082D800093041F2F80900F80910DFF8C090C0F839
:1082E800BC7FC0F8F096DFF8B890C0F8E846C0F850
:1082F800709EDFF8B090C0F8EC36C0F8C49FC0F8A4
:10830800F43680F8F816C0F8684EC0F86C3EC0F82D
:10831800743E80F8781EC0F8C03FC0F8C83F80F8A7
:10832800CC1F40F80A6041F2100A3DE0FD20000031
:10833800E51F0000D51F0000A91F0000B5200000A0
:10834800D9200000B51F000091200000BF2A0000BE
:108358009B220000ED2200003D2000006D2000005F
:1083680009210000C521000045220000F921000074
:108378008722000091220000E91F0000A5220000CA
:10838800E1220000F72200000D23000099290000D7
:108398001723000003230000212300002B230000E3
:1083A8003523000041230000F74F40F80A3041F21E
:1083B800140A40F80A9041F2180A40F80A3041F2CB
:1083C8001C0A00F80A2041F25C0AC0F86C7FEF4FE3
:1083D800C0F8749FC0F81C7FED4FC0F8703FC0F81C
:1083E800783F80F87CEFC0F8203FC0F8249F80F8E1
:1083F8002C5FC0F8283F40F80A7000F5835AE54F13
:10840800CAF8003041F2640A40F80A9041F2680A5A
:1084180040F80A3041F26C0A00F80AE041F2AC0A6E
:1084280040F80AC041F2B00A40F80A3041F2B40AF2
:1084380040F80A9041F2B80A40F80A3041F2BC0A02
:1084480000F80A2041F24C1A40F80A8041F2501A0A
:1084580040F80A3041F2541A40F80A9041F2581A8A
:1084680040F80A3041F25C1A00F80A2041F2FC0A8E
:1084780040F80A7000F5885AC74FCAF8003041F230
:10848800041A40F80A9041F2081941F2901A40F88B
:10849800093041F20C1900F8092041F2881940F816
:1084A800097041F28C19B84F40F80930DFF8EC92A6
:1084B80040F80A9041F2941A40F80A3041F2981AAA
:1084C80000F80A1041F2782A40F80A6041F27C2A42
:1084D80040F80A3000F5945ACAF8009041F2842A0C
:1084E80040F80A3041F2882A00F80A2041F2D81AE6
:1084F80040F80A7041F2DC1AA74F40F80A3000F53C
:108508008F5ACAF8009041F2E41900F5805A40F8F1
:10851800093041F2E81900F809E0DFF88492C0F860
:10852800087FC0F8109FC0F8F86FC0F80C3FC0F87B
:10853800143F80F8181FC0F8FC3FCAF8009041F2B9
:10854800040A914F40F80A3041F2080A00F80A205C
:1085580041F2280AC0F8609F00F58159C0F8587F99
:10856800C0F85C3FC0F8643F80F868EFC9F8006065
:1085780041F2240940F80930DFF8289240F80A90BF
:1085880041F22C0A40F80A3041F2300A00F80A5049
:1085980000F5865AC0F8807F4FF00707C0F8889F1B
:1085A800C0F8843FC0F88C3F80F890BFCAF800C07C
:1085B80041F2C40A40F80A3041F2C80A40F80A9069
:1085C80041F2CC0A40F80A3041F2D00A00F80A50C9
:1085D80000F58B5ACAF8008041F2641A40F80A3054
:1085E80041F2681A40F80A9041F26C1941F2A82A3F
:1085F80040F8093041F2701900F80970664FDFF849
:10860800A891C0F8BC75604FC0F8D89FC0F86C75C9
:10861800DFF898915D4FC0F8B09AC0F81C75DFF884
:1086280090915B4FC0F8C495C0F80C66C0F81496DA
:1086380080F81C26C0F87495C0F8D04FC0F8D43F15
:10864800C0F8DC3F80F8E01FC0F8A84AC0F8AC3A90
:10865800C0F8B43A80F8B81AC0F8C035C0F8C835C0
:1086680080F8CC15C0F81036C0F81836C0F8703548
:10867800C0F8783580F87CE5C0F82035C0F8249536
:10868800C0F85C76C0F86496C0F8B496C0F8549701
:10869800C0F8049700F595593E4F80F82C5580F89E
:1086A800BC2680F85C27C0F8FC7680F80C27C0F858
:1086B8002835C0F86036C0F8683680F86CB6C0F85F
:1086C800ACC6C0F8B036C0F8B836C0F84C87C0F8A9
:1086D8005037C0F85837C0F80037C0F80837C9F81D
:1086E800006041F2A429284F40F80930DFF8C4900F
:1086F80040F80A9041F2AC2A40F80A3041F2B02A18
:1087080000F80A5000F5905ACAF8007041F2042A9D
:108718004FF0070740F80A3041F2082A40F80A905B
:1087280041F20C2A40F80A3041F2102A00F80AB047
:1087380000F59A5ACAF800C041F2443A40F80A30A3
:1087480041F2483A40F80A9041F24C3A40F80A306F
:1087580041F2503A00F80A5000F59F5ACAF80080D2
:1087680041F2E43A40F80A3041F2E83A40F80A9017
:1087780041F2EC39DFF840A040F8093041F2F03915
:1087880000F809701AE000BFD51F0000B5200000EE
:10879800D920000091200000A91F000085230000B7
:1087A800C92300000D2400004524000071240000A6
:1087B8009D240000D12400000925000041F2282949
:1087C800F14F40F8094041F22C2940F8093041F2B4
:1087D800302940F809A041F23429DFF8C8A340F84D
:1087E800093041F2382900F80910DFF8BC93C0F8C5
:1087F800F865C0F8B09FDFF8B493C0F878A8C0F85F
:108808000096C0F88098DFF8A893C0F88862C0F88E
:10881800A84FC0F8AC3FC0F8B43F80F8B81FC0F804
:10882800FC35C0F8043680F808E6C0F87C38C0F893
:10883800843880F888B8C0F88C32C0F89092C0F8B4
:108848003C7DD24FDFF86C93C0F8EC7CD04F80F8B9
:108858009852C0F89C7CCF4FC0F8449DC0F8DC7D8E
:10886800CD4FC0F88C6DC0F8949D80F89C2DC0F851
:10887800F49CC0F8A49C80F8AC5CC0F8E49DC0F8F7
:10888800349E80F83C2EC0F89432C0F8403DC0F8C1
:10889800483D80F84C1DC0F8903DC0F8983DC0F8A0
:1088A800F03CC0F8F83C80F8FCECC0F8A03CC0F8FC
:1088B800A83CC0F8E03DC0F8E83D80F8ECBDC0F841
:1088C8002CCEC0F8303EC0F8383EC0F8CC8EC0F888
:1088D8007C7EAD4FC0F8D49EC0F8B07CAB4FC0F8DA
:1088E800849EC0F8007DAC4FDFF8CC92C0F8E07EE3
:1088F800AA4F80F8DC2EC0F8407EA34F80F88C2E5B
:10890800C0F8B89CC0F8A06DC0F8A89D80F8B02D3C
:10891800C0F8089DC0F8E89E80F8F02EC0F8489E80
:10892800C0F8D03EDFF89492C0F8D83EC0F8803E38
:10893800C0F8883EC0F8B43CC0F8BC3C80F8C01C05
:10894800C0F8A43DC0F8AC3DC0F8043DC0F80C3DEB
:1089580080F810EDC0F8E43EC0F8EC3EC0F8443EA4
:10896800C0F84C3EC0F8887C884FC0F8909CC0F88E
:10897800809DC0F8D87CC0F8E09CC0F8209EC0F864
:10898800C09EC0F88075DFF83892854F80F8502E69
:10899800C0F8786D80F8882D80F8282E80F8C82EC9
:1089A800C0F82066C0F8289680F83056C0F88C3C8D
:1089B800C0F8943C80F8981CC0F87C3DC0F8843D11
:1089C800C0F8DC3CC0F8E43C80F8E8ECC0F818CE0D
:1089D800C0F81C3EC0F8243EC0F8B88EC0F8BC3EB3
:1089E800C0F8C43EC0F82436C0F82C36DFF8D4A14D
:1089F800C0F88435C0F88895C0F8D0754FF00707DF
:108A0800C0F8C896C0F8689741F25029C0F8D8A5B0
:108A180080F8D05680F87077C0F88C3580F890B51B
:108A2800C0F8D435C0F8DC3580F8E015C0F8C0C609
:108A3800C0F8C436C0F8CC36C0F86087C0F86437D0
:108A4800C0F86C3740F8094041F25429DFF878A1A2
:108A580040F8093041F258294B4F40F809A041F23B
:108A68005C29DFF868A140F8093000F5935989F8C6
:108A78000010DFF85C91C0F8BC70444FC0F8C49097
:108A8800C0F80C61C0F81491C0F8C030C0F8C83004
:108A980080F8CC10C0F81031C0F8183180F81C21CB
:108AA800C7663B4FC0F87490C7613A4FC0F824902E
:108AB800C0F85C71C0F86491C0F8B491C0F85492E1
:108AC800C0F80492344FDFF80C9180F82C5080F8ED
:108AD800BC2180F85C22C0F8FC7180F80C22036786
:108AE800836780F87CE003628362C0F86031C0F875
:108AF800683180F86CB1C0F8ACC1C0F8B031C0F8CA
:108B0800B831C0F84C82C0F85032C0F85832C0F8BA
:108B18000032C0F80832C0F8A845C0F8AC35C0F833
:108B2800B095DFF8B490194FC0F8B090DFF8AC906A
:108B3800C0F80073C0F83098194FDFF8A490C0F857
:108B480050734FF00707C0F83093DFF8989080F81B
:108B5800382880F83823C0F8A063C0F8A89380F8B4
:108B6800B053C0F80893C0F858A3C0F8B43580F8DB
:108B7800B8E5C0F8A840C0F8AC30C0F8B43080F808
:108B8800B8E0C0F828482FE0A91F0000D51F000052
:108B9800B5200000D92000009120000055200000D9
:108BA800BF2A0000092000003525000061250000CB
:108BB800E52900006525000095250000C525000071
:108BC800F5250000352600006B260000F126000080
:108BD8006D260000092A0000112A0000392A000029
:108BE8006B2A0000A1260000C0F82C38C0F83438E1
:108BF800C0F82843C0F82C33C0F83433C0F8A43385
:108C0800C0F8AC33C0F80433C0F80C3380F810B3A4
:108C1800C0F85433C0F85C3380F86013C0F840C41F
:108C2800C0F84894C0F8E89480F8F074DFF80C9421
:108C3800F34FC0F8A898C0F80078C0F80898C0F8B2
:108C48004899C0F8E899EF4FDFF8F4A3DFF8F493F8
:108C580080F85054C0F8A06880F8B058C0F8507830
:108C68004FF00707C0F858A841F2442A80F8505935
:108C7800C0F84434C0F84C34C0F8E084C0F8E43498
:108C8800C0F8EC34C0F8A438C0F8AC38C0F80438E0
:108C9800C0F80C3880F810B8C0F85438C0F85C3800
:108CA80080F86018C0F840C9C0F84439C0F84C3999
:108CB800C0F8E089C0F8E439C0F8EC39C0F810957C
:108CC800DFF8849380F8F079C0F8909741F23C2956
:108CD800CD4F80F8185580F89857C0F80845C0F867
:108CE8000C35C0F81435C0F88847C0F88C37C0F880
:108CF800943740F8097000F59259C14FC9F800300F
:108D0800DFF8489340F80A9041F2482A40F80A30C0
:108D180041F24C2A00F80A1041F28C2A40F80A6005
:108D280041F2902A40F80A3041F2942A40F80A9019
:108D380041F2982A40F80A3041F29C2A00F80A20A9
:108D480041F2EC1A40F80A7041F2F01AAF4F40F8BD
:108D58000A3041F2F41A40F80A9041F2F81A40F841
:108D68000A3041F2FC1A00F80AE041F29C1A40F875
:108D78000A7000F58D5AA64FCAF8003041F2A41ABD
:108D880040F80A9041F2A81A40F80A3041F2AC1AA9
:108D980000F80A5041F2DC2A40F80A7000F5975AA8
:108DA8009C4FCAF8003041F2E42A40F80A9041F298
:108DB800E82A40F80A3041F2EC2A00F80AB041F2F9
:108DC8002C3A40F80AC041F2303A40F80A3041F2F1
:108DD800343A40F80A9041F2383A40F80A3041F201
:108DE8003C3A00F80A2041F2CC3A40F80A8041F2B5
:108DF800D03A40F80A3041F2D43A40F80A9041F2A9
:108E0800D83A40F80A3041F2DC3A00F80A2041F238
:108E18007C3A40F80A7000F59C5A794FCAF800303D
:108E280041F2843A40F80A9041F28839DFF820A2EA
:108E380040F8093041F28C3900F80920DFF8149223
:108E4800C0F86844C0F8709441F26839C0F86C34CE
:108E5800C0F8743480F8781440F8094041F26C394D
:108E680040F8093041F2703940F809A041F27439EC
:108E780040F8093041F2783900F80910DFF8D89144
:108E8800C0F86849C0F87099C0F86C39C0F87439EE
:108E980080F87819C0F86C7A5C4F80F82C5AC0F8C2
:108EA8001C7A80F86C5B5A4F5A4DDFF8B091C0F8C5
:108EB8005C7BC0F8FC5B524F574DC0F80C6B80F8D8
:108EC8001C2B80F8BC2BC0F8103BC0F8149BC0F8D2
:108ED800183BC0F8703AC0F8749AC0F8783A80F82D
:108EE8007CEAC0F8203AC0F8249AC0F8283AC0F8BA
:108EF800603BC0F8649BC0F8683BC0F8ACCBC0F8D6
:108F0800B03BC0F8B49BC0F8B83BC0F84C8CC0F874
:108F1800503CC0F8549CC0F8583C80F85CBCC0F881
:108F2800003CC0F8049CC0F8206BC0F8285B80F8AF
:108F3800302BC0F8807AC0F8885AC0F8C85B80F82F
:108F4800D02B364DC0F8F86A80F8082B80F8A82B8B
:108F5800334F2B4E334AC0F8083C80F80CBCC0F89D
:108F6800243BC0F82C3BC0F8843AC0F88C3A80F80F
:108F780090EAC0F8C07BC0F8C43BC0F8CC3BC0F84E
:108F8800FC3AC0F8005BC0F8043BC0F8586AC0F867
:108F98005C3AC0F8605AC0F8643A80F868EAC0F8E9
:108FA80098CBC0F89C3BC0F8A05BC0F8A43BC0F8C5
:108FB800504DC0F8582D1C4AC0F8543DC0F8302D0B
:108FC8001A4AC0F85C3DC0F8982E194A80F8601D0E
:108FD800C0F8D82A174AC0F8284DC0F8182C164AE5
:108FE800C0F82C3DC0F8343D80F8381DC0F8904ECC
:108FF800C0F8943EC0F89C3E80F8A01E30E000BF48
:10900800D51F0000BF2A0000A91F0000B5200000DE
:10901800D9200000912000008D2800009928000028
:1090280055200000A5280000CF280000F9280000DE
:10903800232900004D29000053290000392700008A
:10904800892700007D2A0000A12A0000CD27000002
:109058006B280000612800007528000081280000A6
:10906800C0F8D04AC0F8D43AC0F8DC3A80F8E01A20
:10907800C0F8104CC0F8143CC0F81C3C80F8201C08
:10908800C0F8E84BC0F8EC3BC0F8F02BC0F8F43B54
:1090980080F8F81BBDE8F08F00230C494FF6FD72ED
:1090A80003708370437010B58C5C4FF6FC728A5C59
:1090B80002EB04228280FD22C270827942F02002F3
:1090C800827141F20842835410BD00BF30870020EE
:1090D80038B5837904465A0720D423F01003C51CF9
:1090E800818883712846090AFEF790FE217928466F
:1090F800FEF78CFEA1792846FEF788FEA379084A78
:10910800012043F00403A3714FF6FF73D15C4FF6BF
:10911800FE73D35C03EB0123A38038BD002038BD68
:109128003087002084B070B5064605A880E80E0098
:1091380006A80B4631C810F0010F4FEA600018BFAF
:109148003258304418BF5358984715F0010F01465C
:109158004FEA65000CBF23463358304418BF1B59EB
:10916800BDE8704004B018472DE9F04F00F5A0584D
:1091780089B006460F4691464FF0000A4FF0000BA3
:1091880008F10808002F2CDD98F800304BBBB38895
:1091980003AD5A1CB280154A12F803E0142303FBEE
:1091A8000EFE06EB0E04B64408340FCC0FC5236838
:1091B8009EF818402B6008AB8DF81C4013E903009B
:1091C80003AB8DE8030030460ECBFFF7ABFF1AEB7D
:1091D800040A4BF1000BB9F1010F18BF01243F1B22
:1091E800D0E75046594609B0BDE8F08F30870020D7
:1091F800034B1A780AB1002200E001221A70704766
:10920800BC3B002010B504460BF01AFE204610BDEA
:10921800094B82B000211A78D2B28DF80720074A8C
:109228001160074A127822B919789DF807209142EF
:10923800FAD002B0704700BFBC3B0020747A00200F
:109248002F870020034B01461B7813B9024800F012
:1092580099BC70472F8700201F87002008B5034856
:1092680000F046FABDE80840FDF728BF1F87002038
:1092780038B5FDF763FE20B3FDF7E2FBFDF7D2FC3E
:109288000446FDF76BFE0546812C18D1002000240A
:10929800FDF75AFE104B1C70FEF710F800F0CCFEDC
:1092A800284600F047FF21460C4800F0DDFA0B483D
:1092B80000F08EFC0A4A0B490B480BF065FD1420A0
:1092C80006E0FDF7BDFB00F095FE00F0CBFF0A209D
:1092D800BDE838400AF08EBB2F8700201F8700208A
:1092E800FF520700613D0000183B002010B50A211D
:1092F800084C09480BF034FB08480BF0DFFD20460A
:10930800074A4FF480710DF007F92046BDE8104078
:10931800FCF76CB909870020B9360020883A00208C
:10932800F10000007FB5FF231A211B220A4804938D
:10933800039302938DE806001722162100F01CF90A
:10934800064A074907480CF072F90AF025FB064B54
:10935800186007B05DF804FB1F870020DC39002087
:10936800753D0000183B0020787A0020154B1649FF
:1093780010B51879154BC8771A78154C013224782E
:10938800D2B21A701A78944208D800221A70114A78
:1093980012781AB1887601210F4A11701A780F4B8A
:1093A80053F8222022F01F0302F52042BFF34F8F0B
:1093B8000B490B6020339A42FBD8BFF34F8FBFF3A2
:1093C8006F8F10BD7C7A002000800E40157C002035
:1093D800137C0020AF860020AB8300208C7A00200D
:1093E80068EF00E010B504460BF046FC204610BDBF
:1093F80013B502AB03E90600C37C0099002B2ED0FD
:1094080072B6C37CDA0705D5324A4369146823402B
:1094180083621360C37C9B0705D52F4A8369146850
:109428002340C3621360C37C5C0705D52B4AC3691C
:109438001468234003631360C37C1A0705D5284AC0
:10944800036A1468234043631360C37CDB0605D5B5
:10945800244A436A146823408363136062B68368AE
:109468008B422AD0204B81609A69204BC2F30114A9
:10947800C2F3826253F824300132B3FBF2F211B125
:10948800B2FBF1F300E013467BB1B2FBF3F2914279
:1094980038BF0133B3F5817F02D2022B04D901E032
:1094A80040F20113023B00E000235A0843EA02237A
:1094B800120402F47F021343C360036800221A6196
:1094C80003225A62C2681A64019A1A6601221A6152
:1094D80002B010BD80E100E084E100E088E100E036
:1094E8008CE100E090E100E000C00F403809002066
:1094F80003685966DA6D12F4F81FFBD0586FC0B2D2
:1095080070470368186E20F47F6222F00F0242F061
:109518000F021A6659661A6F9207FCD41866586FBC
:1095280080B27047C37CE3B1DA0702D5826A0D4B7B
:109538001A60C37C9B0702D5C26A0B4B1A60C37CB6
:10954800590702D5026B094B1A60C37C1A0702D56A
:10955800426B074B1A60C37CDB0602D5826B054B56
:109568001A60704700E100E004E100E008E100E073
:109578000CE100E010E100E070B50446FF209DF822
:109588001C6023709DF81030A07123719DF8143071
:10959800E071002063719DF81830A270E3702072AA
:1095A8001046617001219DF820500AF06BFA0121E4
:1095B80060780AF067FA012160780AF031FA01212F
:1095C800A0780AF02DFAFF2E0FD0FF2D0DD0012123
:1095D8003046A571E6710AF055FA022128460AF0CC
:1095E80051FA0121E0790AF01BFA204670BD00000B
:1095F8002DE9F843224D0446894680780021174614
:109608009846BDF820600AF00BFA2A212846FFF791
:109618006FFFA07801210AF003FA49462846FFF7B0
:1096280070FFA07801210AF0FBF941462846FFF7B0
:1096380068FFA07800210AF0F3F92B212846FFF7EC
:1096480057FFA07801210AF0EBF939462846FFF7C1
:1096580058FFA07801210AF0E3F931462846FFF7C0
:1096680050FFA07800210AF0DBF92C212846FFF7EB
:109678003FFFA0780121BDE8F8430AF0D1B900BF47
:10968800383A002037B5174B0446174A0D46174895
:109698008DE80C0002AB13E90600FFF7A9FE0021D4
:1096A800A0780AF0BDF9002160780AF0B9F93621EE
:1096B8000E48FFF71DFF0121A0780AF0B1F91DB18E
:1096C8000123A021237201E0602125720748FFF7DA
:1096D8000FFF012160780AF0A3F90448FFF722FF81
:1096E80003B030BD0700008000879303383A00209C
:1096F8002DE9F04F044685B00179564800F0B6FFD1
:10970800E178544800F0E4FF6179524801F00CF820
:10971800504800F09FFE2078FF2817D001210AF05A
:10972800B1F9012120780AF07BF964200AF062F986
:10973800002120780AF074F964200AF05BF9207897
:1097480001210AF06DF9C8200AF054F9424D0DF1D3
:109758000808DFF810A10A260395A946CDF808A045
:109768003C483E4F98E80600FFF742FE002160782B
:109778000AF056F9013E16F0FF064DD03D4600218D
:10978800A0780AF04DF915F8021B3248FFF7B0FE31
:109798007F7827F07F0B07F07F075FFA8BFB012F9D
:1097A8000BD90121A078013F0AF03AF915F8011BFD
:1097B8002848FFB2FFF79CFEF1E74FB16F1C01216B
:1097C800A0780AF02DF929783D462248FFF790FE47
:1097D800BBF1000F01D12F46CCE76F1C2D7801217A
:1097E8006078FF2D08BF4FF4FA750AF019F9194887
:1097F800FFF798FE28460AF0FDF8CDF808A0CDF846
:109808000C903D46134898E80600FFF7F1FD00214B
:1098180060780AF005F9DEE7607801210AF000F9BE
:10982800EF23324631460093204640F23F13FFF7BC
:10983800DFFE0848FFF776FE094B314620461E70CA
:10984800FFF720FF0121204605B0BDE8F04FFFF7E4
:1098580019BF00BF383A002007000080911F006040
:10986800AF86002000879303F0B51B4B85B00446F4
:109878000F460293F025194B1948039304AB13E9DB
:109888000600FFF7B5FD002160780AF0C9F8EF235C
:1098980000222046009340F23F131146FFF7A8FE2E
:1098A8004FF4A07639460E48FFF72BFE013EF9D15A
:1098B800013DF5D1607801210AF0B2F8EF232A467C
:1098C80029460093204640F23F13FFF791FE0448D3
:1098D800FFF728FE05B0F0BD00879303070000805E
:1098E800383A00202DE9F0431D4685B01F4B044649
:1098F800BDF930708846029391461D4B1D4803936D
:1099080004ABBDF8346013E90600FFF771FD0021D0
:1099180060780AF085F8781E1FFA89F26B1E1FFA24
:1099280088F17D43104400270B4480B29BB200901D
:109938002046FFF75DFEAF4205DA31460D48FFF7D6
:10994800E0FD0137F7E7607801210AF069F80022A5
:10995800EF2320461146009340F23F13FFF748FEDD
:109968000448FFF7DFFD05B0BDE8F08300879303E7
:1099780007000080383A00202DE9F04F89B09B4657
:109988001FFA82FA81469DF850308846BDF8485043
:10999800002B0393BDF84C6014BF0F2307235344D7
:1099A8009BB204931BF8017B06AB002F00F0BF802D
:1099B800704A1FFA88F8704802EBC7076F4A069288
:1099C8006F4A079293E80600FFF712FD002199F805
:1099D80001000AF025F8049A08F1070341460092AD
:1099E80048469BB25246FFF703FE07F1080305936A
:1099F800039B002B44D03C785F48E2074FEA64049D
:109A08004CBF29463146FFF77CFDE3074FEA640463
:109A180059484CBF29463146FFF773FDE0074FEA26
:109A2800640455484CBF29463146FFF76AFDE107F3
:109A38004FEA640450484CBF29463146FFF761FDA0
:109A4800E2074FEA64044C484CBF29463146FFF709
:109A580058FDE3074FEA640447484CBF294631469E
:109A6800FFF74FFDE00744484CBF29463146FFF752
:109A780048FD6308404814BF29463146FFF741FDB9
:109A880017F8014B3C48E1074FEA64044CBF2946EC
:109A98003146FFF736FDE2074FEA640436484CBF0B
:109AA80029463146FFF72DFDE3074FEA64043248A3
:109AB8004CBF29463146FFF724FDE0074FEA64040E
:109AC8002D484CBF29463146FFF71BFDE1074FEAF9
:109AD800640429484CBF29463146FFF712FDE207C6
:109AE8004FEA640424484CBF29463146FFF709FD74
:109AF800E30721484CBF29463146FFF702FD6308BA
:109B08001D4814BF29463146FFF7FBFC059B9F42C1
:109B18007FF46EAF99F80100012108F1080809F0F7
:109B28007FFF15480FFA88F8FFF7FCFC3AE7134A5D
:109B380011480692124A079293E80600FFF758FC6C
:109B4800394699F8010009F06BFFEF233A46394688
:109B58000093484640F23F13FFF74AFD012199F868
:109B6800010009F05DFF0448FFF7DCFC09B0BDE81F
:109B7800F08F00BFB31F0060383A002000879303BE
:109B8800070000808A11054B01F03F014FF4207057
:109B980053F8223000FB0130704700BF8C7A002058
:109BA80030B5002209484FF42074951102F03F03A4
:109BB80050F8255004FB035303F5207523F8021BC6
:109BC800AB42FBD10132F02AEFD130BD8C7A0020B4
:109BD8002DE9F04F844B0024074684481C7087B059
:109BE80002798046824B02F11001824D1C70824B33
:109BF800DFF808B243F821505311012102F01F0287
:109C08009B004FF4163501FA02F203F1604303F5A5
:109C180061431A60B5F5204F5BF824202E464FEAC1
:109C2800840928BF4FF420462AB906F140000BF0FA
:109C380049FD20F01F02714B43F8092082B9252104
:109C48006F4803920AF08CFE21466E480BF095F996
:109C58006C480BF033F942F2107009F0CBFE039A0E
:109C680026F00101134600201144994202D023F83E
:109C7800020BFAE7A101DFF8ACA14FF00109AD1B17
:109C880051F80A3001F140014C441A604FF00202C9
:109C980083F807909A609A80C6F1000283F80690CC
:109CA800DA60C6F34F02DA83DA82574A1A614FF054
:109CB80000029A8251F80A209A619A8B22F0800257
:109CC8004FEA02424FEA12429A839A8B92B242F0CA
:109CD80010029A839A8B92B242F002029A8399D127
:109CE800DAF80020294638469A619A8B22F08002D9
:109CF8001204120C9A839A8B92B242F010029A8341
:109D08002A46424B1C70EF2440F23F130094FFF7A1
:109D18006FFC29463846FFF743FF4946787809F033
:109D28007FFE3B4800F096FB3A4B394804930723E3
:109D3800059306AB13E90600FFF75AFB364B1A6981
:109D480022F001021A615A6A42F008025A620F228E
:109D58001A66C3F81C901A6942EA09021A6198F84F
:109D680004302E4A9B0003F1804303F56C231D60E9
:109D78001A60D8F80030DAF80020998B101D21F00D
:109D88008001090490E84140090C998311685860E2
:109D980002F11400C3F80CE019609E60166907C848
:109DA8001E6199612946DA615861787809F038FEB0
:109DB8002A4640F23F13294638460094FFF718FC1C
:109DC8002946B87809F02CFE2C211148FFF790FBA2
:109DD8004946B87809F024FE98F80420104BDA7642
:109DE80007B0BDE8F08F00BF157C00207C7A00200A
:109DF800AB830020DD3E0000003C00208C7A002070
:109E0800C4360020883A002064C03940137C002002
:109E1800383A00200087930300C0394010000080C2
:109E280000800E40804000200D4B1A4603F12001AF
:109E380010B542F8601B00211A6403F1A002094C16
:109E4800C3F8802003F1E0022046C3F8C0200AF0DE
:109E5800C5FE2046044A0549BDE810400BF0E7BBA3
:109E6800804000207C7A0020DC390020553F00002B
:109E780070B5D1F1FF040A4D4FF00C0608BF7F24DE
:109E880011F0800106FB005017BF6B6B4160C3EBFC
:109E9800034303FA02F21CBF92FBF4F3436070BD64
:109EA8003C7A00204FF0020C043091FBFCF32DE9C2
:109EB800F04F89B002934B4B1A681E6906925A6894
:109EC800DD690092DA689C6A05929A69069904929B
:109ED8005A6A0392DA6A93F830300793009B03EBCF
:109EE800010C059B002106EB0309049B8A4605EB40
:109EF8000308039B04EB030E0B46029FBA4554DA92
:109F0800744506DD9310012183EAE2139BB243EA0C
:109F180002424FEA2E730AF1010AA6440430C3F143
:109F2800170BC3F1120742FA0BFB42FA07F78BEA49
:109F3800070B01279F4002FA03F3013F0BEA0707CB
:109F48003B43294FC3F3072B0193C3F3074317F888
:109F58000BB0264FFF5C9DF804304BEA070B244FEB
:109F6800FB5C4FEA9C074BEA030B4FEA990307F0A7
:109F78000057B14403F000531F444FEA9803A84424
:109F880003F000533B44BDF81C7003EB8B531B15C7
:109F9800A3F5006313FB07F31BB220F8083C20F875
:109FA800063C009B9C440123A7E70298039F20EAF4
:109FB800E07004FB0074049F05FB0075059F06FB19
:109FC8000076009FBE46069F0EFB007023B1054B2E
:109FD8001860DE609D615C6209B1024BDA6209B00B
:109FE800BDE8F08F3C7A0020AF840020AF850020C8
:109FF800AF83002008B5FCF74FFB034B1860FCF754
:10A008002BFD024B186008BD206600202466002046
:10A01800A1F1C0031F2B044B96BF01F01F0101F0F3
:10A028007F017F31196070479C7A00200022014B24
:10A038001A6070479C7A002038B53248FFF72CF830
:10A048003148FBF723FC2F493048FBF7F1FA2F483A
:10A05800FBF7F8FA00232E491846585401332C4AC6
:10A06800B3F5803FF9D100232A4C03F50041185D70
:10A0780001335054B3F5805FF7D10023264C03F524
:10A088004041185D01335054B3F5005FF7D1002308
:10A09800224C03F56041185D01335054B3F5005F5D
:10A0A800F7D11F4B42F674521E4D5A631E4A1F4C7D
:10A0B800DA6200231E485A1102F00401DA1002F095
:10A0C80002020A43C3F380010A435A555A1002F0A8
:10A0D800100103F008020A4359001A559A0021F0AA
:10A0E8007F0102F0400211435A0102F020020A43A4
:10A0F8001A540133B3F5807FDDD1BDE83840FFF74E
:10A10800F5B800BF28660020C07A0020A87A002091
:10A1180030870020B3230060B33300604A14002066
:10A128003C7A0020AF830020F8FF7F00AF84002036
:10A13800AF8500202DE9F34104464548FCF790FA25
:10A148002046FCF78DFF434980462046FCF70AFF6E
:10A15800074620460BF023FC0023411E98420ADDE7
:10A16800E25C2E2A03F1010203D18B4201D0144490
:10A1780001E01346F2E72378374C03F0DF02502A58
:10A1880011D13A46022101A8FCF734FF9DF80430AA
:10A198009DF805503A46A8F1020143EA0525AB1E91
:10A1A80043449EB21CE0362B10D007D8322B0AD07D
:10A1B800342B0CBF4FF4804500250CE0412B08D010
:10A1C800612B06D007E04FF4005504E04FF4C0457A
:10A1D80001E04FF4204505EB08033A4641469EB29C
:10A1E8006019FCF707FF3846FCF71EFFFF21EBB2AA
:10A1F800C5F30725F2B2194884F82B3084F82D30BE
:10A20800330A84F82F2084F8303084F8323084F808
:10A21800343084F8AF3084F8312084F8332084F85F
:10A22800371084F8381084F8AE2084F82C5084F85D
:10A238002E50FEF731FF012244F620610748FEF751
:10A2480093FF0748FCF70CFA02B0BDE8F08100BFA5
:10A25800EA360020F73600203087002028660020E4
:10A26800FB36002038B5012254481146FEF77CFF22
:10A2780001215348FBF746FC5248FBF7DFFA5148E7
:10A28800FBF7DCFA4E48FBF73AFC0028EBD04C48C9
:10A29800FBF735FC10B14A48FBF72EFCFEF7B8FF78
:10A2A800494B1C6814B9494B1C685CB1484B45487C
:10A2B80053F8244014F4803118BF0121FBF7BCF98E
:10A2C800A1B204E021463F48FBF7B6F921463D48D4
:10A2D800FBF7B0F93F4B404D1C6814F0600F46D1B6
:10A2E800296804F0100211F0100102D132B10122E4
:10A2F80001E01AB911463348FBF7A0F92B6804F0BE
:10A30800040213F0040F03D13AB10122114601E00F
:10A318001AB901212B48FBF791F92B6804F00802C0
:10A3280013F0080F02D132B1012200E01AB902215C
:10A338002448FBF783F92B6804F0010213F0010F9E
:10A3480002D132B1012200E01AB903211D48FBF7FE
:10A3580075F92B6804F0020213F0020F02D132B132
:10A36800012200E01AB904211648FBF767F9002218
:10A3780049F20A032C60194C1046E15CFFF778FD9E
:10A38800012249F20B031046E15CFFF771FD02223E
:10A3980049F20C031046E15CFFF76AFD49F20D0330
:10A3A80000220320E15CFFF763FD49F20E030C4A2B
:10A3B800E35C03F00F0382F8303038BD28660020D4
:10A3C800C07A0020A87A00209C7A00202466002009
:10A3D8008002002020660020347A00203087002088
:10A3E8003C7A002038B50C4C0C48FDF7B3FD0C4DF9
:10A3F8002046FBF735FA20460A4C2A460A490BF054
:10A4080016F92046FBF7FEF82A4620460749BDE81C
:10A4180038400BF00CB900BFC07A00202866002035
:10A42800DC390020A87A0020F10300009501000023
:10A43800C38B1B0402D4C1F30E0105E0C38BC1F327
:10A44800080103F47E431943C183C38B9BB2C382C3
:10A45800704700004368196830B50A685C6822EAEA
:10A468000402744C0A60A26922F0E05222F0300221
:10A4780042F0006242F01002A261047C6E4A1C4461
:10A48800247C02EB0414A568B8242C60457C1D4488
:10A4980095F8245002EB0515AD682C60857C1D44A9
:10A4A80095F8385002EB0515AD682C600D685C68AE
:10A4B8002C430C60017C5C1803EB8101247C496906
:10A4C80002EB041464682160417C5C180A3194F83A
:10A4D800244053F8211002EB041464682160817C45
:10A4E8005C1803EB810194F83840C96B02EB041245
:10A4F80052681160827C996C1A4492F844200A6070
:10A50800027C196A1A44127F0A60427C596B134410
:10A51800022293F830300B6003681A610F229A65A3
:10A52800C37C002B2ED072B6C37CDD0705D5434A09
:10A53800436911680B4083621360C37C9C0705D58F
:10A548003F4A836911680B40C3621360C37C590793
:10A5580005D53C4AC36911680B4003631360C37C8B
:10A568001A0705D5384A036A11680B40436313601C
:10A57800C37CDB0605D5354A436A11680B40836303
:10A58800136062B6324983688B4227D0294B8160B9
:10A598009A69304BC2F30114C2F3826253F8243033
:10A5A8000132B3FBF2F2B2FBF1F37BB1B2FBF3F28F
:10A5B8008A4288BF0133B3F5817F02D2022B04D9C6
:10A5C80001E040F20113023B00E000235A0843EA8D
:10A5D8000223120402F47F021343C36003680022BB
:10A5E8001A6103225A62C2681A6407221A66012293
:10A5F8001A61C37CE3B1DD0702D5826A164B1A6083
:10A60800C37C9C0702D5C26A144B1A60C37C5907E5
:10A6180002D5026B124B1A60C37C1A0702D5426B33
:10A62800104B1A60C37CDB0602D5826B0E4B1A6096
:10A6380030BD00BF00C00F40AC09002080E100E041
:10A6480084E100E088E100E08CE100E090E100E0D6
:10A6580000093D003809002000E100E004E100E0C5
:10A6680008E100E00CE100E010E100E04368427C12
:10A678001A4430B592F824208A4225D093F8242031
:10A68800914205D093F8252091421DD1012100E087
:10A6980000211C6825685C68254214D00B4CB8253D
:10A6A80004EB0212926815605A1892F8245004EBD1
:10A6B800051401F10A05646853F825505B6B2560A1
:10A6C80092F830201A60417430BD00BFAC090020F8
:10A6D8004368027C1A4430B5127C8A4221D01A7C25
:10A6E800914204D05A7C91421BD1012100E0002103
:10A6F8001C6825685C68254212D00A4CB82504EB12
:10A708000212926815605D182A7C04EB02140A1D77
:10A7180003EB820264681B6A526822602A7F1A600F
:10A72800017430BDAC0900204368827C1A4430B5FE
:10A7380092F838208A4226D093F83820914205D0E2
:10A7480093F8392091421ED1012100E000211C68B4
:10A7580025685C68254215D00B4CB82504EB02121D
:10A76800926815605D1895F8382004EB021401F121
:10A778000E0203EB820264689B6C5268226095F8B3
:10A7880044201A60817430BDAC09002070B54BB309
:10A79800046840F2012525611C46066811B10D7850
:10A7A800013101E090F83C50013C756605682E6F58
:10A7B800B60705D46D6FEDB20AB115700132013BD1
:10A7C80005686D69ED07F1D5002CE6D153B1016834
:10A7D8000C6FA407FAD4496FC9B20AB111700132DB
:10A7E800013BF3E770BD0000836C10B51A7904468D
:10A7F8001C4BDA77426C12791A77826C12791A77C5
:10A80800026CDAB1B2F5004F04D3A2F5FF427F3AE9
:10A8180002640BE0436C11461868FFF709FEA36C4D
:10A82800216C1868FFF704FE00232364A36C1A79CF
:10A838000C4BDA76626C1279DA7610BD03680F2158
:10A84800996540F20131DA6119614FF47C5159611F
:10A858000323114680F83D30C06C0368BDE8104002
:10A868001B68184700800E4008B50248FFF7BCFF78
:10A8780008BD00BFE839002008B50248FFF7B4FF5B
:10A8880008BD00BF383A002070470020704700001C
:10A898000023064A436013680BB9106070475A6872
:10A8A8000AB11346FBE75860704700BF287B0020B9
:10A8B8000020704700207047704730B5039C012581
:10A8C8001B024560002C9DF8105043F0800318BF10
:10A8D8004FF0004443EA0242002D44EA020414BF48
:10A8E8004FF4004500252C438460C16021F47F614A
:10A8F80021F00F0101F58053036101F50053436115
:10A9080001F5405301F580418361C16130BD00000C
:10A91800436A026A0BB11A6201E004490A600AB18B
:10A9280053627047024A1360704700BF14660020E4
:10A9380010660020436A026A0BB11A6201E00449FA
:10A948000A600AB153627047024A1360704700BF39
:10A958001C66002018660020F8B54FF480314D4B76
:10A9680040244FF480554FF400564FF4404743F2CB
:10A97800420E1A6A900704D59F625962C3F828E00C
:10A98800F7E7900401D45E62F3E7D00401D45D6276
:10A99800EFE7002AEDDA12F4803001D09962E8E797
:10A9A800520601D45C62E4E73B4A3C4CD2F8803062
:10A9B80043F00303C2F880304FF04042384B9A63AB
:10A9C8004FF440425A630522186003F58F130A209A
:10A9D800C3F8B4200822C3F8A422324B5A6842F0C4
:10A9E80080625A604FF08062C3F8842009F002F850
:10A9F800D4F8403143F00203C4F84031D4F8403170
:10AA080013F00205FAD102F0A7FC2B46264A0121D1
:10AA180042F823100133202BFAD14FF48072002121
:10AA2800224808F097FF0023214A13700122C4F836
:10AA380090200322C4F8A8211B4AC4F84831C4F85E
:10AA48005421C4F84C31C4F858311A4B1A4AC4F886
:10AA58004031D4F8843143F48053C4F88431D4F8B5
:10AA68005831D4F85431154BC3F80022144B4FF425
:10AA780080321A60134BC4F84831D4F8483143F097
:10AA88001203C4F84831D4F8483143F44023C4F8D9
:10AA98004831F8BD00800D4000C00F4000022E4034
:10AAA80000A00D4000800042004000205B7C002098
:10AAB800147C0020158B0100ED590000003C00209B
:10AAC8000CE100E004000003C36870B504460D46BD
:10AAD800002B4AD0632948D908F05EFF234BA060B9
:10AAE8001A68234E5AB96561013D1C604FF0404316
:10AAF800A261E261C6F88850C6F88C3070BDD6F8FD
:10AB08008C1021F07F418D4218D272B600204FF090
:10AB18000072491BC6F88C00C6F844211A686561A2
:10AB2800013D1C604FF04043A261E0615161D46176
:10AB3800C6F88850C6F88C3062B670BD6D1A936935
:10AB48007BB15A69954209D2521B5A61DA69A361ED
:10AB5800E2616561DC61E3699C6170BDAD1A1A460A
:10AB6800EDE76561A361E261946170BDC86500208D
:10AB780000022E4070B50A460646036999684906E0
:10AB880001D41B68FAE74021956803F13404916009
:10AB98001168196051685960D168D96011691961E3
:10ABA8005169596191699961D1699E62D961D16A86
:10ABB800D962116B196302F1340103C984E80300F7
:10ABC800D16BD96319460868012801D00968FAE7EA
:10ABD8000A601946106000200C68A24205D00C6873
:10ABE800486208460C622146F6E7002248620A627B
:10ABF80096F8342012F0FD0F05D1094A1068586202
:10AC080040B9084804E0084A1068586210B9074873
:10AC1800036000E00362116001209D6070BD00BF09
:10AC28001066002014660020186600201C660020AC
:10AC38002DE9F04F85B082460D4693460393CB88A5
:10AC4800B3F5804F57D802F03BFB0646002852D098
:10AC580002F036FB044608B9304608E0EB88CBB171
:10AC680002F02EFB30B9304602F032FB204602F0EB
:10AC78002FFB40E095F9007001210023EA888DE858
:10AC88000A00FB0FFF435946FFF717FE3060FF0F1E
:10AC9800046001E0012730604FF000094FF001081F
:10ACA80029463046CDF804900223CDF800900822BA
:10ACB800FFF703FE3B4649462046CDF804804A4646
:10ACC800CDF80080FFF7F9FDDAF80030C4F82CB0B1
:10ACD8003146A362EB8823632B6863636B68C4F80F
:10ACE8000080A363039BDAF80000E36305B0BDE8C6
:10ACF800F04FFFF73FBF002005B0BDE8F08F2DE90A
:10AD0800F74F8146884617469A4602F0D9FA064612
:10AD1800002840D07D1E0446AD0B75B102F0D0FA74
:10AD280038B93046356802F0D3FAA64233D02E46F9
:10AD3800F7E72060013D0446EFE70123C4F82890B7
:10AD4800C4F82C80236027636563A563C4F83CA01E
:10AD58003446B7F5804F99F835304146204693BFC1
:10AD6800BA464FF4804A4FF0000B4FF0010B5246A1
:10AD78008DE82008FFF7A1FDBBF1000F04D1D044F6
:10AD8800CAEB07072468E4E73146484603B0BDE844
:10AD9800F04FFFF7EFBE002003B0BDE8F08F8268E8
:10ADA800110608B507D48268120406D5836ADB6BDE
:10ADB8001BB1984701E0002008BD012008BD000034
:10ADC8002DE9F8432C4B4FF000081C68002C50D09C
:10ADD8002046FFF7E4FF256A002844D020462E4687
:10ADE800FFF796FDA36858063AD5A76A20462C4671
:10ADF800002502F06DFA9EB1B36AD6F820909F4202
:10AE080001D04E46F7E73046FFF782FD0DB12E62BE
:10AE180000E03546C6F82080A64208BF4C46F0E759
:10AE28003B6923F01F033BB19A6851061DD53B616E
:10AE3800C7F80C80C7F81880002DC7D0AB681A0473
:10AE480008D5FA6B32B143F040032846AB60AB6AD1
:10AE5800DB6B98472E6A284602F03AFA3546EBE74C
:10AE6800204602F035FA2C46B0E79A681A681B6843
:10AE7800D7E7BDE8F88300BF146600202DE9F0414C
:10AE8800524CD4F844516E03C4F844510FD5504B7A
:10AE98001E6866B13046FFF782FF376A28B1304630
:10AEA800FFF736FD304602F013FA3E46F1E7280375
:10AEB8000FD5484B1E6866B13046FFF770FF376AFA
:10AEC80028B13046FFF736FD304602F001FA3E461B
:10AED800F1E7A90701D5FFF773FF6A073ED5D4F854
:10AEE80084613A4A46F02A03C4F88431B3071DD571
:10AEF80016F00108384B0ED01978012916D801210F
:10AF080025F080751970354BC2F880304FF04043FA
:10AF1800C2F884300AE083F800800222304B314FB7
:10AF28009A63386800F070FDC7F80080370715D4B9
:10AF3800294A1378022B11D170070FD503211170FC
:10AF480042F21072C4F880204FF04042C4F88420C6
:10AF5800D4F88421910501D5214A5363EA011AD511
:10AF68001D4B1A78012A08D102221A70D4F88431AC
:10AF780043F48073C4F884310DE0032A0BD1042212
:10AF88001A700022D4F884011146C0F3816000F0E1
:10AF9800FFFA144B1860AB0115D5134A116891B12B
:10AFA8008B6913604BB10022DA615B69013BC4F81D
:10AFB80088304FF04043C4F88C30C8680368BDE857
:10AFC800F0419B681847BDE8F08100BF00022E40A1
:10AFD800146600201C660020147C0020A086010056
:10AFE80000A00D40D47A0020C8650020844B002AB8
:10AFF80008BF01225943036B2DE9F04F1B7D85B033
:10B00800090C022B4FF0010360D10F2A01F15701FF
:10B018004FF0FF35DFF8ECC128BF0F224909013A8C
:10B0280003FA02F2B2F5807FA8BF4FF48072D40809
:10B0380018BFA3B20024A0F840302B4627460026AC
:10B0480017F80CE017448E44764538BF7646FF2F34
:10B05800DFF8B0E1F4D9B54288BF234604F1010412
:10B0680088BF3546A242E9D1BB2D01D90020C4E0F2
:10B07800C9B21C46A0F84420A0F8463080F84A100F
:10B08800FF2C06D81EF804500D440EF80450144442
:10B09800F6E7012A01D1FF220EE0022A03D103F0CC
:10B0A8000101552207E0042A99BF03F00301112288
:10B0B80003F0070101228A40DB0880F83620A0F857
:10B0C8004230002380F83730012096E0052443EA17
:10B0D8005305AA4204D9013C4FEA4303F7D1202380
:10B0E8009AB20392BDF80C20A0F8402090F83520C1
:10B0F80022B984314A090221029203E06631022210
:10B10800490902924FF0FF324FF0000C1546E6460F
:10B118000192E0463B4A4FF0000B02EBC80614468A
:10B12800029A96F800A096F802909244F77889441B
:10B1380032790F44CA450A4405D9BA4509D9524556
:10B1480038BF524608E0B94503D94A4538BF4A4690
:10B1580002E0BA4238BF3A46019F0136BA4238BFC8
:10B16800DE460BF1010B3CBF01924546BBF1040FD3
:10B17800D6D19844B8F11F0FCCD90CF1010C9C45DD
:10B18800C7D1019ABB2A3FF671AFBDF80C20AEB209
:10B198009DF808C0C9B2A0F84420A0F84660A0F8FD
:10B1A80048E080F84AC080F84B101F2D18D80EEBE5
:10B1B800C5021D44A75C02F102086744A75414F8AD
:10B1C80008700F4404F8087002F10308043214F8F8
:10B1D80008700F4404F80870A75C0F44A754E4E70C
:10B1E8000123A0F8426003FA0EF280F836201C22F0
:10B1F80002FA0EFE80F837E0184605B0BDE8F08F79
:10B20800AB2A01005B7C0020F0B51C4D40F0020623
:10B21800B0F84040B0F842102F461F292CD855F8F6
:10B2280021204FEA810ED3070AD402F0060C22F03F
:10B238001F03BCF1020F0FD1B3F840C064450BD90E
:10B24800026047F80E6015E0834213D01A68D207EF
:10B2580006D41B6823F01F03B3F840209442F3D9A7
:10B268001A46824206D0126832F01F02F9D11A68D3
:10B2780002601E602144D0E7F0BD00BF00400020FE
:10B288002DE9F84F0A9F05460E4690469A4602F069
:10B2980007F80446002800F08A8002F011F8814679
:10B2A80028B9204602F004F84846BDE8F88F4FF068
:10B2B800400B60220021204608F04CFB5A46002132
:10B2C800484608F047FB0123032EC9F80030C9F8A7
:10B2D80008B0C4F810902563636184F835A084F839
:10B2E800346010D10B9A39462046FFF77FFE82461C
:10B2F800002861D1484601F0EBFF204601F0D8FF55
:10B308005046BDE8F88FB8F1000F08D06B680BB94C
:10B318006C6004E09A6B0AB11346FBE79C6316B1B4
:10B3280000210B4605E02B7D0121012B8CBF00235A
:10B3380001236A7D287D42F0704242EA003242EAE7
:10B34800082242EA074242EAC36343EA813194F899
:10B358003630616043F08043EA7D43EAC253AA7DF8
:10B3680043EA024394F8372043EA0223A36036F005
:10B37800020317D1124B44F00201D3F858216AB9DD
:10B38800626842F4004262602160C3F85841D3F811
:10B39800402142F02002C3F8402108E013682360EE
:10B3A800116004E0032E204604D1FFF72DFF20464C
:10B3B800BDE8F88FBDE8F88FB8F1000FB0D0A5E769
:10B3C80000022E40F8B590F83430044613F0FD0F13
:10B3D80068D00022614850F822309100DE0711D46D
:10B3E80023F01F039C4207D123680B500AE021F089
:10B3F8001F018C4204D00B461968CD0702D4F6E72A
:10B40800216819600132202AE5D1236BB4F8446021
:10B418001B7D94F84A70022BB4F8463007D1504986
:10B42800FF2B25D85A5CD21B5A543344F8E71A46E6
:10B43800B4F848E094F84B5049491F2A18D80EEB45
:10B44800C2033244C85C03F1020CC01BC85411F893
:10B458000C00401B01F80C0003F1030C043311F835
:10B468000C00401B01F80C00C85C401BC854E4E702
:10B478003C4B1D686DB3AB6A2E6A9C4201D03546C1
:10B48800F8E72846FFF756FA236933F01F0203D07E
:10B498009D42F4D01B68F8E79D42F0D0284601F0A1
:10B4A80017FFECE7036823F01F0398421FD12E4BC8
:10B4B800D3F8402122F02002C3F84021D3F84421D8
:10B4C80012F40042FAD1284BC3F85821274B1D68C3
:10B4D8006DBB206930F01F0304D0056801F0F8FE49
:10B4E8002846F7E72046BDE8F84001F0E1BE1A68B3
:10B4F80022F01F02944201D01346F8E76268120452
:10B5080003D55A6842F400425A6022681A60164B02
:10B51800D3F8402142F04002C3F84021D3F8442137
:10B528009706FBD52022104BC3F84421CEE7AB6A1F
:10B538002E6A9C4201D03546CAE72846FFF7E8F94B
:10B54800236933F01F0203D09D42F4D01B68F8E74B
:10B558009D42F0D0284601F0BBFEECE700400020F9
:10B568005B7C00201C66002000022E401466002030
:10B578000023064A8360436013680BB91060704764
:10B588005A680AB11346FBE75860704708660020FE
:10B59800F7B505460F46164601F072FE0446002828
:10B5A80039D02422002108F0D5F925750823002573
:10B5B800E675204665752A46A775294600932B46E9
:10B5C8000195FFF75DFE0646206020B9204601F090
:10B5D8005FFE304620E001F083FE22680F4B2061B9
:10B5E8002046D36301230E4982F835300D4A137083
:10B5F8004FF400230C4A81E80C002B460B4AFFF756
:10B6080017FB0B4A13680BB9146004E09A680AB177
:10B618001346FBE79C60204603B0F0BD01630000C1
:10B62800C0600020FB86002080060001C058002072
:10B63800A47A0020F0B50E695EB3D76A18B1335CFE
:10B648000133DBB200E003461FB37A78032A20D126
:10B65800335400253A7803EB52013129C2BFC3F1B4
:10B6680032025200D2B2A91CCCB2A24206EB0304A9
:10B6780007D9302B0D4604D80133795CDBB2E17071
:10B68800F1E70022E2700130C0B2022801D8335439
:10B69800F9E7F0BD2DE9F04F2E4F85B0064600259D
:10B6A8003C68DFF8B8800397DCB1A268BAB9B8F88B
:10B6B800003020462168093B0093274BD1F80090C1
:10B6C8003146C84750B163680DB16B6001E0039A19
:10B6D80013600023A6606360F46038E02546646860
:10B6E800E2E71E4B1E4DB3F80080A84409354545D6
:10B6F8002DD26B7895F800A0042B26D1BAF1090F4A
:10B7080023D1039B4FF00009C5EB080B1C68E4B17B
:10B71800A368C3B923680122CDF800B031461B687D
:10B7280020461F462B46B84760B16368B9F1000F41
:10B7380002D0C9F8043001E0039A1360F36863602B
:10B74800F460A660A1466468E1E75544CFE705B018
:10B75800BDE8F08F08660020C9580020E67B00206D
:10B76800C0580020084B094A10B5116818780130F4
:10B778000A46802828BF012022B1547DA042F6D075
:10B788009268F9E7187010BDFE860020A47A0020A0
:10B798002DE9F0410746C06B28B1036839465B685C
:10B7A800BDE8F0411847BB6A0B268E4D1C6B237E03
:10B7B8000E2B00F21581DFE813F00F0029003E0080
:10B7C8005900650074008A009300A900B300C900FD
:10B7D800D000DD00F6000B012168824B4A68D87959
:10B7E80022F0FF6323F4E02343EA00434B60FFF7B2
:10B7F800B9FF002300047C491A4640F4A0604B605E
:10B8080008602046FFF714FA0123DEE076494FF47A
:10B81800901520684B886375426822F07F021343B5
:10B82800704A43602046714B81E828000023FFF7E7
:10B83800FFF90223C9E02B7963766B79A376AB799C
:10B84800E3766A7A2B7A43EA0223E383EA7AAB7ACD
:10B8580043EA02232384A97BEB7B2A7C6B700B438E
:10B8680029701343AA7076D0032357E05E496048D5
:10B87800604B614A81E8090000232046FFF7D8F9A8
:10B888000423A2E02B79032B65D96B79032B62D1B2
:10B89800EA79AB7943EA022363842B78E3B1052381
:10B8A8003CE0504A608C12F8043B4F491B0443F0BB
:10B8B800407343F4D0630B6040F0FF63204643F4C9
:10B8C80080234B600023FFF7B3F906237DE03A4657
:10B8D80021460020FFF7AEFE6B78E3B107231DE099
:10B8E800404A608C537804323F491B0443F040734C
:10B8F80043F4D0630B6040F0FF63204643F4802399
:10B908004B600023FFF794F908235EE03A4621468E
:10B918000120FFF78FFEAB78EBB10923237646E7CA
:10B92800304A608C937804322F491B0443F04073EB
:10B9380043F4D0630B6040F0FF63204643F4802358
:10B948004B600023FFF774F90A233EE03A4621468C
:10B958000220FFF76FFE267629E723494FF41023CC
:10B96800264A204681E80C0000231E4AFFF760F9AA
:10B978000C232AE01B4A2046D1789378204A43EAD0
:10B9880001231949B3F5006F88BF4FF40063138092
:10B9980013881A4A1B040A604B600023114AFFF7F8
:10B9A80047F90D2311E00F4B20460F49DA7922772A
:10B9B8001A7A62775B791B0443F410630B600023E7
:10B9C8001A464B60FFF734F90E232376BDE8F08161
:10B9D8002046FFF75FFE0F2300222376094B1A70DB
:10B9E800BDE8F081C0580020C0600020800600013A
:10B9F800800600030000FC07C458002080060002EF
:10BA0800E67B0020FB860020F8B5054600282FD0ED
:10BA1800C4680027174E54B1236820461B6998470D
:10BA280063683268A760626034601C46F3E76C683C
:10BA38002CB1A66B2046FFF7C5FC3446F8E728680A
:10BA4800FFF7C0FC0C4A136893B1AB420DD1AB6849
:10BA58000CB9136000E0A360286908B101F04EFC3E
:10BA68002846BDE8F84001F013BC1C469B68EBE78C
:10BA7800F8BD00BF08660020A47A0020F8B5054686
:10BA880000F1100400F12006002754F8040F20B13B
:10BA98000368A968DB6998472760B442F5D1F8BD07
:10BAA800406910B103681B6A1847704710B5CC0885
:10BAB80011F0070100EB040317BF005D08460841B9
:10BAC800013318BFC1F10801914205D213F8014BA7
:10BAD8008C4008312043F7E707D91F2A9FBF01236D
:10BAE80003FA02F202F1FF32104010BD2DE9F04FC7
:10BAF800012A87B004460F461D46DDF840E001D014
:10BB08000020FAE0BEF1180FFAD91B795A1E012A53
:10BB1800F6D86A79032AF3D1AA79012A02D1EA79F7
:10BB2800012AEDD06A7A082AEAD9A97A2129E7D127
:10BB380095F80EC0BCF1000FE2D00620032111FBDE
:10BB48000C018A42DCD102F10906B645D8D300219E
:10BB580001EB4100284490F80F80B8F1220F0AD178
:10BB680090F811C0017C41EA0C21B1F5487FA4F896
:10BB7800D01304D9C4E701316145E9D3C0E70721EF
:10BB880011FB03618E45BBD3012B22D1A95D072987
:10BB9800B6D12A44917A0529B2D1117B0329AFD1B4
:10BBA80092F80EE0567BD07A46EA0E2692F80FE01D
:10BBB80010F00F02A4D000F0F0008028A0D1384681
:10BBC8008DE84040FFF75CFB0023E0602361A6841A
:10BBD80077E0AB5D072B93D1AB189A7A052A8FD102
:10BBE8001A7B032A8CD1997B5A7B93F80BA042EAE3
:10BBF800012BDA7B1AF00F01049281D01A7C072AF4
:10BC08007FF47EAF5A7C052A7FF47AAF93F81390BD
:10BC1800B9F1030F7FF474AF1A7D9E7C93F81580F9
:10BC28009B7D42EA082816F00F0205933FF468AF9F
:10BC38000AF0F003802B03931ED116F0F00A7FF46C
:10BC48005FAF049B0A46CDF800B0494601933846D9
:10BC58000123FFF715FB059BE06032460193494637
:10BC6800CDF8008053463846FFF70AFBA4F824B005
:10BC78002061A4F8268021E0039B002B7FF440AFCD
:10BC880006F0F006802E7FF43BAF059B4946CDF8C1
:10BC98000080384601930123FFF7F2FA049BE06025
:10BCA800524601934946CDF800B03846039BFFF74A
:10BCB800E7FAA4F824802061A4F826B02369104A82
:10BCC800DA63E36838460F4A0F49DA630023B4F8A9
:10BCD800D0236361A361E3612362AB7884F8A4365F
:10BCE800AB78A16204F1280143EA024304F130026F
:10BCF800E3622346FEF79CFF012007B0BDE8F08F02
:10BD0800FD680000376E00008106002210B5044669
:10BD1800032100F5787001F006FB04F5A060052109
:10BD280001F00EFB04F5C860012101F02BFB204651
:10BD3800BDE81040FFF71CBC70B504460D4611481D
:10BD4800114909F0D2F8D4F87836EA6A60699A425B
:10BD580002BF94F8753623F0010384F87536D4F8D9
:10BD68007C36EA6A9A4202BF94F8753623F00203D9
:10BD780084F8753628B1036829469B68BDE8704089
:10BD8800184770BD883A0020073700200146C06B6D
:10BD980008B1FFF7D1BF70470023064A4360136814
:10BDA8000BB9106070475A680AB11346FBE7586030
:10BDB800704700BFF47A0020F8B50B4B05460E46D5
:10BDC8001C687CB123682946AA6820461F68334648
:10BDD800B84728B1022805D1012385F8803601E04B
:10BDE8006468EEE72046F8BDF47A00202DE9F047B4
:10BDF800002400F13005B0F8D083074626462146D6
:10BE0800A844A1464FF0010A80F8D243454501D322
:10BE180000224FE02B78FE2B02D105F20115F5E741
:10BE280003F00302022A08D0032A0AD0012A0DBF10
:10BE38006A7801350022023506E0B5F8012003359D
:10BE480002E0D5F8012005354545E1D803F0FC03AB
:10BE5800842B14D008D8082B14D0802B28D0042B7E
:10BE6800D4D11FFA82F9D1E7A02B0DD002D8902B9C
:10BE78001ED0CBE7B02B1BD0C02B14D0C6E787F859
:10BE8800D2A3C3E791B2C1E75EB9032C09D841EA4E
:10BE980009413846FFF790FF07EB84030134E4B209
:10BEA8005861013603E00EB93146AFE7013EF6B2FC
:10BEB8000021ABE7032C06D8231D013407EB8303CD
:10BEC800E4B25A60F6E7BDE8F087000070B50446B2
:10BED80040690D4620B96A6B1D4B9A4237D105E07F
:10BEE8000368DB6898470028F5D070BDB4F8D033F4
:10BEF8002A6B9A422BD12046FFF778FF2346A28C63
:10BF080004F55471E068FEF7FAFE2346A28C04F5A6
:10BF18006471E068FEF7F3FEA06840F24C53C28BF0
:10BF28009A4214D1038CB3F51A7F03D040F22F4202
:10BF380093420CD1074B04F12801074AA3624FF43E
:10BF48008023E3622346BDE87040FEF771BE70BDF2
:10BF5800810600222109F403A63B00202DE9F04FB9
:10BF6800B0F8D033002400F13009A3B0A046A346AE
:10BF78004B442746A2460990159116A81192002114
:10BF880030220F9307F0E6FC059404940E9408946D
:10BF98000D94039407940C940F9B994580F0668147
:10BFA80099F80030FE2B04D199F8013003339944F5
:10BFB800F2E703F00302022A0BD0032A0ED0012A6B
:10BFC8000DBF99F8015009F10109002509F102098D
:10BFD80008E0B9F8015009F1030903E0D9F8015064
:10BFE80009F105090F99894500F2408103F0FC0326
:10BFF800742B3DD010D8142B24D004D8042B1ED079
:10C00800082B3ED0C8E7242B27D0282B45D0182B47
:10C01800C2D1ADF8585042E0942B2CD007D8842BCD
:10C028002CD0902B00F01A81802BB5D16BE0B02B6F
:10C0380000F01481C02B50D0A02BADD131E0ABB2B1
:10C048000893A9E7012A01D16BB202E0022A02D1C2
:10C058002BB20493A0E704959EE7012A01D16BB2A5
:10C0680002E0022A02D12BB2059395E7059593E7E2
:10C078001FFA85FB90E71FFA85F88DE7EBB20D9361
:10C088008AE7172F88D81F2D86D922AA7B1C02EB96
:10C098004706DFB226F8305C7EE7ADF85A50FF2736
:10C0A8007AE7039BA3B9089ABDF8583043EA0243DC
:10C0B8000C93079B032B9DBF099A013307994FF0F7
:10C0C800000A9FBFDBB202EB81020793D2F814A0EB
:10C0D800039B0133DBB20393C0E0039B002B00F00A
:10C0E800BD80013B13F0FF03039340F0B780BAF122
:10C0F800000F00F0B380DAF8003050464FF0000A25
:10C108009B699847AAE0099B93F8D2332BB19DF815
:10C1180054300D9A9A4240F0A18015F0010306931D
:10C1280040F08D80BAF1000F00F08980DAF8003015
:10C138005046059A0C9900922A461B691E46049B94
:10C14800B04715F0020503D1089B26461F0474E08A
:10C15800182F06D9BDF85A300126BDF85850069355
:10C1680019E0B8F1010F11D9012F0FD818BF0E9B94
:10C178004FF001060CBFBDF8585003F47F454FF649
:10C18800FF7318BF05F58075069304E0069E4FF609
:10C19800FF7335460693089B01220A941B041293E9
:10C1A8000BF1FF33109302FA03F3139302FA0BF324
:10C1B8005B42149300230B930B9B43453FD226B15C
:10C1C800069B9D420BD26F1C0AE06F1C22AB172FF7
:10C1D80003EB450528BF172735F8305C00E02F46EC
:10C1E800129B5A460A992B4311980E93FFF75EFC4F
:10C1F800049B0246002BDAF8003007DA10991E2952
:10C2080004D8139908421CBF14990A435B69504625
:10C218000E9998470A9B0E953D465B440A930B9BE3
:10C2280001330B93C8E75A4631461198FFF73EFC95
:10C23800049B834206DD5E4401354545F3D308FB84
:10C248000B440BE0059B8342F5DBDAF8003040EA4B
:10C258000701012250465B699847ECE74FF000035D
:10C268000027ADF85830ADF85A3095E623B0BDE850
:10C27800F08F70B504464069CD6A0E6B18B103683B
:10C288005B68984748B994F8D233A3B933462A462D
:10C298004FF480712046FFF761FE04F56473A28CA9
:10C2A800E0689D4223460CBF294604F55471BDE859
:10C2B8007040FEF724BD012EEFD92978731E6A1C41
:10C2C80041F48071E6E70146C06B08B1FFF7D1BFC2
:10C2D800704770B5044600F55876002594F89E33EB
:10C2E8009D4206D256F8040F08B1FFF78DFB0135C1
:10C2F800F4E700251C2204F55970C4F8A453294614
:10C3080084F89E53C4F86053C4F8805384F8A1534A
:10C3180084F8A253C4F8A75307F01CFB84F8AB5366
:10C3280084F8AC5384F8AD5384F8AE5384F8AF5313
:10C3380084F8B05384F8B15384F8B25384F8B353F3
:10C3480070BD0000F8B504460D460AB10020F8BDDE
:10C358004D49C0F838134D49C0F81813A96921F0A0
:10C368007F4121F0FF01B1F5106FEFD1E97E02297D
:10C37800ECD880F8982303F1100206981030811A3F
:10C3880019440F2957D912F8101C092951D112F84C
:10C398000F1C04294DD112F80C1C012949D112F89F
:10C3A8000B1C092945D112F8096C022E41D812F844
:10C3B800071C07293DD112F8061C052939D112F8A6
:10C3C800051C01F0F001802933D112F8041C03295F
:10C3D8002FD112F8031C01292BD112F8021C41BBE2
:10C3E80094F8981312F80DEC12F80E7C31B984F811
:10C3F800997312F80D6C84F89A6309E094F899C35C
:10C40800674518D194F89B73B7420FD284F89AE322
:10C4180012F8096C84F89B6312F8056C06F00F0695
:10C4280084F89C6312F8016C84F89D63013184F8E8
:10C4380098131032A3E794F89833002B86D0002184
:10C448001C2204F55970C4F8A41384F89E13C4F888
:10C458006013C4F8801384F8A11384F8A213C4F8F5
:10C46800A71307F077FA0A4B04F5627204F55671C0
:10C47800C4F858334FF480132846C4F85C33234675
:10C48800FEF7D6FB0120F8BD553700206B3700209A
:10C49800A006002910B5044607210C3000F036FF2D
:10C4A80004F59070022100F03EFF04F5F0700421BD
:10C4B80000F046FF04F53870012100F063FF2046C4
:10C4C800BDE81040FFF754B870B504460E4601B3F6
:10C4D80090F89E3399421CD890F8A123012592B96F
:10C4E8000C4B80F8A153B540C0F858330346C4F844
:10C4F8005C1300F556718068FEF79AFB94F8AB332D
:10C5080023EA050503E08D4090F8AB331D4384F81A
:10C51800AB5370BD2303080070B590F89E330446F2
:10C528000E468B4224D390F8A1330125D3B90029B4
:10C5380080F8A15300F5617205FA06F514BFA3232C
:10C54800A023C0F8583341F4802300F55671C0F891
:10C558005C3303468068FEF76BFB94F8AC3323EA40
:10C56800050503E08D4090F8AC331D4384F8AC53C7
:10C5780070BD00002DE9F04104460E4607F00CFAA4
:10C5880004F546739E4219D194F8B373B7B30125E5
:10C59800A84694F89E339D4209D808FA05F33B4211
:10C5A80003D029462046FFF7B7FF0135F1E73046AB
:10C5B80044F62061BDE8F041FEF786BA04F54E73F3
:10C5C8009E421BD194F8A263C6B1751E254495F806
:10C5D800A433082B12D1A368002794F8A30332468A
:10C5E80084F8A27304EB8604597DFEF7D1FF044B4F
:10C5F800C4F860031F70092385F8A433BDE8F081EF
:10C60800FA86002070B504460E4601B390F89E33B2
:10C6180099421CD890F8A123012592B90C4B80F8B7
:10C62800A153B540C0F858330346C4F85C1300F56D
:10C6380056718068FEF7FCFA94F8AD3323EA0505D5
:10C6480003E08D4090F8AD331D4384F8AD5370BDC1
:10C658002301100070B504460E4601B390F89E33CE
:10C6680099421CD890F8A123012592B90C4B80F867
:10C67800A153B540C0F858330346C4F85C1300F51D
:10C6880056718068FEF7D4FA94F8AE3323EA0505AC
:10C6980003E08D4090F8AE331D4384F8AE5370BD6F
:10C6A8002301110070B504460E4601B390F89E337D
:10C6B80099421CD890F8A123012592B90C4B80F817
:10C6C800A153B540C0F858330346C4F85C1300F5CD
:10C6D80056718068FEF7ACFA94F8AF3323EA050583
:10C6E80003E08D4090F8AF331D4384F8AF5370BD1D
:10C6F8002301120070B504460E4601B390F89E332C
:10C7080099421CD890F8A123012592B90C4B80F8C6
:10C71800A153B540C0F858330346C4F85C1300F57C
:10C7280056718068FEF784FA94F8B03323EA050559
:10C7380003E08D4090F8B0331D4384F8B05370BDCA
:10C748002301130070B504460E4601B390F89E33DA
:10C7580099421CD890F8A123012592B90C4B80F876
:10C76800A153B540C0F858330346C4F85C1300F52C
:10C7780056718068FEF75CFA94F8B13323EA050530
:10C7880003E08D4090F8B1331D4384F8B15370BD78
:10C798002301140070B504460E4601B390F89E3389
:10C7A80099421CD890F8A123012592B90C4B80F826
:10C7B800A153B540C0F858330346C4F85C1300F5DC
:10C7C80056718068FEF734FA94F8B23323EA050507
:10C7D80003E08D4090F8B2331D4384F8B25370BD26
:10C7E8002303040010B540F6013390F89A1390F82B
:10C7F8009923044643EA014300F55671C0F85C23C7
:10C808000022C0F8583303468068FEF711FA012366
:10C8180084F8A13310BD70B505460024012695F8AB
:10C828009E339C420BD806FA04F3D5F880231342B2
:10C8380003D021462846FFF76FFE0134EFE72B4669
:10C8480005F56071D5F860030122BDE87040FEF778
:10C8580056BA0146C06B08B1FFF7DDBF704738B55F
:10C8680090F8B33304460D462BB944F6206100F521
:10C878004670FEF729F9012194F8B333A94019430A
:10C8880084F8B31338BD012303FA01F190F8B333E8
:10C8980023EA010180F8B313704700002DE9F04145
:10C8A800054614460E4600297AD090F89E339942E0
:10C8B80076D84F1E074497F8A423092A70D8DFE8D2
:10C8C80002F00505121212121236515BE40767D501
:10C8D800022387F8A433FFF7C2FF31462846BDE894
:10C8E800F041FFF78FBEE0071DD50132D2B2072A0B
:10C8F80087F8A42354D12B4B197800294DD12A4904
:10C908000978002949D10121284619703146FFF7D5
:10C91800BAFF314687F8A4232846FFF73BFF85F87E
:10C92800A263BDE8F0812846FFF7ADFF33E0A10719
:10C9380018D53146FFF706FF0823A20587F8A43368
:10C9480005D414F4806F0CBF0023022300E00123F8
:10C9580085F8A33305F54E7046F2A811BDE8F041FD
:10C96800FEF7B2B814F001041AD131462846FFF791
:10C9780049FE0C4B1C700EE014F0010410D100EBC2
:10C988008108D8F86003FFF73FF8C8F860433146DC
:10C998002846FFF737FE012300E0062387F8A43373
:10C9A800BDE8F081FA860020FB86002037B50B46EB
:10C9B80000225F4D044680F8A1235A6B098FAA42D2
:10C9C80022D05C4DAA4202D0A32A43D13BE090F882
:10C9D8008A3380F89E3390F88B3380F89F3390F831
:10C9E8008D3380F8A03390F89833012B01D9FFF7E5
:10C9F800F9FE012594F89E339D422BD829462046FE
:10CA0800FFF762FD0135F5E790F89E33994225D18D
:10CA1800D0F8603313BB90F89D33012590F89C2320
:10CA2800032101932B4600958068FEF729FC426894
:10CA3800414A2346C4F8600304F56071C2632A467C
:10CA4800FEF75DF906E01A6B042A07D1DB6A1A685B
:10CA5800FFF724FF94F8A133002B67D194F8AB13A8
:10CA680049B191FAA1F12046B1FA81F103B0BDE8CC
:10CA78003040FFF729BD94F8AD1349B191FAA1F1FF
:10CA88002046B1FA81F103B0BDE83040FFF7BABDE6
:10CA980094F8AE1349B191FAA1F12046B1FA81F1A7
:10CAA80003B0BDE83040FFF7D5BD94F8AF1349B1E6
:10CAB80091FAA1F12046B1FA81F103B0BDE8304006
:10CAC800FFF7F0BD94F8B01349B191FAA1F12046EF
:10CAD800B1FA81F103B0BDE83040FFF70BBE94F81E
:10CAE800B11349B191FAA1F12046B1FA81F103B02D
:10CAF800BDE83040FFF726BE94F8AC1349B191FA6F
:10CB0800A1F12046B1FA81F103B0BDE83040FFF74A
:10CB180003BD94F8B21349B191FAA1F12046B1FAD4
:10CB280081F103B0BDE83040FFF734BE03B030BD3B
:10CB380023030800A0060029C3730000704790F87B
:10CB48008432013BDBB280F8843203B94361704719
:10CB5800A0F10C00FFF7F3BF0123C0F8801280F8A2
:10CB68008532002380F886327047A0F10C00FFF769
:10CB7800F3BFF8B50B0C04460E461B04B3F17F4F08
:10CB88003BD089B2002938D0012390F887E200F21F
:10CB9800862003700023DDB275451CD230F8027F71
:10CBA8000133B942F7D142BBD4F87C3213B1D4F87F
:10CBB8008002984794F88732013BDBB284F88732C9
:10CBC8009D421AD204EB45020135B2F88A12EDB241
:10CBD800A2F88812F4E782B1D4F8783213B1D4F805
:10CBE8008002984794F88732032B9FBF5A1C03F59D
:10CBF800A27384F8872224F81360F8BDA0F10C0012
:10CC0800FFF7B7BF002343627047A0F11800FFF792
:10CC1800F9BF8B78834210D0CB7883420DD00B7943
:10CC280083420AD04B79834207D08B79834204D060
:10CC3800CB791B1A584258417047012070470000B1
:10CC480038B50D460F220749284608F0B0FE0446BD
:10CC580030B92A460449054808F047F9204638BD46
:10CC6800012038BD7A3700208A370020883A002012
:10CC7800A0F11800FFF7E4BF012A73B504460D467A
:10CC880046D1069A182A43D91879002850D05A79DB
:10CC9800032A3DD19A79012A3AD1DA79012A37D182
:10CCA8005A7A092A34D19A7A212A31D19A7C072AC8
:10CCB8002ED1DA7C052A2BD11A7D02F0F0018029C9
:10CCC80026D112F00F0221D0597D032920D1D88A0C
:10CCD800083838281CD81B7E0826284601930123CB
:10CCE8000096FEF7CDFA134AA0652346C26304F105
:10CCF80064013246FEF703F840F2D943EA8B9A42C0
:10CD08004FF0000306D140F6213205E010460FE04F
:10CD180000200DE040F62122E26504F15C01236663
:10CD2800002223462846FDF783FF012084F891025C
:10CD380002B070BD4D7D0000F8B505460E46184896
:10CD48001F461849144608F0D0F86B6A0BB1B34275
:10CD580021D16869F8B9AA6802BB04F45F43B3F546
:10CD6800A06F1AD114F0400018D06FB10F220E49ED
:10CD7800384608F01CFE044630B90C49084808F04B
:10CD8800B4F86C622046F8BD0949054808F0ADF8CA
:10CD98006E620120F8BD0020F8BD1046F8BD00BF46
:10CDA800883A0020CA3700207A370020FB37002055
:10CDB80030380020A0F11800FFF7BEBF90F8853288
:10CDC80010B50446E3B190F88632B3B9D0F87C3296
:10CDD80083B194F887326BB1013BD4F87C22D4F844
:10CDE8008002DBB284F8873203F5A27334F813109B
:10CDF8009047EEE7002384F88732002384F88532D1
:10CE080010BDA0F10C00FFF7D9BF00000B498B4201
:10CE180002D00B498B420ED1836893420BD14169F2
:10CE280009B18A4207D1436190F88432013380F80E
:10CE38008432012070470020704700BF8000010045
:10CE480001000C00A0F10C00FFF7E0BF10B504468C
:10CE58000221803000F067FA042104F5A07000F088
:10CE68006FFA012104F5107000F08CFA2046FEF7E5
:10CE78007FFB04F10C00FEF78FFF04F11800FDF7AB
:10CE880007FD002384F8903210BD0346806868B11E
:10CE980093F8912252B940F621311A66D9650121D9
:10CEA80083F8911203F15C01FDF7C2BE012283F8F9
:10CEB80090227047002310B580F8913240F6213354
:10CEC8004A6B04469A4210D10A6B72B940F6212384
:10CED800026600F15C01C3650123BDE8104080F8DB
:10CEE800913203468068FDF7A3BE94F890322BB1C7
:10CEF8002046FFF7CAFF002384F8903210BD704720
:10CF0800F0B5560619D500242B4D062606FB04F36A
:10CF18005F5BBA420ED190F8782012F0010F264AD2
:10CF2800134401D01A7944E05A88150641D502F015
:10CF38007F0202E00134102CE8D100231F4D35F8A0
:10CF480023609C00B24203D11C4B23449A7830E002
:10CF58000133192BF3D154062AD490F8783011F004
:10CF6800220F4FF0000018BF42F040029B07144BFD
:10CF780048BF82F0400233F81040A24208D111F0B5
:10CF8800110F02D000F01F0213E000F120020AE0A6
:10CF980001306028EFD100230A4931F8130082429A
:10CFA80003D103F1A00292B203E00133602BF4D164
:10CFB80000221046F0BD00BF280F0020C40E00203C
:10CFC800C81200208813002010B5044680F86E109F
:10CFD80080F86F20FFF794FFA36CA4F86C0013B1DE
:10CFE800BDE810401847FFF78AFF10BD0346806868
:10CFF80050B1064A03F15C01DA654FF480321A66D3
:10D0080003F17802FDF714BE704700BF2109000242
:10D0180090F8783010B403F001048C4207D061F323
:10D0280000035DF8044B80F87830FFF7DFBF5DF848
:10D03800044B704790F8783010B4C3F340048C4226
:10D0480007D061F341035DF8044B80F87830FFF7AF
:10D05800CDBF5DF8044B704790F8783010B4C3F337
:10D0680080048C4207D061F382035DF8044B80F89A
:10D078007830FFF7BBBF5DF8044B704710B5532AF3
:10D08800044680F86E1084F86F2009D190F8781063
:10D0980001F00101BDE8104081F00101FFF7B8BFC0
:10D0A800392A09D190F8781081F00201BDE81040C2
:10D0B800C1F34001FFF7BEBF472A09D190F87810A5
:10D0C80081F00401BDE81040C1F38001FFF7C4BF3F
:10D0D800FFF716FFE36CA4F86C0013B1BDE810402D
:10D0E8001847FFF70CFF10BD2DE9F041044600F189
:10D0F800710600F1770700F1640816F8015F032D47
:10D108000ED941462846FFF784FD48B92A4694F8C7
:10D1180070102046FFF7B2FF636D0BB128469847A1
:10D12800B742EAD1636D33B904F1650604F16B07C0
:10D1380004F170081CE00025012606FA05F394F8AE
:10D148007020DBB2134208D094F86420134204D153
:10D1580005F16700636DC0B298470135082DECD121
:10D16800E2E741462846FFF754FD58B3B74204D0DA
:10D1780016F8015F032DF9D9F3E7236D63B921464A
:10D18800A06D082251F8643F23674B686367234604
:10D19800BDE8F041FDF7B3BD0025012606FA05F309
:10D1A80094F87020DBB2134208D194F8642013423B
:10D1B80004D005F16700236DC0B298470135082DEA
:10D1C800ECD1DCE72A4694F864102046FFF7FCFE11
:10D1D800236D002BCAD028469847C7E70146C06B85
:10D1E80008B1FFF781BF70472DE9F8430D460446A3
:10D1F8001F4990461F4807F078FE2B78012B29D14C
:10D2080004F17107022604F16409B0450ADD17F834
:10D21800012F032A04D949461046FFF7FAFCE0B16A
:10D228000136F2E76E1C05F1070804F1700937466C
:10D2380017F8012F032A04D949461046FFF7E9FCDD
:10D2480088B1B845F4D133680120236773686367F0
:10D25800BDE8F8830020BDE8F88394F870102046F4
:10D26800FFF70CFFDCE769782046FFF7ADFEE8E73B
:10D278005A380020883A0020A0F11800FFF7B4BF00
:10D28800024B186808B102681A60704700660020EF
:10D29800024B1A6818600260704700BF00660020E1
:10D2A800024B186808B102681A607047F4650020DC
:10D2B800024B1A6818600260704700BFF4650020CE
:10D2C800024B186808B102681A6070470C660020A3
:10D2D800024B1A6818600260704700BF0C66002095
:10D2E800054B186830B102681A6000230370437058
:10D2F8008370C370704700BF04660020024B1A6831
:10D3080018600260704700BF04660020242310B52F
:10D3180003FB010104468C4204D220462434FFF763
:10D32800B7FFF8E710BD602310B503FB0101044601
:10D338008C4204D220466034FFF7BAFFF8E710BDEC
:10D3480010B500EB811104468C4204D220464034CB
:10D35800FFF7BEFFF8E710BD08B501210648FFF743
:10D36800D5FF01210548FFF7DEFF04210448BDE889
:10D378000840FFF7E5BF00BFD0650020A0410020AE
:10D3880020420020352310B503FB010104468C42DE
:10D3980004D220463534FFF7B1FFF8E710BD00236B
:10D3A800C3600361704770B5B0F84250044690F806
:10D3B8005230AD0803F0FF0243B1EBB2816B92002B
:10D3C80080F8523003460069FDF799FC94F8533011
:10D3D80003F0FF0253B1EDB22346E16B920084F8EB
:10D3E80053502069BDE87040FDF789BC70BD00004E
:10D3F800012AF7B504460D4640F0C6801A78092A76
:10D4080040F0C2805A78042A40F0BE805979012938
:10D4180002D19A79032A04D00239102940F2B48043
:10D428000021089800221844093384F8542084F80D
:10D438005520984251D91F78032F40F2A580DE1954
:10D44800B042C0F0A1805A78042A46D00B2A44D0B2
:10D45800242A0DD19A78511E032902D80121334676
:10D46800E7E7F12A40F09080DB78022BF6D08BE0DA
:10D47800052A2FD1062F40F28780DA78023A012A4E
:10D4880000F282809A7812F0F00713D0802F7BD1B7
:10D4980094F85470002FE2D102F00F0284F854205F
:10D4A800DA7884F856205A791B7943EA0223A4F8DB
:10D4B8004030D4E794F85570002FD0D184F8552027
:10D4C800DA7884F857205A791B7943EA0223A4F8BA
:10D4D8004230C4E7252AC2D056E0002954D094F837
:10D4E8005420E2B1B4F84030B4F84A10994216D347
:10D4F8000020009394F85610012301902846FDF768
:10D50800BFFEE06068B1234A2346616BC263B4F88A
:10D518004020FDF7F4FB012384F8483001E00023A4
:10D52800E36094F85520BAB1B4F84230B4F84A1020
:10D53800994211D3002694F8571028468DE84800E0
:10D548003346FDF79DFE206140B1134BC36384F859
:10D55800526084F8536001E0002323610023A4F89B
:10D568004E30A4F8503084F8593084F85A3084F892
:10D578005B3084F85C30A4F88031E36833B9206903
:10D58800003018BF012002E0002000E0012003B0B5
:10D59800F0BD00BF098200003382000010B50446C8
:10D5A800032100F5F070FFF7BEFE04F54070072177
:10D5B800FFF7C6FE04F598600121FFF7E3FE00239C
:10D5C8002046C4F88431C4F88831C4F88C31C4F8D2
:10D5D8009031C4F89431C4F89831C4F89C31C4F837
:10D5E800A031C4F8A431C4F8A831C4F8AC31C4F8E7
:10D5F800B031C4F8B431C4F8B831C4F8BC31C4F897
:10D60800C031C4F8C431C4F8C831C4F8CC31C4F846
:10D61800D031A4F84E30A4F85030E3602361BDE85F
:10D628001040FDF7A5BF8A680B6BC2F30E42991A2A
:10D63800B0F84E30B0F85020890870B50446002084
:10D6480088420ED0656B55F8205045B1B4F84C604F
:10D658000133B34228BF0023666C46F823500130DB
:10D66800EEE79342A4F85020A4F84E3024BFB4F853
:10D678004C105218013AD31AB4F84020B3EB920F69
:10D6880006D32346616BE068FDF739FB012300E010
:10D69800002384F8483070BD0146C06B08B1FFF71D
:10D6A800C2BF7047CB6A826B934203D1002380F8D4
:10D6B80052307047C26B934202D1002380F8533036
:10D6C80070470146C06B08B1FFF7ECBF704790F890
:10D6D8004030013BDBB280F8403003B983607047CB
:10D6E800012380F8423070470B0C89B2092B10B522
:10D6F8000FD10139072924D8012390F8434003FAB0
:10D7080001F112B924EA010100E0214380F8431035
:10D7180010BD012B0FD13039082912D8DFE801F0EC
:10D7280005071011111111110900426410BD82641E
:10D7380010BDC26410BD0C2B03D1B1F50E7F00D112
:10D74800026510BD90F842302BB1012380F84130BA
:10D75800002380F842307047002383617047A0F1AE
:10D768000C00FFF7F9BF000070B504460E460E48DE
:10D7780015460E4907F0B9FBA3690BB1B34210D1A6
:10D78800A06870B905F45F43B3F5A06F0AD115F02E
:10D79800800007D00649044807F0A7FBA6610120CE
:10D7A80070BD002070BD00BF883A00208A38002074
:10D7B800C2380020A0F10C00FFF7D6BFC2B10B7829
:10D7C800022B17D14B78042A80F8433091F90230A4
:10D7D800436491F90330836407D991F90430052A29
:10D7E800C3641CBF91F905300365012280F841200C
:10D7F8001046704700207047A0F10C00FFF7DEBF0D
:10D80800A3F10113012B0BD883680BB19A4207D1FE
:10D8180090F840308260013380F840300120704732
:10D828000020704710B50446FEF7B6FA04F10C0064
:10D83800BDE81040FDF72CB82DE9F843089D0746D0
:10D84800164603EB01090C464C450ED03B683246A0
:10D8580021463846DB6804F10108984730B1204674
:10D86800099A31464446A847EEE70120BDE8F88307
:10D878002DE9F04105461F4602EB01080C464445D8
:10D888000DD02B68204606991E6AB84721460246E5
:10D8980028460134B0470028F1D1BDE8F0810120C5
:10D8A800BDE8F0814FF0FF307047704737B5054647
:10D8B8000C4606F01BF91C4B984202D800232B801B
:10D8C8002EE0694607F062FB9DF806309DF80510CA
:10D8D800503B9DF804209BB27F2B0BD80131C9B275
:10D8E8000C2907D81F2A05D842EA411242EA4323E5
:10D8F8009BB200E000239DF802102B8017299DF8A9
:10D9080001209DF800300AD83B2A08D83B2B06D8BE
:10D91800520142EAC12242EA53039BB200E00023CB
:10D92800238003B030BD00BFFFA5CE120A46D0F851
:10D93800841400B58FB051B1002368468DF80030CB
:10D948008DF801308DF8023002F0BAFB0DE0D0F806
:10D95800880450B18DF831100B468DF832108DF8CF
:10D9680033100146684600F013FE0FB05DF804FB63
:10D978000A46D0F8841400B58FB071B10023684608
:10D988008DF800308DF801308DF8023002F098FBE8
:10D99800A8B1684602F0D1FA11E0D0F8880470B155
:10D9A8008DF831100B468DF832108DF83310014682
:10D9B800684600F0EDFD10B1684600F0BDFE0FB0FE
:10D9C8005DF804FB0A46D0F8841400B58FB079B12D
:10D9D800002368468DF800308DF801308DF802304C
:10D9E800012302F06DFBA8B1684603F0DFF911E0EE
:10D9F800D0F8880470B18DF8311001238DF83210F9
:10DA08008DF833100146684600F0C2FD10B1684633
:10DA180000F04FFE0FB05DF804FB10B5D0F8844459
:10DA28008EB00A466CB1002304F5896168468DF80A
:10DA380000308DF801308DF80230012302F002FC2D
:10DA480010E0D0F8881461B1012301F589616846B6
:10DA58008DF831408DF832408DF8334000F0B8FF32
:10DA680000E008460EB010BDD0F8843430B5154635
:10DA78008FB0ABB1002203F5896468468DF80020A9
:10DA880013468DF801208DF802200A46214602F03F
:10DA9800C3FAD8B12A462146684602F028FC15E0A8
:10DAA800D0F8880490B100F589640A4668468DF874
:10DAB800313021468DF832308DF8333000F00AFDD0
:10DAC80020B12A462146684600F0E2FF0FB030BD7B
:10DAD800D0F8803433B198794FF4007303FA00F02A
:10DAE80080B27047D0F8840408B1D0F83C0470477D
:10DAF80003460430D3F8842410B512B1D469013C2C
:10DB080004E0D3F888440CB1D4F83044FFF7E0FFC0
:10DB1800A4FB000110BD38B50346051DD0F88404E8
:10DB280020B1C469013C03F0D9FD08E0D3F88804AA
:10DB380020B1D0F8304401F0BAFE00E00446241ABF
:10DB48002846FFF7C5FFA4FB000138BD38B500F52E
:10DB58009265FF23044680F8C41480F8B834284638
:10DB680005F0B8F8C4F88C54284604F08FFC30B996
:10DB7800D4F88C142046BDE8384003F019BF0020C3
:10DB880038BD70B588B0064601A805AD06F29C44BC
:10DB980080E80E0007C885E80B00204695E80E00CF
:10DBA80004F01EF9C6F88C442CB196F8B304B0FA08
:10DBB80080F0400900E0204608B070BD7FB50C46F3
:10DBC80005461E4805F000FCFE2C85F8CD440ED114
:10DBD8004FF00001281DFFF7B9FF044685F8CC0473
:10DBE80040BB2E20032105F04DFF204623E0362CB4
:10DBF8004FF000001FD8124B2E1D8DF80500029320
:10DC0800C5F8C03404AB03908DF8044085F8BD0412
:10DC1800C5F8C404304685F8BC4413E90E00FFF784
:10DC2800B0FF20B1D5F89014304603F0C1FE85F856
:10DC3800CC0400E0012004B070BD00BF1D840000CA
:10DC480040787D0130B590F8B83485B00446FF2B94
:10DC580004D190F8C414FFF779FF19E0D0F8BC1488
:10DC6800D0F8C0248DF8043004AB90F8B954029170
:10DC78008DF80550039213E90E00FFF782FF38B1C3
:10DC8800D4F88C14204605B0BDE8304003F090BEAF
:10DC980005B030BD2DE9F041D0F890448CB006466F
:10DCA8001F460CB9002024E0236820469B6998474A
:10DCB800B0F5405F8046F5D94FF4007007F002FDDB
:10DCC80005460028EED0B8F1806F02463B46214653
:10DCD80001A802D901F0AEF901E003F0DBFA04462D
:10DCE800284607F0F7FC002CDCD0301DFFF7AAFF10
:10DCF80001200CB0BDE8F0817FB5D0F890640546EE
:10DD08000EB9002027E090F8CC2490F8CD34BAB1B1
:10DD1800FE2B05D03368694630469B6B98471AE05E
:10DD2800336830465B6C9847421CF3D090B995F83D
:10DD3800CD34FE2BE5D103212E2005F0A3FEE0E72C
:10DD4800FE2B03D1064B9B689B03DAD5281DFFF7F2
:10DD580079FF00E0012085F8CC0404B070BD00BF55
:10DD6800008000421548164A164BC0F89424164AFB
:10DD780003600023C0F8A024144AC0F88434C0F813
:10DD8800A8240722C0F88834C0F8AC24012280F8FF
:10DD98009C3480F8B524292280F89D3480F8BA3460
:10DDA80080F8C83480F8CC34FF2380F8B7240849B9
:10DDB800084A80F8CD3407F03ABC00BFEC60002078
:10DDC8008008002050080020E008002000093D00DD
:10DDD8001B840000DC390020F0B500F1240385B075
:10DDE80005460F4601AC164693E8070084E807008D
:10DDF8007A012146286A01F0ECFC012805D1324657
:10DE08002146286A01F096FC00E0002005B0F0BD2C
:10DE180010B5044600F02AFD002384F8313084F858
:10DE2800333010BD38B50D46144600F124010022E8
:10DE3800006A01F07FFC20B143892B80038901200F
:10DE4800238038BD38B50D46144600F12401002260
:10DE5800006A01F06FFC20B1C3892B8083890120FF
:10DE6800238038BD38B50D4690F83110044651B9B5
:10DE7800382205F06FFD40230120256284F83130F7
:10DE880084F8330038BD002038BD0000F0B40C78A9
:10DE98004D1C202C01D12946F9E71A4F11609160D9
:10DEA8000D460E4615F8014BDCB12F2C13D01F2C54
:10DEB80024D9A4F12201C9B21D2903D827FA01F1F6
:10DEC800C9071BD404F0BF013C2917D05C2C0DD125
:10DED80014E02F2C05D10E4611F8014B202CF8D157
:10DEE800F9E71E601146F0BC01F04EBB2E2C01D1A3
:10DEF8002946D5E7202CFBD09560F9E70020F0BC37
:10DF0800704700BF010100312DE9F84F90F8333018
:10DF180004460E461546DF0777D5580603D494F80D
:10DF2800313019070CD5D4E90001D4E9042310EBEA
:10DF3800050841F100094B4508BF424500D2151AB2
:10DF4800A94604F1180AB9F1000F43D0206AD4E9B0
:10DF58000023D0F8381401EA0208C8F3080BB8F116
:10DF6800000F1ED1134307D194F831305A064CBF25
:10DF7800D0F83434E36905E094F833305B0603D510
:10DF8800A3690133A3610CE05246A16901F0EDFBDE
:10DF980000283ADB05D194F8313013F0500F19D12D
:10DFA80033E0276A4FEA5822A16997F845E4023915
:10DFB800D7F82C0401FA0EF1014401EB0208BBF179
:10DFC800000F4FD1B9F5007F4CD3D7F81C12884504
:10DFD80004D147E0C9EB0500BDE8F88FB9F5806FBB
:10DFE8002AD301234FEA592B03FA0EF39A1A9345C1
:10DFF80028BF9346884512D80BEB080399420ED2E6
:10E0080007F5047005F08BF948B994F832304FF0F1
:10E01800FF3043F0020384F83230BDE8F88FD7F8B8
:10E0280014023246414603681F695B46B847002818
:10E03800EBD04FEA4B270AE0D7F8140232464146A4
:10E048000368DB6898470028DFD04FF400773E4428
:10E05800C7EB0909D4E90023D21943F10003C4E945
:10E06800002370E70022414607F5047005F07DF9AA
:10E078000028CAD0CBF5007700EB0B0130464F459E
:10E0880028BF4F463A4605F0CBFBE0E7F7B501223B
:10E098000DF1070104468569D0E90067FFF734FFF1
:10E0A8000128A5610CBF9DF807004FF0FF30C4E9B7
:10E0B800006703B0F0BD2DE9F74F1F4690F831B067
:10E0C8008369044616460193BBF1000F52D0D0E98C
:10E0D8000089B94508BF904550D056EA070302D1D8
:10E0E8000023836143E01BF0080F05D0D0E9040149
:10E0F800B94208BF90423DD3236A16F1FF3093F826
:10E1080045A447F1FF3100930AF1090A5FFA8AFA38
:10E11800524607F091FA94F833200546530603D582
:10E12800E3691D44A56122E018F1FF30524649F128
:10E13800FF3107F081FA854202D358EA09030AD170
:10E148001BF0400F16BF009BE369D3F83434A3617A
:10E1580004F1180809E02D1AFAE74246A169206A75
:10E16800013D01F002FB002804DD002DF5D1C4E9D2
:10E17800006703E0019B0020A36100E0012003B0D9
:10E18800BDE8F08F2DE9F04F9A4690F831308DB008
:10E1980004460E46154673BB91F8313013F0500F04
:10E1A80029D00AF00303012B00F08281022B40F0F2
:10E1B8007A8103230AF0080949EA03090DB32B6998
:10E1C8004FF00F08002230460E33B3FBF8F808F181
:10E1D800020800235FFA88F8FFF76DFF4FF0000B85
:10E1E8005F46202204A93046FFF78EFE002800F083
:10E1F800BC80202808D0002084F8310084F833003F
:10E2080062E14FF00308E9E79DF81020110611D4E8
:10E2180027B93368203B0193B369009347453CBF56
:10E228000137FFB212B14FF0000BDAE7002D40F0D2
:10E238009C80E0E7BBF1000F27D1474538BF002796
:10E24800852ACED13822594620464FF0010B05F0D9
:10E2580081FB9DF811309DF8142084F8303002F0CD
:10E268003703D20658BF43F0080384F83130336AC5
:10E278002362B36963623368203BA36296F8333044
:10E28800C3F3801384F82C30ABE7C02A2BD19DF858
:10E29800113084F83390980744BF49F0400384F85C
:10E2A8003330DDE90623C4E90423099BE361DDE992
:10E2B8000A23C4E902231DB91AF4006F9BD126E092
:10E2C8002B682A696B604FF00003AB819DF813300F
:10E2D8009A42A8D1BDF81420AB8AD11AD1F1000B0B
:10E2E8004BEB010B7DE7C12A9DD12A4604A92046A4
:10E2F80001F0CCF808B9834673E7AA89002A7FF4AD
:10E3080070AF6968AA6891427FF46BAFD4E71AF4DA
:10E31800884F03D194F833309A0705D594F83130F3
:10E3280013F0110F7FF467AF1AF4806F10D094F8D0
:10E3380033309B077FF55FAF002200232046FFF7AD
:10E34800BAFE00283FF457AF204600F07FFC08E0F3
:10E358001AF4804F00F0AE802046D4E90423FFF77A
:10E36800AAFE00283FF447AFA4E01AF4007F3FF468
:10E3780042AF19F0020F3FF43EAF002D3FF43BAF20
:10E3880047451CD2202204A93046FFF7BDFD50B9ED
:10E398003046D6F818A000F088FA00283FF42BAFD2
:10E3A800C6F818A0ECE720287FF425AF27B9336812
:10E3B800203B0193B36900930137FFB2E0E73822AD
:10E3C8000021204696F8337005F0C4FA336AC7F383
:10E3D800801708F1FF3A2362082384F82C705FFA4B
:10E3E8008AFA84F831300027009B6362019BA3629C
:10E3F8002B68AF816B605FFA87FBC3454FD2012260
:10E4080059462046FFF7E8FC064600283FF4F3AEDD
:10E4180090F90020002AFFF6EEAE2022002105F038
:10E4280099FABBF1000F1ED185233370284B84F86D
:10E4380030A086F801A01B687BB10DF10B020DF12D
:10E448000E0103A89847BDF80C307381BDF80E3053
:10E4580033819DF80B3033751FE045F221437381FA
:10E46800F381738219E0BBF1010F0CD169F07F03CE
:10E47800C02286F801B0327084F833302B69F3700B
:10E48800AB8AB38009E0C12306F11E0B3370AA8959
:10E4980092B96968AA6891420ED10137ABE7204664
:10E4A80000F0E4F910E0002B7FF4A5AE012381E62B
:10E4B80002237FE6012007E0284605F067F826F8E2
:10E4C800020F5E45E3D1E8E70DB0BDE8F08F00BF6D
:10E4D800E87A0020F0B51F4697B0002305460C46A1
:10E4E80001928DF851308DF852308DF85330ADF8D7
:10E4F800143090F831300BB1002047E091F83130FA
:10E5080013F0500FF8D013782F2B12D1019B1A78E3
:10E518002F2A02D101330193F8E7216A1AB9284654
:10E52800FFF7A0FC32E008A8FFF79CFC0028E3D026
:10E5380008AC01AB02AA01992846FFF7A7FC0028FE
:10E54800DAD0019B1B78DBB1002302AA21462846BA
:10E55800FFF718FE0028CFD008AA2B4605F1300E89
:10E5680014461868083353F8041C1646734503C646
:10E578003246F6D1186830602846FFF749FCD8E7DC
:10E588003B4602AA21462846FFF7FCFD17B0F0BD1E
:10E5980019B101F58961FFF79DBF0846704730B48E
:10E5A800134690F8312072B991F8315015F0500F98
:10E5B80009D0D1E90045002504F01F042C4302D1FD
:10E5C80030BCFFF7DFBD002030BC704710B500231A
:10E5D8000478CA03012B42EA5101C25C12FA81F1A4
:10E5E80089B204D1852C14BF0122032200E0012244
:10E5F80013441F2BEDD9084610BD10B5044604F08E
:10E608008EFE58B104F5047004F089FE30B1D4F8D8
:10E6180040040368BDE81040DB691847002010BDBE
:10E62800F8B50446006AA16901B10131012200F080
:10E63800DCFF0128054601D8002638E00123014601
:10E64800206A1A4601F024F806460028F4D0A26988
:10E6580094F8333022B943F0400384F8333025E08E
:10E66800590613D50132954220D023F04003E169C1
:10E6780084F83330A369994208D24F1C206A3A467D
:10E6880001F0C9F80028D7D03946F3E74FF0FF3238
:10E698002946206A01F0BFF80028CDD0A16929B128
:10E6A8002A46206A01F0B7F80028C5D0A56130468F
:10E6B800F8BD70B590F8333004469A0701D40020AD
:10E6C80070BDC5690DB9002528E05B0614D5066A3A
:10E6D800D0E9020196F8452410F1FF3002F1090251
:10E6E80041F1FF31D2B206F0A7FF0023421C2946B0
:10E6F800304600F0CDFF03E02946006A01F0A8F893
:10E708000028E0D1DBE701222046FFF765FB013551
:10E718000028D4D0037803F07F030370E9B294F89B
:10E7280030308B42EFD20023206A84F8313084F8ED
:10E738003330FFF762FF70BD10B590F8313088B004
:10E748000446D90601D400201DE000220023FFF76B
:10E75800B2FC202269462046FFF7D6FB38B12028B4
:10E76800F1D19DF800301A06EDD4002BF1D1082321
:10E77800204684F8313094F8333043F0020384F8AB
:10E788003330FFF796FF08B010BD00002DE9F341C4
:10E7980000260546DFF8D0803746F1B295F83030CC
:10E7A8008B424AD300222846FFF716FB044600286E
:10E7B8004FD00378C02B1DD0C12B37D0852B48D123
:10E7C80095F8313003F037038380D8F8003033B33D
:10E7D8000DF103020DF1060101A898479DF80330D9
:10E7E800BDF806206375BDF80430A281E38122825A
:10E7F800638214E095F8333013F0400F437814BF68
:10E8080043F0020323F002034370D5E90423C0E96F
:10E818000223EB694361D5E90223C0E906232A6A8A
:10E8280092F8103243F0010382F81032394620463C
:10E83800FFF7CCFE01360746AFE7012205F12401B8
:10E84800286A00F077FF20B14780286AFFF7D5FED5
:10E8580030B995F83230002043F0010385F83230A2
:10E8680002B0BDE8F08100BFE87A002010B590F84A
:10E87800313004460BB9012010BD90F833301A0628
:10E8880007D503F07F0380F83330BDE81040FFF769
:10E898007DBF006AFFF7B1FE0028ECD194F8323052
:10E8A80043F0010384F8323010BD2DE9F04190F8AF
:10E8B80031300446580603D5206A01F091F800E08B
:10E8C800A068236AD3F83C341844B0F1806F58D25A
:10E8D8002046FFF7A5FE002853D0256A95F8103288
:10E8E800D90705D505F5047004F019FD002848D0AE
:10E8F8004FF0FF33002605F508754FF4007245F810
:10E90800043C314605F8106C284605F023F8226AC5
:10E91800A3694FF0010892F84514023BD2F82C7411
:10E928008B401F44236A93F8452408FA02F2B24246
:10E9380009D9D3F840042A46B91903681B6A9847CD
:10E94800F8B10136EEE794F83120520614D494F861
:10E95800332062F07F02D4E9020184F83320D3F82F
:10E968003C24002380185941C4E90201D4E9040178
:10E9780012184B41C4E904232046BDE8F041FFF7D3
:10E9880075BF0020BDE8F08110B591F8313004461C
:10E9980013F0500F1AD040F60223FFF7F3FBA8B18B
:10E9A8001023204684F83130FFF77FFF70B1A36948
:10E9B80020460022E3610023FFF77DFBC1232046A8
:10E9C80084F83330BDE81040FFF750BF002010BD79
:10E9D800F0B51F4697B0002305460C460192ADF8E6
:10E9E80014308DF851308DF852308DF8533090F83E
:10E9F8003130002B49D191F8313013F0500F44D009
:10EA080013782F2B0DD1019B1A782F2A02D10133AD
:10EA18000193F8E7216A08A8FFF724FA002834D000
:10EA280008AC01AB02AA01992846FFF72FFA60B398
:10EA3800019B1B781BB3002302AA21462846FFF737
:10EA4800A1FB98B108AA2B4605F1300E14461868A8
:10EA5800083353F8041C1646734503C63246F6D1EC
:10EA6800186830602846FFF7D3F9DAE76FB102AAD1
:10EA780021462846FFF788FF0028E3D105E002AACF
:10EA880021462846FFF780FF00E0002017B0F0BDC0
:10EA9800F0B500239DB004468DF831308DF8323042
:10EAA8008DF833308DF869308DF86A308DF86B3019
:10EAB80090F8313013F0180F01D100203AE0006AC5
:10EAC8000B6A9842F9D140F601236846FFF702FD28
:10EAD8000028F2D00EAA234604F13007164618681B
:10EAE800083353F8041C1546BB4203C52A46F6D121
:10EAF800186809AA04F12403286007CA83E80700F4
:10EB08009DF83030204684F8303094F8333063F084
:10EB18007F0384F83330FFF7A9FE0028CDD0002307
:10EB28003046159302238DF86B3008238DF8693031
:10EB3800FFF7BFFD1DB0F0BD2DE9F84F1C4690F85A
:10EB48003130064688461B079DF828B09DF82CA052
:10EB58009DF830509DF8349039D5A2F2BC7297B226
:10EB68007F2F34D8631E0B2B31D80BF1FF331E2BAC
:10EB78002DD8BAF1170F2AD83B2D28D8B9F13B0F59
:10EB880025D8FFF773FE10B34FEA690319F0010F98
:10EB98004BEA441443EA451508BF4FF0000944EA1C
:10EBA80047244FF0000745EACA2518BF4FF064090B
:10EBB800A4B2BB46ADB208F0010AF9B296F83030FB
:10EBC8008B4234D300223046FFF706F910B90020F3
:10EBD800BDE8F88F0378852B04D0F8D3C03B012B10
:10EBE8001FD9F4E796F83130326A03F0370383808F
:10EBF80092F8103243F0010382F81032BAF1000F94
:10EC080001D00582448218F0020F1EBF80F81490CC
:10EC18000581448118F0040F1EBF80F81590858186
:10EC2800C48159460137FFF7D1FC8346C5E7012265
:10EC380006F12401306A00F07DFD0028C7D0A0F855
:10EC480002B0306AFFF7D9FCBDE8F88F73B590F8C9
:10EC5800333004469A0701D4002054E0C569002DDA
:10EC680040D003F04003866903F0FF01F3B1236A43
:10EC7800D0E9020193F8452410F1FF3002F10902AE
:10EC880041F1FF31D2B206F0D7FC421C2EB1013D52
:10EC9800731CAD1B01932A4401E00195E6611AB388
:10ECA80000230199206A00F0F3FC19E08EB102AA52
:10ECB800006A42F8041D314600F057FD0028CBDBFE
:10ECC80009D04FF0FF32A169206A00F0A4FD10B905
:10ECD800C2E70195C661019931B1206A00F0B8FD1B
:10ECE80010B9B9E701200EE0D4E900232046C4E9B1
:10ECF8000223C4E9042394F8333063F07F0384F8D3
:10ED08003330FFF7B3FD02B070BD00002DE9F74FB7
:10ED180090F83330894604469246990740F1BB8003
:10ED28001A0706D404F11803D0464FF0010B0093DC
:10ED380062E0D0E90423FFF7BEF90028F2D1AAE087
:10ED4800206A2668D0F838341E40C6F30805002E1D
:10ED580056D0D4F820E0760AA1699EF845240239F5
:10ED6800DEF82C34914019443144002D7CD1B8F59B
:10ED7800007F80F09A80D4E90423D4E900679F4299
:10ED880008BF964234BF012205220EF5047004F034
:10ED9800ECFA00287FD0C5F5007628444946464558
:10EDA80028BF46463544324604F03AFDB5F5007FA3
:10EDB80006D1206A00F5047004F0B1FA00286AD080
:10EDC800B144C6EB0808D4E90001821941F10003F7
:10EDD80010461946C4E90023D4E904238B4208BF2E
:10EDE800824209D294F83330024663F07F0384F8F4
:10EDF80033300B46C4E90423B8F1000FA0D135E045
:10EE0800A76937B394F833305B061AD590F84524D0
:10EE1800E36909320193D2B2D4E9020110F1FF305B
:10EE280041F1FF3106F008FC019B1844874205D3E5
:10EE38002046FFF7F5FB00288BD12CE00137A761AE
:10EE480087E7009A394600F090FC002823DB80D140
:10EE5800EEE7E36933B92046FFF7E2FBD8B1A369CF
:10EE6800E36176E7A36174E701228EE7D4E9000144
:10EE7800D4E902238B4208BF824202D2C4E90201CC
:10EE880002E0254B1B6873B194F8333063F07F03BD
:10EE980084F8333007E094F83230002043F001035F
:10EEA80084F8323035E0504633E0B8F5806FDEF84C
:10EEB8001C72DEF8140214D30BFA02F34FEA582C32
:10EEC8009E1B6346B44528BF3346B9424FEA4326E2
:10EED80002D8CA18974215D30268556A4A46A84705
:10EEE8006CE7B9424A4602BF4FF0FF338EF8105222
:10EEF800CEF81C3203681B6A98470028CBD04FF421
:10EF080000765DE74FF0FF328EF81052CEF81C22E3
:10EF1800E2E703B0BDE8F08FE87A00208368014695
:10EF2800C3F3080363B100200A69D0540133B3F571
:10EF3800007FF9D1C8680A69036809681B6A18471D
:10EF480001207047826803460069C2F3080210B4C2
:10EF58008154586801EB70015960996801319960D2
:10EF680040F2FF118A420AD1D86819680268146A07
:10EF78004A1C1A601A6923465DF8044B1847012099
:10EF88005DF8044B704738B50C46C9B20546FFF723
:10EF9800D9FF28B1210A2846BDE83840FFF7D2BF7B
:10EFA80038BDF8B500240746846080E81200A0B296
:10EFB80004F0E4FBA04206460AD001463846FFF7B3
:10EFC800E2FFA0B3651CB5F5803F0BD22C46EEE7F7
:10EFD800651CB5F5803F0AD2A8B204F0CFFB854284
:10EFE80005D122E03846BDE8F840FFF797BF2C1B53
:10EFF800B4F5007F0CD34FF6FF713846FFF7C3FF17
:10F00800A8B1A1B23846FFF7BEFF0028DBD10EE059
:10F018003446A54201D82546D5E7A1B23846FFF7C0
:10F02800B2FF01340028F4D101E00135D1E7002016
:10F03800F8BD00002DE9F04F1F46034687B00D4686
:10F04800D96014461A610B68019008469B69984775
:10F05800B0F5801F814607D2002F00F01381924936
:10F068003846F6F7FEFF09E10026012301365B006A
:10F07800F6B2202E05D09945F8D81C2E01D80823C1
:10F0880003E0A6F10B08C8F347031A2E0293029A6D
:10F098004FF0000186BF013601234FF4005320468C
:10F0A80088BF76104FF0010B4FF0000888BFB340BF
:10F0B8000093009B5E009B00C3EB090A0493029B2C
:10F0C8002AFA03F303FA02FA4FF40072039304F0E6
:10F0D80041FC072384F8BFB184F8C0B1B24484F876
:10F0E800C231FE2384F8C181224684F8C331FF234C
:10F0F800C4F8C661414684F8C431284684F8C5314D
:10F108004AF65523C4F8CAA1A4F8FE312B681B6A35
:10F118009847002800F0B1804FF40072414620461D
:10F1280004F018FCEB2304F2FD12F421237076237B
:10F13800266463709023C4F84480A3704523C4F800
:10F1480048A0E3705823C4F84C8023714623A66571
:10F1580063714123C4F86490A3715423A4F86A80AE
:10F16800E371202384F86EB023726372A372009B4C
:10F1780084F8708023656365039BE3650423236635
:10F188004FF48073A4F86830092384F86C309DF834
:10F19800083084F86D30802384F86F3004F17703E9
:10F1A80003F8011F9342FBD14FF000094AF655239B
:10F1B800C846A4F8FE31A9F16A03012B06D9B9F1B2
:10F1C800700F1CBF14F8093003EB780809F1010926
:10F1D800B9F5007FEFD12B682246314628461B6AD5
:10F1E8009847002849D02B68224606F10C0128468A
:10F1F8001B6A9847002840D04A460021204606F15D
:10F20800010A04F0A7FB4AF6552306F1090904F29E
:10F21800FF1BA4F8FE31631E0593059B13F8012F0D
:10F228009B4502EB7808F9D12B68224651462846BF
:10F238001B6A984708B32B6822460AF10C01284636
:10F248001B6A9847C8B10AF1010ACA45E5D106F117
:10F258000B0A4FF400720021204604F07BFB059B4B
:10F2680013F8012F9B4502EB7808F9D12B68224649
:10F27800494628461B6A984738B91FB10B49384692
:10F28800F6F7EFFE4FF0000AF0E02B68224609F18E
:10F298000C0128461B6A98470028EED009F10103A3
:10F2A800534505D09946DAE7E9380020403900206F
:10F2B800231F04F5FE7243F8048F9A42FBD12B6892
:10F2C8002246514628461B6A98470028D5D02B6805
:10F2D800224609F10D0128461B6A98470028CCD020
:10F2E8001FB164493846F6F7BCFE009B4FF4007224
:10F2F800002120461E44039B4FEA830904F02AFBA1
:10F30800F82309F2072904F113022370FF214FEAB9
:10F31800592A234603F8011F9A42FBD14FEA99392B
:10F328004FF00008B8FBF9F309FB138323B91FB1A9
:10F3380051493846F6F795FE2B68224606EB080138
:10F3480028461B6A9847002897D0B8F1000F05D1C6
:10F358004FF400724146204604F0FCFA08F1010817
:10F36800C245DFD11FB145493846F6F77AFE029B00
:10F378004FF0010808FA03F8039B03F1070A4FEA64
:10F38800DA0A0AF2FF1B4FEA5B2BD845FFF475AF88
:10F398004FF40072002120464FF0000904F0DAFA19
:10F3A800072323702B682246049928461B6A494480
:10F3B800984700283FF461AFB9F1000F01D184F8F4
:10F3C800009009F10109CB45ECD11FB12C49384611
:10F3D800F6F747FE009B0198334403EB08094946BA
:10F3E800FFF7DFFD00283FF448AF019B9B68B3EBB4
:10F3F800482F3FF642AF1FB122493846F6F731FE93
:10F408004FF4007200212046002604F0A3FA81225E
:10F418000323C14484F820200222237062638222DD
:10F42800C4F838A084F84020019A52686365019BAB
:10F4380062649B68E665A3652B68224606EB0901B2
:10F4480028461B6A9847824600283FF416AF2EB913
:10F458004FF400723146204604F07CFA0136B0457C
:10F46800EAD11FB108493846F6F7FBFD504607B008
:10F47800BDE8F08FFF3800202F3600207C390020AF
:10F488000C39002023390020323900202DE9F041C1
:10F4980015460E4601F11E08AB8936F8024F43B9EE
:10F4A8006A68AB689A4204D1B4FA84F04009BDE8AE
:10F4B800F081284604F06AF804F060F9074620460F
:10F4C80004F05CF9874204D14645E5D10120BDE846
:10F4D800F0810020BDE8F0812DE9F84F90F8313037
:10F4E80082468946002B47D002F1FF380D46022795
:10F4F800002488449AF83030BB4237D3002239467A
:10F508005046FEF769FCB8B30378C12B34D10646E0
:10F5180000F11E0B234636F8024F73B104F5105262
:10F5280092B2B2F5806F27D29B021648C4F3090441
:10F538001840044304F580300CE004F520539BB2D6
:10F54800B3F5006F02D38CB1204603E0B3F5806FAA
:10F5580007D311E04246294604F083F830B1054646
:10F568000024B345D6D10137FFB2C3E70023C9EB66
:10F5780005002B70BDE8F88F002089F80000BDE871
:10F58800F88F00BF00FC0F0070B50B6800240D4613
:10F598004FF6FF764B608C810C61AB891BB96A68AA
:10F5A800AB689A4219D0284603F0F0FFB04212D057
:10F5B80004F0E4F8E30343EA540454FA80F4C4F38F
:10F5C8004E0343EAC433041214FA83F42B6901335B
:10F5D800A4B22B61E1E7002070BD2869AC82013834
:10F5E800FE288CBF0020012070BD2DE9F84F804611
:10F5F8009246894609B18C1E01E0D0F82044D8F81B
:10F6080030349C4228BF0024012304F00707C4F3C8
:10F61800C80B2646254603FA07F7FFB2D8F82C147C
:10F628000022404601EB153103F09FFE70B33B46C4
:10F638005946475C1F4205F101050DD1AA1B5245E9
:10F648000BD1B9F1000F04D1BAF1010F08BFC8F806
:10F658002064B01CBDE8F88F2E46AC4215D0D8F80F
:10F668003024954204D25B0013F0FF03E2D103E09B
:10F6780000264FF400713546013101234FF0000B8D
:10F68800B1F5007F1F46D4D3C8E70120BDE8F88F45
:10F698002DE9F84317468A1E0646D0F83004D119DA
:10F6A8009846814240D8D6F82034B8F1000F09D0E6
:10F6B8009A420BD8994209D9814228BF0021C6F83D
:10F6C800201403E09A4238BFC6F8202402F0070548
:10F6D8000123D6F82C14C2F3C80403FA05F501EB8C
:10F6E8001231EDB20122304601F1010903F03DFE6D
:10F6F800D0B103192A4600F500701978114214BFD9
:10F708000124002444450FD05140013F19700ED008
:10F71800520012F0FF02F0D101331446012249468B
:10F7280098421546E9D1DDE70020BDE8F8830120BD
:10F73800BDE8F88338B50D46D0F8381400F50470E4
:10F748006B6819402B689C1E90F8353204FA03F355
:10F7580003EB5123D0F81C12194403F006FE18B12C
:10F768006B68C3F30803184438BD38B5D0F8303493
:10F778000C46154601338B4202D24FF0FF3038BD9C
:10F78800D0F82414002200F5047001EBD41103F022
:10F79800ECFD0028F1D0A400C4F308040059286047
:10F7A800013018BF012038BD73B5064602AD0024EC
:10F7B80045F8041D2A4601993046FFF7D6FF002870
:10F7C80004DB04F10104F5D1204600E0002002B07A
:10F7D80070BD70B50D46D0F83844496806460C40EF
:10F7E800A3180A446A6090F845440934E4B223FA3D
:10F7F80004F474B12B7A23B12B6801332B60013CDC
:10F80800F7E72A4629683046FFF7AFFF0128F6D008
:10F8180070BD012070BD012938B50C46154601D8C8
:10F82800002038BDD0F8303401339942F8D8D0F8E8
:10F838002414012200F5047001EBD41103F095FDA6
:10F848000028EDD0A400C4F308040551012038BDF8
:10F858002DE9F34107460C460E4601AA21463846D3
:10F86800FFF783FFB0F1000801DA00251BE0002252
:10F8780021463846FFF7CFFF05460028F5D0621C21
:10F88800B8F1000F02D0019B9A4208D00023921BC6
:10F8980031463846FFF7FCFE0028E6D0019E019C61
:10F8A800B8F1000FD9D1284602B0BDE8F0812DE9A2
:10F8B800F04100240646D0F82C1400F504772546BC
:10F8C8000022384601F1010803F04FFD00B300F1B2
:10F8D800FF3E05F5805C1EF8011FFF2901D10834A1
:10F8E8000AE049B10822012319424FEA430318BF2D
:10F8F8000134013ADBB2F7D10835D6F83004854235
:10F9080002D3001BBDE8F08165454146E3D1D7E746
:10F91800BDE8F081F0B54FF0FF330446002587B00D
:10F928000846E3601146C4F81C3284F8445405AB19
:10F93800C4F8400404F50872606004F50477257083
:10F94800C4F8140284F8105202950195009503F04A
:10F9580047FD10F0FB0F01D100203CE0059E2A4630
:10F968003846314603F001FD05460028F4D01B490E
:10F978000522033006F01BF801460028ECD195F863
:10F988006C30092BE8D12B6D3344C4F824346B6DEB
:10F99800C4F82834AB6D1E44C4F82C64EB6DC4F86D
:10F9A80030342B6EC4F8343495F86D300125C4F822
:10F9B8002004204684F8453409332A4605FA03F31F
:10F9C800C4F83C34013BC4F83834FFF70EFE40233A
:10F9D800284684F8443407B0F0BD00BF50390020F1
:10F9E80010B50446D0F83414FFF7DEFE94F8453419
:10F9F8000933DBB2984010BD10B50446283003F037
:10FA08008EFC50B104F50E7003F089FC28B1206813
:10FA18000368BDE81040DB691847002010BD0246A6
:10FA280038B552F8105F04468068294601F0F3FDA6
:10FA380078B1A37815B943F0400305E00135226990
:10FA4800AA4202D023F04003A370A37863F07F0397
:10FA5800A37038BD2DE9F0410378044603F0200374
:10FA680003F0FF050BB1002635E042691B4B9A42B3
:10FA7800F9D8FFF7D4FF06460028F4D0A06805227D
:10FA8800216983792830023950F8147C99400F4451
:10FA9800394603F06AFC80460028E4D0294601254F
:10FAA8004FF4007203F056FFA3681A79AA420AD9E4
:10FAB80018684246E91903681B6A98470028D2D09B
:10FAC8000135EDB2F0E79A794FF40073934062691B
:10FAD80012FA83F363613046BDE8F081FFFD1F0031
:10FAE80010B5044680680A462830A16903F03DFC39
:10FAF80020B1A38803F00F0300EB431010BD70B5CD
:10FB0800047805460E4684B92422214603F022FFD4
:10FB1800AE60F379102B03D0202B06D1402300E0F0
:10FB2800202301202B70A87070BD002070BD38B54F
:10FB3800CB6804460D4623B98968BDE83840FFF70D
:10FB4800DEBF2422002103F005FF102301202370CB
:10FB5800A070AB68A360EB68236238BD2DE9F74F4E
:10FB68008378044689461646DD0776D50378180754
:10FB780003D5E36962699B1A07E0990608D5A3686B
:10FB88001A896369C3EB42139BB29E4228BF1E4683
:10FB980037464FF0000804F1100A002F41D02378AF
:10FBA800626913F0200FA068C2F308054FEA5221DA
:10FBB80002D0036A194424E090F8058001EA080895
:10FBC800BDB9B8F1000F14D122B95A064CBF036A67
:10FBD800236A49E01B0705D5A378590602D523698E
:10FBE800013341E05246216901F0B2FC002834DBC0
:10FBF80013D0A36821699A7902395B699140194445
:10FC08004144D4F808B0002D4ED1B7F5007F4BD34E
:10FC1800DBF83430994206D146E0237813F0700FB0
:10FC28001BD0F01B52E0B7F5806F2CD322787D0AE9
:10FC3800920606D49BF80420C8EB0202954228BF1E
:10FC48001546994212D84A1993420FD20BF128004F
:10FC5800019103F064FB019940B963784FF0FF30DC
:10FC680043F00203637031E02361C2E7DBF82C0044
:10FC78004A460368D3F810B02B46D8470028ECD082
:10FC88004FEA452B09E0DBF82C004A460368DB689D
:10FC980098470028E1D04FF4007B6369D944CBEB47
:10FCA80007075B44636178E700220BF1280003F043
:10FCB8005CFB0028D1D0C5F5007B41194846BB45FF
:10FCC80028BFBB465A4603F0ABFDE6E703B0BDE8E4
:10FCD800F08F73B501220DF10701044646690569E5
:10FCE800FFF73CFF0128666125610CBF9DF80700FE
:10FCF8004FF0FF3002B070BD436937B5C3F3431509
:10FD0800044605B169B901220DF107012046FFF744
:10FD180025FF40B2012801D0002008E063691F33A5
:10FD280000E02033A0686361383000EB451003B071
:10FD380030BD2DE9F0410446076900780E460028D9
:10FD480046D065698D4247D009B921613AE002077A
:10FD580003D5E36999423BD807E0830605D5A36834
:10FD68001B89B1EB431F33D82CE0D4F808E0731E8D
:10FD7800A1789EF80620490602F10902D2B223FAB8
:10FD880002F303D5226A134423611BE0691E21FA9A
:10FD980002F2934200D34DB942064CBFDEF8202050
:10FDA800226A22611D4604F1100809E09B1AF9E74E
:10FDB80042462169A068013D01F0CAFB002807DD21
:10FDC800002DF5D1A378666123F02003A37003E02A
:10FDD80027610020BDE8F0810120BDE8F081F8B579
:10FDE8000F4616460021242204461D4603F0B2FDA4
:10FDF800B868A68006F00F0600F138023B6AA060DA
:10FE080002EB4612E360D17A0E073FD401F01701E6
:10FE18002170D37A13F0180F9DF8183008BF41F0FD
:10FE28000801E37005F0030308BF2170012B08D017
:10FE3800022B04D053BB6B0528D4012302E0032313
:10FE480000E00223A370A3789F0703D5217811F05F
:10FE5800110F1BD105F008016E0543EA0103A370D9
:10FE6800436B918AA361538B43EA014104D589B15D
:10FE780001F011FC70B909E02162D369E3616B04F8
:10FE88000DD5E1692046FFF754FF40B900202070E6
:10FE9800A070F8BDA37863F07F03A370EFE701209B
:10FEA800F8BD2DE9F743037806460D469146BBBBDE
:10FEB8000B7813F0700F33D04C6914F01F042FD156
:10FEC800274600212846D5F81480FFF715FF38B3D8
:10FED80003782BB32E2B01D10024F2E7E52BFBD0BE
:10FEE800C27A02F0080E0EF0FF01BEF1000F0FD12A
:10FEF800C4B1421E0A30CB0143EA510112F8013F56
:10FF080053FA81F19042C9B2F5D18F4208D109E084
:10FF18000F2AE1D15A06D4D503F01F04477BD0E756
:10FF2800002007E000944B46C8F34F12294630469C
:10FF3800FFF755FF03B0BDE8F08310B5037804461A
:10FF4800DA061FD50021FFF7F4FE01212046FFF74E
:10FF5800D3FE10B9637853B114E003783BB1E52BB5
:10FF6800F3D02E2BF1D0C37A1B07EED40AE0082376
:10FF780020462370A37843F00203A370BDE8104025
:10FF880000F014BF002010BD37B503780446002BDD
:10FF980034D090F90230002B2ADA0121FFF7A0FDB6
:10FFA800054628B96378002043F00103637026E012
:10FFB8000378E52BF6D023781B0744BFE369C361B8
:10FFC800236A43831B0C83820E4B1B6863B10DF1BC
:10FFD80003020DF1060101A89847BDF804302B83F0
:10FFE8006B82BDF80630EB82A37803F07F03A37021
:08FFF800A068FFF701FD0028DD
:02000004600199
:10000000D4D000E0012003B030BD00BFE87A00206A
:1000100010B50446FFF7BCFF00232370A37010BD8A
:10002000F0B51F4695B0002306460C4601928DF8A8
:1000300008308DF809308DF80A30ADF83830037883
:100040000BB100203EE00B7813F0700FF9D013785D
:100050002F2B12D1019B1A782F2A02D10133019341
:10006000F8E7A1681AB93046FFF74DFD2AE002A86B
:10007000FFF749FD0028E4D002AC01AB0BAA0199BF
:10008000304600F04BFE0028DBD0019B1B789BB173
:1000900000230BAA2146304600F018FD0028D0D0DE
:1000A000354602AC0FCD0FC40FCD0FC42B683046C0
:1000B0002360FFF7ADFFDFE73B460BAA2146304642
:1000C00000F004FD15B0F0BD19B101F58961FFF72D
:1000D000A7BF0846704770B506460C46FFF758FFA5
:1000E000054608B900250EE000213046FFF7FCFC6C
:1000F0000028F7D0214600F1200350F8042B984245
:1001000041F8042BF9D1284670BD30B589B00D46B1
:1001100014466946FFF7DFFF28B1BDF810302B8089
:10012000BDF80E30238009B030BD30B589B00D4622
:1001300014466946FFF7CFFF28B1BDF818302B8071
:10014000BDF81630238009B030BD2DE9F0410B78A1
:1001500088B004460E4613F0700F1CD040F6022300
:1001600000F0B4FCB8B1012710252046A770257017
:10017000FFF774FC78B12369002120462362FFF762
:10018000DCFD2046FFF704FF28B139462046FFF783
:10019000ABFC034608B9002055E0C57202466F4625
:1001A00000F1200C6D461068083252F8041CBE465F
:1001B0006245AEE803007746F5D19F8A2021B3F867
:1001C0001A802E238DF800300023EA1801330A2B01
:1001D0005170FAD1A0680122216A8379283002394E
:1001E000994050F8143C194403F0C3F80346002822
:1001F000D1D0ADF81470AE4607460DF1200CADF825
:100200001A807246083703CA624547F8080C47F857
:10021000041C9646F5D12E2220338DF80120326A37
:1002200008AE110CADF81A20ADF814102A460833A8
:1002300003CAB24243F8080C43F8041C1546F5D132
:10024000A068FFF7DDFB08B0BDE8F081F0B51F4600
:1002500095B0002306460C460192ADF814308DF897
:100260002C308DF82D308DF82E300378002B3FD1B7
:100270000B7813F0700F3BD013782F2B0CD1019B10
:100280001A782F2A02D101330193F8E7A1680BA84D
:10029000FFF739FC60B30BAC01AB02AA0199304601
:1002A00000F03CFD20B3019B1B78DBB1002302AAC8
:1002B0002146304600F00AFC58B135460BAC0FCD54
:1002C0000FC40FCD0FC42B6830462360FFF7A0FE8C
:1002D000E1E76FB102AA21463046FFF736FF00285A
:1002E000EBD105E002AA21463046FFF72EFF00E0E1
:1002F000002015B0F0BD2DE9F04303789BB0002736
:10030000044613F0180F884691468DF820708DF83A
:1003100021708DF822708DF844708DF845708DF83D
:10032000467001D10020B3E082688B689A42F9D10F
:100330002646FFF72DFE11AD0FCE0FC50FCE0FC510
:100340003368394620462B60FFF7CEFB0028E9D002
:1003500003466A4600F120076D461868083353F8D3
:10036000041C1646BB4203C63246F6D1227808AEBC
:1003700002F0080202F0FF0352B140F601234A46A0
:1003800041463046FFF74CFE0028CBD0002707E05F
:100390004A4641463046FFF759FF0028C2D0109F19
:1003A0000E9B01212046A361BDF82430A3809DF857
:1003B0002330E3700B9BE36000238DF820308DF831
:1003C0002230FFF791FB0028ACD00DF10D0300F1B6
:1003D0000D020DF11D0153F804EB8B4242F804EBC2
:1003E000F9D1198811809B7893709DF80B30C372F6
:1003F000002F3CD0A068BB1E0022817928308B40A2
:1004000050F8141C194402F0B4FF00288AD000F1FF
:100410002003AE4600F1400C1868083353F8041C62
:100420007246634503C29646F6D13946A06801F08C
:1004300036F900283FF476AFA0680122216A83795B
:1004400028300239994050F8143C194402F091FFC9
:1004500000283FF467AF00F120032A46083303CA9F
:10046000B24243F8080C43F8041C1546F5D10023AA
:1004700011A8199302238DF8463008238DF84430D3
:1004800000F098FC00283FF44DAFA068FFF7B8FAE1
:100490001BB0BDE8F0832DE9F84F1C4603780646F3
:1004A0000F461B079DF828B09DF82C909DF830A0B2
:1004B0009DF8345002D40020BDE8F88FA2F2BC723F
:1004C0001FFA82F8B8F17F0FF5D8631E0B2BF2D814
:1004D0000BF1FF331E2BEED8B9F1170FEBD8BAF1A1
:1004E0003B0FE8D83B2DE6D8FFF752FD0028E2D0BD
:1004F00001213046FFF7F8FA0028DCD04BEA44141B
:100500006B1044EA4828FC0743EA4A131FFA88F8AC
:1005100043EAC92348BFA0F81280B9079BB207D5A8
:1005200015F00105A0F81080C38118BF642545733C
:100530007A0744BFA0F81880C382B068FFF760FA5A
:10054000BDE8F88F13B5837804469B0701D40020DB
:100550002AE0036A3BB3016989B102AA00238068DB
:1005600042F8043D00F0F8FF0028F0DB09D06FF0FE
:1005700070422169A06801F024F810B9E7E70193FF
:100580000162019949B963692046E361A37863F088
:100590007F03A370FFF7FCFC06E0A06801F07FF882
:1005A0000028F0D1D3E7012002B010BD2DE9F84FAB
:1005B0008378894604461546990740F18E801A07CC
:1005C0000AD46369DB439D4200F287802F464FF0D7
:1005D000000A4FF0FF3B46E0C169FFF7AEFB002881
:1005E000EFD17AE0A068C2F30808467916EA5226ED
:1005F0003DD0D4F808E021699EF8063002399940D0
:10060000DEF8143019443144B8F1000F48D1B7F581
:10061000007F6CD26269E3699A4243D2A37813F0F7
:10062000200F0CBF012205220EF1280002F0A1FECE
:10063000002852D0C8F5007640444946BE4228BF43
:100640003E46B044324603F0EFF8B8F5007F05D1DE
:10065000A068283002F067FE00283ED06369B144EC
:10066000BF1B334463616269002FBBD11CE0B8F14A
:10067000000FBED1216941B1A3785B0621D5E369A2
:100680009A421ED201312161B3E7236A33B9204671
:10069000FFF7C9F908B323692362AAE72361A8E732
:1006A0000122C1E70522BFE7E3699A4201D9E2616D
:1006B00002E02D4B1B68BBB1A37863F07F03A370EE
:1006C00012E004F1100200F047FF002805DB3FD1E3
:1006D0002046FFF7A8F900283AD16378002043F0BC
:1006E00001036370BDE8F88F2846BDE8F88FB7F5C1
:1006F000806FDEF83420DEF82C0014D39EF804302E
:100700009E1B7B0AB34228BF33468A424FEA4326E8
:1007100003D303EB010C624515D30268D2F82480A1
:100720004A46C04798E78A424A4608BF8EF828A042
:10073000036808BFCEF834B01B6A98470028CCD0B5
:100740004FF400768AE78EF828A0CEF834B0E4E7BC
:10075000D4F808E021699EF8063002399940DEF8A5
:100760001430194453E700BFE87A0020411E00F11D
:100770000A020020C30143EA500011F8013F53FA76
:1007800080F09142C0B2F5D1704710B549010446DE
:10079000FFF7D3FA28B120460021BDE81040FFF74B
:1007A000AFBA10BD2DE9F04F05468DB0164607468D
:1007B0008846994603AC0FCD0FC40FCD0FC42B68EC
:1007C00001252360336873600023B3814D451CD835
:1007D000C5EB080103A889B2FFF7D7FF834608B924
:1007E00000202AE04FF0000A5FFA8AF259463846A4
:1007F00000F0A4FDB38904464BB97268B3689A420D
:1008000005D1B0FA80F0400917E0012015E030462C
:1008100002F0C0FE0190204602F0B4FF019B0446A6
:10082000184602F0AFFF8442DAD10AF1010ABAF1A8
:100830000D0FD9D10135EDB2C8E70DB0BDE8F08F8D
:100840002DE9F04F05468DB016468A461F4603AC8B
:100850004FF0010B0FCD0FC40FCD0FC42B68002537
:1008600006F116002360A846FFF780FF3368814633
:10087000B5817360BB4528D8CBEB0A0103A889B2C8
:10088000FFF783FF002843D0059ABB4500F104041D
:100890004FF0000192F8283043F0010382F828302D
:1008A0000CBF4BF040035B4680F80C8080F80D9045
:1008B00003704FF00F03A0F81A80C372B38933B9E5
:1008C0007268B3689A4202D119E0012020E03046F4
:1008D000019102F05FFE0199042902D824F8030C6B
:1008E00003E00A2994BF2080608001310234C9B23C
:1008F0000D29E3D10BF1010B5FFA8BFBBAE725B1B0
:1009000001354FF6FF70EDB2E6E728460125E3E733
:100910000DB0BDE8F08F024600F120012DE9F04353
:1009200052F8153B2024876802F8014F9142FBD111
:100930001E782E3E18BF01261D4601332A782E2A26
:10094000FAD07B1EAB429E4607D800224FF0070C20
:100950004FF008091146904610E09EF80020013B38
:100960002E2AEFD1F1E72B782E2B0AD1AE450CD1F0
:100970004FF00A0C08214FF010090135BD42F2D3A7
:1009800044E0222B13D07C2B11D0A3F12A04052C98
:1009900001D82D2B0BD1A3F13A04052C07D9A3F1D3
:1009A0005B04022C03D9A3F121045D2C04D903F0CC
:1009B000C003802B13D124E0614507D9BCF10A0F95
:1009C00023D0AE4521D30EF1FF351AE0A3F1610427
:1009D000192C08D8203B49EA0202DBB209E0614544
:1009E000ECD85F230026A3F14104192C98BF49EAF3
:1009F00008084C1C0144E4B28B75062C03D804751E
:100A000001E00026B9E72146B7E70026837D202BC9
:100A100011D03EB118EA020F18BF02224275012020
:100A2000BDE8F083027D0123437510447E22827568
:100A30003122C275F3E70020BDE8F0832DE9F843C9
:100A400007460E460D7D62244FF07E0801F116091F
:100A500002F0A6FF032D80B228BF03252B1DDBB2B9
:100A600000F00F02F118013B0009092ADBB294BF24
:100A7000303237329D428A75F2D3731900213846DD
:100A800083F81680FFF759F901213846FFF738F946
:100A9000014628B97878B0FA80F04009BDE8F883BB
:100AA00003784BB1C37A1B07EED40B22484604F0FF
:100AB00073FE0028E8D102E00120BDE8F883601E43
:100AC00010F0FF04C4D12046BDE8F8832DE9F04FB3
:100AD0008BB00E46924603930B78069013F0700F7E
:100AE00001D1002014E1069B1B78002BF9D113697A
:100AF0000D220C33B3FBF2F3DBB202939AF81530FC
:100B00009B0700F00281029B03F1010B5FFA8BFB54
:100B10004FF0000900213046FFF70FF9C8460AF1EF
:100B200016034C464D46CDF81090CDF8149007931F
:100B3000776900213046C7F34F17FFF7E1F818B97E
:100B40007378002B60D0CCE70378E52B00D043B955
:100B5000002C08BFB9465C453CBF0134E4B223B960
:100B600052E05C4538BF002403E0E52B01D10025AD
:100B7000DEE72E2BFBD0C27A0F2A27D175B903F0FE
:100B80001F08029A4245D3D1590602D4DDF80880E5
:100B9000CEE7437B90461546049309E008F1FF3801
:100BA0005FFA88F84345E2D1437B049A9A42DED14A
:100BB000B8F1010FBCD1791C2B465246304689B2A0
:100BC000FFF7F0FD002808BF0025B1E71307CED4DA
:100BD0004DB1B8F1010F84D1FFF7C8FD049B8342EA
:100BE0007FF47FAF0CE00B22079904F0D5FD0028BD
:100BF0009ED19AF81530D80702D50123059397E7BF
:100C0000039B190579D56CE7039B9A057FF569AFBE
:100C100003F00303013B012B3FF663AF002C08BF39
:100C2000B9465C4502D3059BBBB91DE000213046A7
:100C3000FFF766F810B973784BB152E70134E4B2AC
:100C4000EFE7B3681B791C44E4B2A345EBD9304607
:100C5000FEF704FF0028F4D143E751463046FFF782
:100C6000EDFE00283FF43DAF0BF1FF355246304614
:100C7000EDB209EB05072B46BFB23946FFF7E0FDA1
:100C800000283FF42EAF39463046FFF77EFD04467C
:100C900000283FF426AF2022002102F05FFE5346D9
:100CA00053F8162F22605A6862601A8922819B7A53
:100CB000A3729AF8153003F018032373164B1B68C0
:100CC0007BB10DF123020DF1260109A89847BDF86B
:100CD00024302382BDF82630E3819DF823306373EE
:100CE00004E045F22143238223836382B26892F8B1
:100CF000283043F0010382F8283000953A46039BE0
:100D000031460698FFF76FF802E04FF0010BFFE65F
:100D10000BB0BDE8F08F00BFE87A0020F7B51446AD
:100D20001E46084601310378202BFAD00025204FBB
:100D30002060037843B32F2B26D001AA011D02F0B7
:100D4000DFFC88B3019AB2F5803F2CBF0223012358
:100D50007F2A1D4413D81F2A26D9D3B2A3F122011A
:100D6000C9B21D2903D827FA01F1C9071CD403F021
:100D7000BF033C2B18D05C2A16D02E2AD9D0202AAB
:100D8000D7D02561A060D4E72369013BFE2B0BD8A7
:100D9000024610F8013B202BFAD02F2BF8D03260FE
:100DA0002046FFF7B8FD00E0002003B0F0BD00BF13
:100DB00001210031F0B500238BB004468DF80430DA
:100DC0008DF805308DF8063083789A0717D5016ABB
:100DD00019B1806800F063FC88B101212046FEF75C
:100DE00083FE054658B1FFF7C1FCE5260023074600
:100DF0002E702370A370A068FEF702FE08B90020D1
:100E00002FE0E3786BB3214601A8FEF794FE00289B
:100E1000F5D00125E378AB42F1D3A18801A8491BA5
:100E200089B2FFF7B2FC0028E9D0C37A0F2BE6D1D4
:100E3000027802F01F039D42E1D1437BBB42DED129
:100E40000670A16891F8283043F0010381F828303A
:100E5000530603D5A068FEF7D3FD02E00135EDB2DD
:100E6000D8E70BB0F0BD0000486810B50C4658B18B
:100E70000B894A8901339BB29A420B8104D80349FA
:100E8000F5F7F3F800232381206810BD2F360020EA
:100E9000F0B5044687B00E46154600214FF40072A7
:100EA000406A02F05BFD206A10B12049F5F7DDF8D9
:100EB000636A03AAE0690393236AE1680493002349
:100EC0000131ADF814306B09ADF8163003680092AB
:100ED0006A1E9F6A164BB84708B9002024E0206AB2
:100EE00010B11449F5F7C1F8F822636A102E4FF0DB
:100EF000FF001A704FF001030CBF04220C22616A3C
:100F0000C85401339A42FAD1E069626A0368E16821
:100F10001B6A98470028E0D0E069E568A16803688B
:100F2000626A29441B6A984707B0F0BDFF38002069
:100F3000D1B900007C39002038B5446A4FF4007202
:100F400000210546204602F009FDEB2390222021D6
:100F5000237076236370234603F8022F04F10A02FC
:100F600003F8011F9342FBD14FF40073A4F80B3038
:100F700095F82B3063732B8DE38102232374F823C0
:100F800063752B69E361AB6923624AF65523A4F8C4
:100F9000FE3138BD70B504464FF400720021406A3E
:100FA00002F0DCFC656A2269216805F2BF1002F0DC
:100FB00015FBA369226905F2C31021681A44013A9E
:100FC00002F00CFB94F82A30002185F8C231236925
:100FD000E069C5F8C631A369626AC5F8CA314AF644
:100FE0005523A5F8FE310368BDE870401B6A184719
:100FF000F8B54FF480730446456AD0F814E090F8D1
:101000002B2043606368C3EB0E01B1FBF2F101F2E8
:101010000116360A700000F1A107BB420AD3DB1BA0
:10102000A66003F180062661A1F6F576B6F5704F4D
:1010300003D209E080336360E4E7206A002852D0DD
:101040002A49F5F712F84EE081330126E36000F1FA
:1010500021032685204601FB0233B3F5803FA361BF
:1010600034BF0423062384F82A30FFF793FF0028B7
:1010700039D02046FFF760FF4FF4007305F13502C9
:101080002021A5F81130A368EB82802385F8243055
:10109000292385F82630164BC5F8273005F12A0399
:1010A00003F8011F9342FBD1462385F836304123D4
:1010B00085F83730542385F83830312385F83930B6
:1010C000362385F83A30E069626A036821691B6A51
:1010D000984740B162682046E3681021D21ABDE803
:1010E000F840FFF7D5BE0020F8BD00BF56390020FC
:1010F00087D61200F8B54FF400530446456A0361E1
:101100004FF4804390F82B10436043696268981A4B
:10111000B0FBF1F000F18106F6094FEA460E0EF53C
:1011200000570937BA4203D202F500526260EDE778
:101130004FF6F473A660984207D8206A002800F0A2
:10114000A0805149F4F791FF9BE0A2F5005300FB0A
:1011500001222046CEEB03039BB2238503F5005307
:10116000E360A2F50053A361484B9A4294BF0B235E
:101170000C2384F82A30FFF70DFF002800F081804F
:101180002046FFF7D9FEA36805F1510220216B62CA
:101190000223EB6201232B8606236B86802385F8CE
:1011A0004030292385F84230394BC5F8433005F1EA
:1011B000460303F8011F9342FBD1462385F85230C2
:1011C000412385F85330542385F85430332385F870
:1011D0005530322385F85630E069626A0368216928
:1011E0001B6A984700284CD0E06921690368626A4D
:1011F00006311B6A9847002843D04FF40072002143
:10120000606A02F0ABFB234BE069C5F8FC31036870
:1012100021691B6A626A02319847002831D0E0696F
:1012200021690368626A08311B6A984748B31A4B00
:10123000E0692B6003F1FF53626A03F5005320332A
:10124000C5F8E4314FF0FF33C5F8E831C5F8EC31AB
:10125000036821691B6A0131984790B1E0692169EF
:101260000368626A07311B6A984750B1A26820463A
:1012700094F82B30202103EB4202BDE8F840FFF741
:1012800007BE0020F8BD00BF563900200004FB0057
:1012900087D61200000055AA5252614138B5036248
:1012A00004460B68C161426208469B69984700F298
:1012B000FF736061DB0A062B236006D8206A10B139
:1012C0001B49F4F7D2FE002038BD102B01D80223B1
:1012D00015E0202B01D8042311E0402B01D808236E
:1012E0000DE0802B01D8102309E0B3F5806F01D801
:1012F000202304E0B3F5004F94BF40238023B0F5D2
:10130000800F84F82B30204602D2FFF771FE01E0F7
:10131000FFF7F0FE0546206A25B138B10549F4F71C
:10132000A4FE03E00028CED00349CAE7012038BD5F
:101330006A3900207F3900208D390020042A04D822
:1013400001EB4201B1F8010070470A2A03D801EB12
:101350004201888870470C2A9ABF01EB4201C88875
:1013600000207047F8B50E4601781746D1B311F04A
:10137000600407D0012A35D92F23012033700023C0
:101380007370F8BD2146FEF7AFFB58B30546214602
:101390000822234608292C7804D1202C1ED01022A4
:1013A0002E240FE0A4F1410E0135BEF1190F07D82C
:1013B00090F80CE012EA0E0F04D02034E4B201E001
:1013C000202C08D003F1010E9C46774506D05FFA29
:1013D0008EF306F80C4001310C29DBD100221846AF
:1013E000F254F8BD00203070F8BD00002DE9F04F38
:1013F00000248BB003780746894690468DF8044058
:101400008DF805408DF80640002B5FD0C37813B9E6
:10141000FFF7A8FF5DE0014601A8FEF78CFB00285E
:1014200054D008F1FF384D460126C844FB78B3423A
:1014300047D3B98801A8891B89B2FFF7A6F983466B
:10144000002843D0C37A0F2B40D1037803F01F0349
:101450009E423BD123464FF0000A5FFA8AF259467A
:101460003846FFF76BFF044673B100F5105292B295
:10147000B2F5806F2AD29B021748C4F309041840C2
:10148000044304F580300BE000F520539BB2B3F524
:10149000006F01D320B914E0B3F5806F07D315E0D6
:1014A0004246294602F0E1F858B1054600240AF107
:1014B000010ABAF10D0F01D02346CEE70136F6B28C
:1014C000B4E70023C9EB05002B7002E0002089F887
:1014D00000000BB0BDE8F08F00FC0F00FFF786BFE7
:1014E0001368B3F5807F30B51C4628BF4FF4807475
:1014F00001EB4405A94207D231F8020B0028F9D1CB
:10150000506801305060F5E71B1B136030BD136855
:10151000802B30B51C4628BF802401EB8405A942EE
:1015200007D251F8040B0028F9D1506801305060FF
:10153000F5E71B1B136030BD10B503780446DB07CD
:1015400002D501F0F0FE30B1002304F11000237049
:101550004FF0FF33E36010BD012970B505460C461E
:10156000164602D84FF0FF3070BDC3699942F9D8D2
:10157000C379202B0ED18169022200F50E7001EB98
:10158000D41101F0F6FE0028ECD004F07F0450F8EE
:1015900024300FE0102BE5D18369C1F3072102222B
:1015A00000F50E70194401F0E4FE0028DAD0E4B230
:1015B00030F81430EA6993429ABF0120336000206A
:1015C00070BD012938B50C46154601D8002038BD3C
:1015D000C3699942FAD8C379202B0ED181690322BD
:1015E00000F50E7001EBD41101F0C3FE0028EDD020
:1015F00004F07F0440F824500FE0102BE6D18369FB
:10160000C1F30721032200F50E70194401F0B1FE69
:101610000028DBD0E4B220F81450012038BD2DE9B9
:10162000F341C46805460E4690468C4207D20C46EC
:1016300000270134EB699C4203D9CFB9EC6801273C
:10164000F7E7A64214D001AA21462846FFF784FFF7
:1016500000280DDBEDD0019B002BEAD107B1EC6037
:101660006FF0704221462846FFF7ABFF074608B9E6
:10167000002710E02EB96B6A002B0ADB013B6B627E
:1016800007E0224631462846FFF79BFF0028F2D1AB
:10169000EEE7C8F80040384602B0BDE8F08173B507
:1016A00005460C4601AA21462846FFF755FF061EAF
:1016B00001DA002014E0002221462846FFF781FFCE
:1016C0000028F6D06B6A002BA4BF01336B62EB6875
:1016D0009C423CBF04F1FF34EC60019C002EE1D140
:1016E00002B070BD7FB50446406A002821DA0023AD
:1016F00004F50E7025690393E36901330293FFF744
:101700001BFF024610B94FF0FF3012E0E37920686A
:10171000202B02AB0168019301D1074B00E0074B7E
:1017200000932B464E69A169B0470028EBD003987F
:10173000606204B070BD00BF77C0000049C0000007
:101740002DE9F0434FF0FF3300270446012600F156
:10175000280887B00D4691462160C771C660E162D6
:10176000436380F82870C4F83C12C0F8443280F813
:1017700038724046FFF7E0FE029702460197009755
:1017800005AB4946284601F02FFE10F0FB0F41D073
:10179000059D3A464046294601F0EBFD002839D028
:1017A000037C022B36D1B0F80B30B3F5007F31D17A
:1017B00032E0013A2ED0A6795B000136DBB2A67189
:1017C0008B42F6D1C38A23610BB9436A2361C18975
:1017D000B0F8112029442669228101EB4603A1615A
:1017E0005101236201F2FF1103EB6121B0F81330C4
:1017F000616103B9036A691A1944A379D9404B1C82
:10180000E3614FF0FF33636240F6F47399420BD803
:101810000C23E371002016E0417B0922A7714B1EC7
:10182000217163713346CBE74FF6F47399428CBF55
:10183000C36A10234FF00100266384BF2362202374
:10184000C4F84062E37107B0BDE8F083F8B5002446
:1018500006460D4684638F6BC46387B1014624201E
:1018600000F0A7F80470447084700446B063AD6B58
:101870000FCD0FC40FCD0FC42B68236015E0CB6BC9
:101880009BB10146382000F094F880F8317080F860
:10189000327080F83370F063EB6B03F1340253F86D
:1018A000041B934240F8041BF9D13046F8BD10B533
:1018B0000446806B10B1FEF7ABFB38B9E06B40B16A
:1018C000FCF7AAFA28B10023E36310BD0023A36349
:1018D00010BD002010BD2DE9F04104461746984682
:1018E0000D4611B90020BDE8F081FFF7E0FFD5F803
:1018F000806496B12146242000F05BF80022434624
:101900000270427082703A46A063D5F88014FEF7E8
:10191000DBFBE0B10120BDE8F081D5F88434002B79
:10192000E0D02146382000F044F8434680F831608A
:101930003A4680F8326080F83360E063D5F884146A
:10194000FCF72AFE0028E5D1E063BDE8F081A06342
:10195000BDE8F081F8B50D4604461746FFF7A7FF2E
:10196000AE6B8EB12146242000F023F800220270D5
:10197000427082703A46A063A96BFEF796FA08B1EE
:101980000120F8BDA063F8BDE86B88B1214638207E
:1019900000F00FF83A4680F8316080F8326080F845
:1019A0003360E063E96BFCF7FEFD0028E8D1E063FB
:1019B000F8BD084670470000F8B500260446C0F898
:1019C00088140146C0F880644FF49060FFF7F1FF7F
:1019D000012280F84464054680F8796480F87A64CE
:1019E00080F87B64C4F88404D4F88814FDF796FF6B
:1019F0001D4F58B105F589663046FCF70DFA2946AA
:101A00003046FCF733FA08B1184B22E00026214695
:101A100040F26C40C4F88464FFF7CBFF0122C6712A
:101A2000054680F8486480F8496480F84A64C4F840
:101A30008004D4F88814FFF783FE80B105F5896629
:101A40003046FEF7E5FA29463046FEF75CF830B13D
:101A5000074B1A6802B91D603C600120F8BD0020E8
:101A60003860C4F88004F8BD2C7B0020F07A002098
:101A7000307B002038B504464FF47A750020A5600D
:101A800020712073A064E0642046034D40F8105B91
:101A9000FFF721FF204638BD90070020C07D70472A
:101AA000407E7047036810B41C690123A4465DF8AA
:101AB000044B6047807E7047704710B504461C2178
:101AC00003F006FB204610BD1FB503686946DB6BBB
:101AD0009847B0B39DF8003013F0C0031FD19DF8B4
:101AE00006009DF8073000F003009DF80A209B00D7
:101AF00043EA80239DF8080043EA9010431C9DF8B8
:101B0000090000F00300400040EAD2109DF80520D3
:101B100002F00F021044073803FA00F011E0402BE6
:101B20000ED19DF80900431C9DF8070000F03F000E
:101B300003EB00409DF8083000EB0320800200E03A
:101B4000002005B05DF804FB70B5067E04466EB952
:101B5000051D284601F065FB3146A07D01F05FFBC5
:101B6000FF21284601F0BAFB0123237670BD38B56A
:101B7000037E04466BB1251D0121807D01F04FFBE2
:101B8000FF21284601F0AAFB284601F065FB00234F
:101B9000237638BD70B5037D0546012B0FD0067E38
:101BA0000EB9FFF7D1FF281D01F082FBB0F1FF0451
:101BB00018BF01242EB92846FFF7D9FF01E0002005
:101BC00070BD204670BD00002DE9F843184B044657
:101BD000884691461F681E46051DBFB2284601F083
:101BE00067FBFF28607607D133689BB2DB1BB3F538
:101BF000967FF3DD1D230BE0FE2801D0182307E0BC
:101C00004A464146284601F059FB607638B1252303
:101C10002046E375FFF7ABFF0020BDE8F8832846B8
:101C200001F046FB284601F043FB0120BDE8F883A4
:101C3000B47B00202DE9F0411F46037D04460D468C
:101C4000022B164602D103698B4208D0236829462D
:101C500020461B6D9847C8B10223256123750025D6
:101C6000BD4206EB452106D023682046DB6C984731
:101C700060B10135F4E723691D44637D25615BB1E3
:101C800023682046DB69BDE8F04118472046FFF78E
:101C90006EFF0020BDE8F0810120BDE8F0812DE954
:101CA000F0471F46037D04460D46022B1646DDF81D
:101CB000208002D103698B4208D023682946204640
:101CC0001B6D9847E8B102232561237505EB0609D2
:101CD0004D450BD041462846B8472368014620466B
:101CE000DB6C013598470028F2D10AE023691E44D5
:101CF000637D26615BB123682046DB69BDE8F04760
:101D000018472046FFF733FF0020BDE8F087012089
:101D1000BDE8F087F8B50A4B0E46071D1D681C4646
:101D2000ADB2384601F0C4FAFF2806D023689BB252
:101D30005B1BB342F5DD0020F8BD0120F8BD00BFFC
:101D4000B47B00202DE9F341037D04460D4601924A
:101D50002BB10368DB69984708B9FF2031E0237E87
:101D600013B92046FFF7F0FE25B14FF496712046D7
:101D7000FFF7D0FF261D0DF107070DF1030845F011
:101D80004001304601F0AAFA17F80119304601F077
:101D9000A5FAB845F8D1002D30464FF00B050CBF21
:101DA0009521872101F09AFA304601F081FA3046F8
:101DB00001F07EFA0306607603D5013D15F0FF05BC
:101DC000F5D102B0BDE8F08170B504460D46164667
:101DD00037210022FFF7B6FF324629462046BDE8EC
:101DE0007040FFF7AFBF00002DE9F04788B0044610
:101DF0004FF0000ADFF8889101AD84F818A084F84C
:101E000017A084F81AA0D9F8007085E80E009DF894
:101E100004009DF80560A075DDF8088001F0FCF96C
:101E20000121A07D01F0FBF9544B06F00106A360EF
:101E3000072386F00106E36005AB95E80700251D42
:101E400083E8070028460ECB01F0F4F966752046BA
:101E500084F814A00A26FFF777FE0121A07D01F087
:101E6000DEF9013EFF21284601F038FA16F0FF06A0
:101E7000F7D131460A26A07D01F0D1F90022204693
:101E80001146FFF75FFF0128824612D0013E16F08F
:101E9000FF0601D1012355E04FF4027AFD212846C7
:101EA00001F01CFA284601F003FABAF1010AF9D14F
:101EB000E4E74FF4D57208212046FFF743FF4307BC
:101EC0000ED402230426A376013E284601F0F0F941
:101ED000607616F0FF06F7D1AA2803D0062331E07A
:101EE00084F81AA023682046BFB29B6C984702284A
:101EF0000CBF4FF080460026324629212046FFF7CE
:101F000063FF824640B1D9F800309BB2DB1BB3F5CA
:101F1000FA6FF1DD172315E0236820469B6C984784
:101F2000022808D02046FFF722FE0723C4F80880C5
:101F30000120E3601FE052463A212046FFF702FFEE
:101F400030B112232046E375FFF711FE002012E0A6
:101F5000284601F0ADF900F0C000C028284604BFB3
:101F60000323A37601F0A4F9284601F0A1F928463D
:101F700001F09EF9D6E708B0BDE8F087801A0600A8
:101F8000B47B0020F8B500220E463A210446FFF744
:101F9000D9FE30B112232046E375FFF7E8FD00209B
:101FA000F8BD351D271D384601F082F905F8010DF1
:101FB000B542F8D12046FFF7DAFD0120F8BD38B56B
:101FC000154600220446FFF7BDFE10B11B23E37542
:101FD0000AE0294610222046FFF7F6FD054618B113
:101FE0002046FFF7C4FD03E000252046FFF7BFFDB4
:101FF000284638BD0A460921FFF7E1BF0A460A21F3
:10200000FFF7DDBF38B503680D4604469B6C984763
:1020100003284FF01201204618BF6D022A46FFF731
:1020200091FE30B10C232046E375FFF7A0FD0020A0
:1020300038BD012038BD2DE9F0411F46037D04461F
:102040000D46012B164602D103698B420AD0294660
:102050002046FFF7D7FF10B90020BDE8F08101232B
:10206000256123750025BD4206EB452108D04FF4BC
:1020700000722046FFF7A8FD0028EDD00135F2E7F9
:1020800023691D44637D25612BB123682046DB69EC
:10209000BDE8F04118470120BDE8F0812DE9F04787
:1020A0001E46037D04460D46012B1746DDF82080B1
:1020B000DDF8249002D103698B420AD029462046DC
:1020C000FFF7A0FF10B90020BDE8F08701232561CC
:1020D000237505EB060A55450DD04FF400723946BD
:1020E0002046FFF771FD0028EDD028464A463946C4
:1020F0000135C047EFE723691E44637D26612BB19C
:1021000023682046DB69BDE8F04718470120BDE899
:10211000F08710B500220C210446FFF713FE30B102
:1021200009232046E375FFF722FD002010BD20465D
:10213000FFF71DFD012010BD027D0021022A01755F
:1021400002D103685B6D1847012A01D1FFF7E1BF97
:102150000120704738B503680D4604469B6C9847CC
:1021600003284FF01901204618BF6D022A46FFF7D9
:10217000E9FD30B10E232046E375FFF7F8FC00209F
:1021800038BD012038BD7FB503680E466946044658
:10219000DB6B1546984780B39DF80A305A060CD47D
:1021A00003F03F039DF80B205B0043EAD2136A1C47
:1021B0003243134201D027231EE0A37E2021204674
:1021C000032B1CBF76026D023246FFF7BBFDC8B978
:1021D0002A4621212046FFF7B5FD024690B9262167
:1021E0002046FFF7AFFD68B942F210712046FFF7B5
:1021F00091FD054640B92823E37520460025FFF7E9
:10220000B6FC04E02623F7E72046FFF7B0FC28469B
:1022100004B070BD38B54FF416710446FFF77AFD6F
:10222000054620B1FD21201D01F058F801E01E23D4
:10223000E3752046FFF79BFC284638BD70B5041DAA
:1022400016460546204601F049F84FF40072314623
:10225000204601F048F8FF21204601F03FF8FF2119
:10226000204601F03BF8204601F022F8687600F0A5
:102270001F00052806D020232846EB75FFF777FCC2
:10228000002070BD012070BD38B50D464FF41671A9
:102290000446FFF73FFD10B92423E37505E02A4605
:1022A000FC212046FFF7CAFF18B92046FFF75FFC64
:1022B000002038BD036870B59B6C0D460446164679
:1022C000984703284FF01801204618BF6D022A4690
:1022D000FFF738FD10B10D23E3750AE03246FE2109
:1022E0002046FFF7ABFF054618B12046FFF73FFC3D
:1022F00003E000252046FFF73AFC284670BD10B4E5
:10230000447D1CB15DF8044BFFF7D4BF03685C6AE1
:102310000123A4465DF8044B60470000074B0021F1
:10232000074A9963186B106012681A639A6C22F05E
:1023300081029A64034B1970704700BF00002C4063
:10234000E47A0020B6860020064BC3F8CC01C3F81F
:10235000D001C3F8BC01C3F8C001C3F8C401C3F87D
:10236000C801704700801F40034B04481B6B184096
:10237000B0FA80F04009704700002C4001000F00C7
:10238000024B586A00F00100704700BF00002C406B
:10239000034B586A80F08070C0F30060704700BF44
:1023A00000002C40014B1878704700BFB686002013
:1023B000034B586A80F40060C0F3C020704700BF30
:1023C00000002C40034B586A80F48060C0F38020EA
:1023D000704700BF00002C40034B04481B6B1840A3
:1023E000B0FA80F04009704700002C4002007F11D5
:1023F0004FF47A7306225843224B596AA3F51033DF
:10240000D3F80031C1F3C22103F03F030131B3FB24
:10241000F2F21D4BB3FBF2F30122B3FBF1F10923FE
:1024200030B51401B1FBF4F4A04202D301241346E9
:1024300009E0013BFAD05200F3E7102C03EB020550
:1024400005D001342B46B1FBF3F5A842F5D34FF488
:102450007A70D20143430D4802F47F42B1FBF3F19D
:102460000B4B1960C16A21F47F2323F47F6343F48B
:1024700060231A43631E42EA0313C362436A1B07C5
:10248000FCD530BD00C00F4000EC695E00002C4060
:10249000BC650020014B1878704700BF9F3B0020AF
:1024A000014B1868704700BFE47A0020054B03F128
:1024B000100253F8040B934241F8040BF9D10120A8
:1024C000704700BF8B830020054B03F1100253F8C7
:1024D000040B934241F8040BF9D10120704700BF6F
:1024E0009B830020024B01201B680B60704700BFDC
:1024F000847A002070470000F8B50746064D01F0C9
:102500004FFA0646B847044620B101F049FA801B4D
:10251000A842F7D92046F8BD40420F002DE9F0410E
:102520000C4C0646DFF83080206001F039FA07468F
:10253000B047054650B101F033FAC01B404502D9FF
:102540000023236003E002F0D9FDF1E72060284674
:10255000BDE8F081E07A002040420F0010B504464B
:102560000C2102F0B5FD204610BD000008B500208A
:10257000FFF7EAFE084B47F2B80241F2B801C3F890
:10258000BC23C3F8C023C3F8AC23C3F8B013C3F80B
:10259000B423C3F8B82308BD00801F40054B1B7847
:1025A00033B1054B1B78002B14BF0320022070476A
:1025B00001207047127C0020177C002038B50446AB
:1025C00014480D46FFF798FFF8B9134BA1029D6020
:1025D00007D59A6CE1B222F0FF029A649A6C0A4322
:1025E0009A6424F0FF040C4D0C48EC60FFF784FF64
:1025F00058B92A6B0A4B1A601A682A631A68D207FC
:1026000003D51B6813F4702F01D0002038BD0120C2
:1026100038BD00BFE9CE000000002C40D1CE000044
:10262000E47A002008B5044B04481968FFF7C6FF98
:1026300008B1034B186908BD887A002000001A0D04
:1026400000002C4008B5FFF7EDFF80F48070C0F368
:10265000002008BDFFF7E6BF7FB5134B0D46196894
:10266000FFF7ACFFE8B1114B05F10F061A690092B4
:102670005A6901929A690292DB690393002323F05D
:10268000030404AA144403F003020133D10054F8F4
:10269000102C0F2B22FA01F206F8012DEFD10023A6
:1026A000EB7304B070BD00BF887A002000002C409E
:1026B000054B186810F0020005D01B68034818404D
:1026C000B0FA80F040097047E47A002000007F11E2
:1026D000F8B51D46930706460C46174600D12DB99E
:1026E00025221A4B1A704FF4FD7208E01848FFF7C4
:1026F00015FF38B10A22154B1A7040F2FD12154B26
:102700001A6020E00122144B2D041A70134A144B56
:102710002A40186042F40072124B1F605A60124A3D
:102720009A63124B1B780BB9610200E021463046D8
:10273000FFF744FF38B10E48FFF7F0FE18B9BDE8C7
:10274000F840FFF7B5BF0020F8BD00BF9F3B002059
:10275000ADD10000C4650020B68600200000FF1F38
:10276000E47A002000002C4002007F11177C00203A
:102770000DCF0000174A137813F0C00319D19079D8
:10278000D37900F00300917A9B0043EA8023107A0A
:1027900043EA9010431C507A527900F0030002F093
:1027A0000F02400040EAD1101044073803FA00F04D
:1027B0007047402B0BD1507A431CD07900F03F007A
:1027C00003EB0040137A00EB0320800270470020E7
:1027D000704700BF9B830020037ADB0708D50A4BB4
:1027E0001B6803B11847094B187860B1FFF72ABF7F
:1027F000074B1B780BB1FFF7EFBD064B586A80F013
:102800008070C0F300607047E07A0020117C0020E7
:102810001A7C002000002C4070B51646427A0D4606
:102820002AB10368DB699847044600284DD028493F
:102830008B7A03F0400202F0FF047AB903F03F0301
:10284000CA7A5B0043EAD213721C2A43134205D0B2
:102850002722204B1A7040F2EB2227E01E4B1B78F8
:102860000BB96D02760229461C48FFF7A7FE044605
:1028700028B90F22174B1A7040F2F32216E03146A6
:102880001748FFF79BFE044628B91022114B1A7017
:1028900040F2F6220AE000211248FFF78FFE0446BC
:1028A00038B911220B4B1A7040F2F9220E4B1A6004
:1028B0000BE00E48FFF720FE38B12822054B00241C
:1028C0001A704FF43F72084B1A60204670BD00BF6B
:1028D0009B8300209F3B0020177C002000001A20D3
:1028E00000001A2100001B26C4650020ADD10000A5
:1028F00010B50F4C23780BB9012010BD0D48FFF720
:10290000FBFD00230C4A2370116B0C4B19601968F6
:10291000116320B91A680A4B1340002BECD01F2218
:10292000084B00201A7040F28122074B1A6010BD3C
:102930001A7C002041CF000000002C40E47A0020E7
:1029400000007F119F3B0020C465002038B5174C64
:1029500000211748A36A23F48033A362FFF72EFEF9
:10296000054638B90922134B1A7040F24222124B25
:102970001A6019E01148FFF7D1FD40B10A220D4B52
:1029800000251A7040F246220B4B1A600CE0636A75
:102990009B0709D5616BA36AE26A23F4803342F096
:1029A0008062E2626163A362284638BD00002C4069
:1029B0000000DB0C9F3B0020C4650020F9CE000026
:1029C00038B50C46FFF794FF0546002830D0194B68
:1029D0005A6AD10507D49A6A22F480329A629A6AB6
:1029E00042F400329A629A6A134842F480329A6240
:1029F000FFF782FDA0B9231F0E4904F5FE744A6A51
:102A00005205FCD503F1400253F8040F9A420862C4
:102A1000FAD194421346F2D10122084B1A7007E012
:102A20002122074B00251A7040F2F732054B1A603D
:102A3000284638BD00002C402DCF00001A7C002015
:102A40009F3B0020C465002010B514480C46FFF7DA
:102A500065FD40B10A22124B00201A7040F25F421D
:102A6000104B1A6010BD104B9A6A22F480329A62A1
:102A70004FF400725A600D4B1B780BB9610200E0F5
:102A800021460B48FFF79AFD30B90E22044B1A700D
:102A900040F26B42034B1A6010BD00BFADD1000085
:102AA0009F3B0020C465002000002C40177C0020C4
:102AB00020003A19F8B507460C4615463E7AF60747
:102AC0001DD596070FD0CE18B44227D03B682A46B2
:102AD000214638461B6A984708B90020F8BD0134E2
:102AE00005F50075F0E70E48FFF7F2FDB0B90E22CC
:102AF0000C4B1A7040F251420B4B1A60F8BDCE18C5
:102B0000B4420BD03B682A46214638461B6A013442
:102B1000984705F500750028F2D1DEE70120F8BDE1
:102B200027003A199F3B0020C465002070B5037A46
:102B30001546ADF5007D0446DA070E4618D5AB07FD
:102B400006D029466D464FF40072684600F06CFED0
:102B500001232A4631461A48FFF7BAFD00282CD136
:102B60000D22184B1A7040F21942174B1A6024E0DC
:102B7000FFF7BEFE08B900201FE0637A022B02D1E6
:102B800063689E420FD023682046DB69984700287F
:102B9000F1D02368314620461B6D98470028EAD0C3
:102BA000022366606372236829462046DB6C9847DF
:102BB0000028E0D06368013363600DF5007D70BDCF
:102BC00001003A189F3B0020C4650020F8B5074675
:102BD0000C4615463E7AF6071DD596070FD0CE183F
:102BE000B44227D03B682A4621463846DB689847DE
:102BF00008B90020F8BD013405F50075F0E70E486E
:102C0000FFF766FDB0B90C220C4B1A704FF46472DA
:102C10000B4B1A60F8BDCE18B4420BD03B682A4665
:102C200021463846DB680134984705F500750028D1
:102C3000F2D1DEE70120F8BD37003A129F3B0020B9
:102C4000C465002038B504461A480D46FFF754FC09
:102C500028B10A22184B1A7040F29D1220E001227E
:102C6000164B21461A70164B164A1860164B174819
:102C70001D605A60164A9A63FFF7A0FC38B9042217
:102C80000D4B1A704FF4D272124B1A6038BD1248B5
:102C9000FFF744FC40B12522074B1A7040F2A712FF
:102CA0000C4B00201A6038BDFFF702FD0028F2D05F
:102CB00038BD00BFADD100009F3B0020B68600208C
:102CC000E47A00204000010000002C4011003A0688
:102CD00002007F11C46500200DCF00002DE9F043F4
:102CE000002301729F4F91B09F49A04DA04E4372A7
:102CF00005202B703B700B7033709E4BD3F8002176
:102D000042F08002C3F80021D3F8002122F03F02F4
:102D1000C3F80021D3F8002142F01802C3F80021C3
:102D2000D3F8002122F08002C3F8002103F510330C
:102D3000D3F8802042F00C02C3F880205A6A22F4B3
:102D400060525A62DA6942F48032DA615A6A42F4B5
:102D500000625A62FFF7F8FA874B88469A6C42F095
:102D600000429A64DA6A42F0807242F40042DA6207
